:1000000000800020BD0100006D7C0200397C0200F0
:10001000397C0200397C0200397C0200397C020004
:10002000397C0200397C0200397C02006D7C0200C0
:100030006D7C0200397C02007D9D0200819D0200E2
:100040006D7C02006D7C02006D7C02006D7C020004
:100050006D7C02006D7C02006D7C02006D7C0200F4
:100060006D7C02006D7C02006D7C02006D7C0200E4
:100070006D7C02006D7C02006D7C02006D7C0200D4
:100080006D7C02006D7C02006D7C02006D7C0200C4
:100090006D7C02006D7C02006D7C02006D7C0200B4
:1000A000D9370200E53702006D7C02006D7C02004A
:1000B0006D7C02006D7C02006D7C02006D7C020094
:1000C0006D7C02006D7C02006D7C02006D7C020084
:1000D0006D7C02006D7C02006D7C02006D7C020074
:1000E0006D7C02006D7C02006D7C02006D7C020064
:1000F0006D7C02006D7C02006D7C0200598B020059
:100100006D7C02006D7C02006D7C02006D7C020043
:100110006D7C02006D7C02006D7C02006D7C020033
:100120006D7C02006D7C02006D7C02006D7C020023
:100130006D7C02006D7C02006D7C02006D7C020013
:100140006D7C02006D7C02006D7C02006D7C020003
:10015000659F0200799F02008D9F0200A19F02000F
:100160006D7C0200098E02006D7C02006D7C020035
:100170006D7C02006D7C02006D7C02006D7C0200D3
:100180006D7C02006D7C02006D7C02006D7C0200C3
:100190006D7C02006D7C02006D7C02006D7C0200B3
:1001A0006D7C02006D7C02006D7C02006D7C0200A3
:1001B0006D7C02006D7C02006D7C0200564B4CF29F
:1001C000205210B51A804DF628121A8000BF00BFC9
:1001D00027F050FD514B4FF010621A60504A9A6060
:1001E000504ADA60504A136813F4807301BF4F49D4
:1001F0000B604FF4A85313604D4B4E491A7810070B
:1002000042BF1A7842F008021A704B4B2A221A7029
:100210004A4A4B4B8B4204D252F8040F43F8040B6A
:10022000F8E7484B484A0021934202D243F8041BA6
:10023000FAE7464A4648002350F8231042F82310B4
:1002400001336F2BF8D1434B434A802103F8011B44
:100250009342FBD1414B3D4A1A60414B8A221A70AE
:10026000A3F5805324225A70A0221A709A7991071C
:10027000FCD59A79D206FCD43A4A937903F00C0360
:10028000082B384BF9D103221A7140225A719A79FE
:100290009406FCD533498A79324B5006FBD5324A55
:1002A000324911600221516020221A709A7902F0BD
:1002B0000C020C2AFAD12E4B2E4A1A602E4B2F4AD2
:1002C0001A6000225A60072243F8042C2C4AC3F813
:1002D0000C2D62B628F008F9144B1B68DA0705D517
:1002E000284827F0C1FE284B284A1A60284B1B7863
:1002F0005B0609D5244C254B22689A4204D121483B
:1003000027F0B2FE002323602EF0D6F827F0B8FCC9
:100310002AF0B9F9FEE700BF0E2005403080044006
:10032000823F04000100002B10D0034014D0034092
:1003300002D00740208DFF1F00E007407C9803009B
:100340001C87FF1F208DFF1F14DAFF1F0082FF1F75
:100350000000000000E400E05FE400E008ED00E0E1
:100360000050064000400640448004400000030165
:1003700004800440C010050014E000E0FF76010096
:1003800000002020CA43BC621CE00340A5C3945A6D
:1003900000F00740FFFFFFFFFFFFFFFFFFFFFFFF32
:1003A000FFFFFFFFFFFFFFFFFFFFFFFFFFFFFFFF5D
:1003B000FFFFFFFFFFFFFFFFFFFFFFFFFFFFFFFF4D
:1003C000FFFFFFFFFFFFFFFFFFFFFFFFFFFFFFFF3D
:1003D000FFFFFFFFFFFFFFFFFFFFFFFFFFFFFFFF2D
:1003E000FFFFFFFFFFFFFFFFFFFFFFFFFFFFFFFF1D
:1003F000FFFFFFFFFFFFFFFFFFFFFFFFFFFFFFFF0D
:10040000FFFFFFFFFFFFFFFFFFFFFFFFDEF9FFFF23
:1004100010B5054C237833B9044B13B10448AFF33E
:1004200000800123237010BD208DFF1F00000000FD
:1004300078980300084B10B51BB108490848AFF382
:1004400000800848036803B910BD074B002BFBD0A0
:10045000BDE81040184700BF00000000248DFF1FBA
:1004600078980300208DFF1F0000000070B505681C
:10047000044628460E4627F047FB864203D0314605
:10048000284627F055FB204670BD2DE9F0418046F7
:100490000E4614461AB3012A02D100230B701EE047
:1004A00027F032FB01250746307097B1AC420ADDD8
:1004B00008EB050027F028FB0746192027F0FEFF70
:1004C00077550135F1E7002D03DD3544002305F8AC
:1004D000013C192027F0F2FF0120BDE8F081204601
:1004E000BDE8F0812DE9F04112491C4600AF90466D
:1004F000054629F0F8FEE31D23F00703ADEB030DDD
:10050000224640466946FFF7C0FF661EE8466C4635
:10051000C8EB04039E4208DD14F8011B284629F0AD
:10052000D5FF192027F0CAFFF2E72846BD46BDE8EF
:10053000F08100BF27210300F0B585B0002401AE93
:100540001046234609220F463146019402948DF845
:100550000C402AF035F830462EF06BF90130C5B268
:10056000E3B29D420AD93B19315D00936846FFF71B
:100570007DFF192027F0A2FF0134F1E7284605B0DE
:10058000F0BD27F07DBA70B5044608460D462EF042
:1005900050F923680246294620465B68BDE8704052
:1005A000184738B50546FFF7EEFF0446284629F000
:1005B00035FD204438BD38B50A220023054629F010
:1005C00051FD0446284629F029FD204438BD27F076
:1005D00057BA002070477047024A1368013313600E
:1005E000704700BF10B9FF1F024A536801335360C0
:1005F000704700BF10B9FF1F2C4B2D4A1B7810B558
:100600002C4C3BB12388C3F309035BB113889BB225
:1006100043B10AE02388C3F30903BBB113889BB23B
:10062000A3B129E02449002312E02188128889B26D
:1006300092B29202642392FBF3F391FBF3F203FB79
:10064000121383B91C4B1A786AB911E01A490123B5
:100650000B7013889BB223B1184B0978187827F0D8
:1006600089FD00232380238801339BB2238010BDA2
:1006700001221A70197813E02388128899B292B275
:100680009202642392FBF3F391FBF3F203FB121348
:10069000002BE8D1084A11780029E4D013701178B2
:1006A000064B187827F066FDDDE700BF28C4FF1F62
:1006B000C6C5FF1F18B9FF1FA9C6FF1F0AB9FF1F34
:1006C00010B5044629F02CFC204610BD10B5034B94
:1006D0000360044622F0ACF9204610BDB03203009E
:1006E00010B50446FFF7F2FF2046142129F0D7FF8A
:1006F000204610BD10B5034B0360044622F098F964
:10070000204610BDEC3E030010B50446FFF7F2FF93
:100710002046142129F0C3FF204610BD10B5034B1D
:100720000360044622F084F9204610BDC83C030053
:1007300010B50446FFF7F2FF2046142129F0AFFF61
:10074000204610BD10B5034B0360044622F070F93B
:10075000204610BD9C3A030010B50446FFF7F2FF97
:100760002046142129F09BFF204610BD27F0E0B958
:1007700038B50C46054627F0C7F9844205D0214616
:100780002846BDE8384027F0D3B938BD38B50C4607
:10079000C1F307210546FFF7EBFF0A2027F08EFE85
:1007A000681CE1B2FFF7E4FF0A20BDE8384027F0FB
:1007B00085BE10B5029C521AE41AA242A0EB0100B9
:1007C000C6BF04FB00000132604390FBF2F0184406
:1007D00010BD10B5029C521AE41AA242A0EB01000F
:1007E000C6BF04FB00000132604390FBF2F01844E6
:1007F00010BD10B50C4604220146204627F0BAF978
:10080000204610BD10B5C0F3072104464FF4D17047
:10081000FFF7ACFF0A2027F051FEE1B240F2A3102F
:10082000FFF7A4FF0A20BDE8104027F047BEF8B547
:100830000C460E1D0D46471A781927F065F905F884
:10084000010BB542F8D12046F8BD27F05DB9FFFF96
:1008500010B50B4C2378042B0DD94FF4CC70FFF757
:10086000F4FF0322212888BFFF20064927F0E2FC7D
:10087000054829F055FB23780133237010BD00BFD4
:10088000A0C5FF1FF16E0100408EFF1F08B540F2AA
:100890009710FFF7DAFF012127F09AFC40F297103A
:1008A000FFF7D3FF002127F065FCFA2027F006FEB2
:1008B00040F29710FFF7C9FF002127F089FC0020C4
:1008C00008BD38B50546FFF7C0FF0446681CFFF7B2
:1008D000BCFF0146204629F0C3FC00B238BD29F018
:1008E000E3BD29F0E5BD03685B68184708B5FFF76D
:1008F0004AFE08BD00230A2229F0B4BB29F0EDBB53
:1009000000230A2229F0AEBB9DF80010009129F0C7
:10091000EFBB38B5054629F0E0FB0446284629F030
:100920007DFB204438BD38B50546FFF7E9FF044696
:10093000284629F073FB204438BDFFFF002A10B47D
:100940000BDB074B541E9C4207D830235A43013A15
:10095000232A02D910BC29F09BBA002010BC704792
:10096000575555051FB50024B0F90C30B0F90A20D1
:10097000B0F90810029403240194B0F90E400094D9
:10098000406825F09BFA04B010BD0B8883834B8828
:10099000C3838B880384704730B502F11704013993
:1009A00000F117030444A34204D011F8015F03F8D7
:1009B000015FF8E780F8242030BD0022FF23828108
:1009C000438200F112024E3022F8023F8242FBD1F4
:1009D0007047FFFF10B5044622F056F8014B236024
:1009E000204610BD9C3A030010B5044622F04CF896
:1009F000014B2360204610BDEC3E030010B50446B9
:100A000022F042F8014B2360204610BDC83C030091
:100A100010B5044622F038F8014B2360204610BD83
:100A2000B032030070B586B08DE80F00194B9DF809
:100A300028601A78052A1D4607D06946164822F014
:100A400045FA011C18BF012100E000212B78032B7F
:100A50001ED1EEB11148FFF751FF009A10490F481F
:100A600029F0F3FA0DF107040DF10F0514F8012F29
:100A70000C490A4829F0E9FAAC42F7D10A4B9DF833
:100A800005201B680593059B0849044829F0DDFAF9
:100A900006B070BDDAC7FF1F38C5FF1F8C8AFF1F65
:100AA000582003005E20030058D8FF1F6420030075
:100AB0002DE9F74F40F21910FFF7C7FE092811D1B1
:100AC000C14BC24D01221A7108225A71C04A1A60E4
:100AD0000022AC5CBC4998180132082A0472F8D193
:100AE0000023D1E00A2859D1BA4CBB4E08236371C8
:100AF0004FF4DE63236033781B0103F0100323728D
:100B00003378DB0003F01003A37233789B0003F00B
:100B10001003237333785B000025012703F01003D3
:100B200025716572E5726573E573A373009794E8A8
:100B30000F00FFF777FFA94A657240F2F163236067
:100B40001378E5729B0003F03C03237213786573FE
:100B50001B099B00A3722573E573A573009794E8A6
:100B60000F00FFF75FFF40F2F26323603378657296
:100B700003F0100323723378E572FB4003F0100397
:100B8000A372337865739B0803F0100323733378E3
:100B9000E573DB091B01A37300974DE00B284ED1D1
:100BA0008F4F8C4C8F4D97F800800023A82623711F
:100BB000082306FB085863714FF4C263D8E90E019D
:100BC00023602CF01BFFC0F307202072D8E90E0130
:100BD0002CF014FF97F80180607206FB0858D8E9E2
:100BE0000E012CF00BFFC0F30720A072D8E90E0114
:100BF0002CF004FF97F80280E07206FB0858D8E951
:100C00000E012CF0FBFEC0F307202073D8E90E0183
:100C10002CF0F4FEFB78607306FB0355D5E90E015A
:100C20002CF0ECFEC0F30720A073D5E90E012CF0E8
:100C3000E5FE0123E073009394E80F00EFE20C2837
:100C400025D16449644800230B7108234B714FF48C
:100C5000E0630B60A5230B7203780478027812F02E
:100C6000010F027802F0010203F0040342F00402D3
:100C700004F0020442EA83020CBF0225002542EA86
:100C800084032B434B72012300930FC9C7E208284A
:100C900040F0FB804F4C524F524E60710023237145
:100CA0003B78A82202FB036393F89030FBB1DFF896
:100CB0003881D8F804504FF48E70FFF7C6FDADB2FE
:100CC00002234246D9B288420AD958F82310A942D1
:100CD00088BF52F8235003F1010388BFADB2F1E79A
:100CE00041F288335D43AB12AD14257263727B7899
:100CF000A82202FB036393F89030FBB1DFF8E88091
:100D0000D8F898514FF48E70FFF79FFDADB20223D3
:100D10004146DAB290420AD903F16502013358F82C
:100D200022E0AE4584BF51F82250ADB2F1E741F266
:100D300088335D43AB12AD14A572E372BB78A82271
:100D400002FB036393F89030FBB1DFF89C80D8F886
:100D50002C534FF48E70FFF778FDADB2022341465D
:100D6000DAB290420AD903F1CA02013358F822E0FC
:100D7000AE4584BF51F82250ADB2F1E741F288335D
:100D80005D43AB12AD1425736373FB78A82202FB9D
:100D9000036696F8903083B3134ED6F8C0544FF4E0
:100DA0008E70FFF752FDADB202233146DAB29042A7
:100DB0001CD903F22F12013356F82270AF4284BFC0
:100DC00051F82250ADB2F1E774C5FF1F8FC5FF1F68
:100DD00001C0CC1CB4C5FF1FF9B8FF1FDD8EFF1F7B
:100DE00001B9FF1FF88EFF1F18CAFF1F41F2883399
:100DF0005D43AB12AD14A573E3734FF4C863236076
:100E000001230093A84D94E80F00FFF70BFE05F1B6
:100E100008062B46002203F8012F9E42FBD1A34F68
:100E2000A3483A7890F800E040F2416302F00F02E4
:100E3000236041F28831531C91FBF3F20EF00F0353
:100E400013FB02F39BB263721B1223723B7802788E
:100E50001B09013391FBF3F1130913FB01F39BB25F
:100E6000E3721B12A3720123009394E80F00FFF7B3
:100E7000D9FD002305F8013FB542FBD140F24263A2
:100E800023608C4B1B7823739DE0012840F0A980E0
:100E9000894C8A4900230822237162712372884A8F
:100EA0006372A372E372237363730B78A82000FB51
:100EB0000323894693F890709046EFB1814E756890
:100EC0004FF48E70FFF7C1FCADB202233246D9B2A7
:100ED00088420AD956F82310A94288BF52F82350F5
:100EE00003F1010388BFADB2F1E741F288335D43FE
:100EF000AB12AD142572637299F80130A82202FB7F
:100F0000038898F890605EB3DFF8B881D8F89851FC
:100F10004FF48E70FFF799FCADB202234146DAB26E
:100F200090420AD903F16502013358F822E0AE4538
:100F300084BF51F82250ADB2F1E741F288335D43EE
:100F4000AB12AD14A572E3725FB95E4ED6F898513C
:100F50004FF48E70FFF779FCADB2022331461CE0EE
:100F60005FB3584F7D684FF48E70FFF76EFCADB2E3
:100F700002233A46D9B288420AD957F82310A94227
:100F800088BF52F8235003F1010388BFADB2F1E7E7
:100F9000AD102573002ED8D10FE0DAB290420AD9F5
:100FA00003F16502013356F82270AF4284BF51F855
:100FB0002250ADB2F1E7AD10657340F26663236075
:100FC0003C4B1B78A373404D2B78E37301230093B4
:100FD00094E80F00FFF726FD2B780133DBB22B706E
:100FE0001FE102282ED1314F314E334B39783578FD
:100FF000082201F00F015A7140F26C7241F2883000
:101000001A604A1C90FBF2F105F00F0212FB01F28C
:1010100092B25A7212129A72264A1278DA723A7898
:1010200031781209013290FBF2F00A0912FB00F24A
:1010300092B200241A7312121C711C725A739C73A0
:10104000DC732EE003280ED11B4B0821597140F2AE
:1010500002611960FF2119721649002208781A717D
:101060005A72987217E0052830D1134B0821597134
:1010700040F2F97119600F49087800F00100187208
:1010800008780978C1F380010022C0F3400099720A
:1010900007491A7158720978D9721A735A739A7378
:1010A000DA730122B9E000BFBBC5FF1FDE8EFF1F50
:1010B000DD8EFF1FF9B8FF1FB4C5FF1F01B9FF1F69
:1010C000F88EFF1F18CAFF1FDC8EFF1F062840F096
:1010D0009A80554C554FDFF86881DFF868A10823E6
:1010E00063714FF4C8632360514B1A7802F0010218
:1010F00022721A78C2F3400262721A78C2F3800236
:10110000A2721A78C2F3C002E2721A78C2F3001215
:1011100022731A78C2F3401262731A781B78DB09C3
:10112000E373C2F38012012300262671A273009399
:1011300094E80F00FFF776FC40F2416323602546F8
:101140004FF0A8094FF0650B16F8083009FB037340
:1011500093F89030E3B14FF48E70FFF776FB0021E7
:10116000002200230BFB06FC01315FFA81FE704573
:1011700008D90CEB010E5AF82EE012EB0E0243F1E7
:101180000003F1E7013892FBF0F21312237262724E
:101190000136042E04F10204D6D10123009395E810
:1011A0000F00FFF73FFC40F242632B60214B002110
:1011B00003F1080203F8011F9342FBD11E4E1F4C9E
:1011C0003278207802F00F02531C41F2883191FBF3
:1011D000F3F200F00F0313FB02F39BB22B721B120E
:1011E0006B72337822781B09013391FBF3F11309F9
:1011F00013FB01F39BB2AB721B12EB720123009342
:1012000095E80F000BE007280BD1074B00221A715D
:101210004FF4407101225A71196000920FCBFFF711
:1012200001FC03B0BDE8F08FB4C5FF1FF88EFF1FAF
:10123000F9B8FF1FBBC5FF1FDE8EFF1FDD8EFF1F2E
:1012400001B9FF1F18CAFF1F2DE9F347C04CC14F5A
:10125000C14E3B78082161714FF4D0712160BF49C4
:101260000878884601284FF0400161720BBFE921E0
:10127000B321A172A1720CBF0321102103F00F034F
:101280000022E1721033FE21E37322712272217376
:101290006173A2730023009394E80F00FFF7C2FB71
:1012A0004FF4207301202360FFF7CFFAFF28054693
:1012B00000F06A813378012B40F06681A84AA823A8
:1012C00003FB0025D5E90E010022A64B2CF0BEF849
:1012D0002CF06CFB00B2C5B2C0F307200023FE2245
:1012E000012123726272A572E07223736273A1738B
:1012F000E273009394E80F00FFF794FB4FF422731E
:1013000023603378012B0ED19749984B0022D1E905
:1013100000012BF0E9FE0022954B2CF0C1F92CF0D6
:101320006DFBC0B200E0C72092490A78894602F0FE
:10133000FF031AB90D222272607210E00B78012BA4
:1013400001D1702308E00B78022B01D18F2303E039
:101350000B78032B0CD1E923237260720023A37254
:10136000E37223734D236373FF23A373BF23E373DC
:10137000002694E80F000096FFF754FB0122A272AA
:101380007D4AE6724FF0FE0A4FF42873107823600E
:10139000642280233146CDF800A063722673667301
:1013A000A673E673FFF705FA207294E80F00009623
:1013B000FFF738FB4FF46073236058236372FD23FB
:1013C000E37207232373F023267284F80AA0637361
:1013D000A67384F80FA094E80F000096FFF722FB95
:1013E00099F800105A4D634A4FF49063236001F05E
:1013F000FF0351B996222A722C22AB72EB722B7327
:101400006B73AB736A72BA2328E01378012B0AD18D
:10141000E8232B722C236B72AE72EE722E736E73F6
:10142000AE73C4231AE01378022B0AD161232B7206
:101430002C236B72AE72EE722E736E73AE734D23ED
:101440000CE01378032B0AD11B232B722C236B7215
:10145000AE72EE722E736E73AE733723EB7300238E
:10146000009394E80F00FFF7DDFA4FF491632360D7
:101470003B78424A364D03F00F030F2B14BFDBB20B
:101480000E237821D25CE1720B322272FE2262724C
:10149000A27222731B0100226273A273E373009293
:1014A00094E80F00FFF7BEFA4FF49463236098F8B6
:1014B0000030012B4FF0B2032B7205D110226A725B
:1014C000AB72EA722B7305E011226A72EA72AB7298
:1014D0002B7310226A73AB73EA73002594E80F0034
:1014E0000095FFF79FFA4FF4B1632360082323723E
:1014F00078236572A372E57225736573A573E5732E
:1015000094E80F000095FFF78DFA3B780133DBB2CA
:101510003B703B7803F0FF020BB9194B1A70194A64
:1015200013780133DBB213701378032B07D999F8C2
:1015300000300133DBB289F800300023137099F8D2
:101540000030032B3AD90B4B00221A7036E000BF53
:1015500074C5FF1F2CC5FF1FFAB8FF1FF18EFF1FB8
:10156000F88EFF1F00001040D091FF1F0000484080
:101570000000E83F3C8EFF1FBCC4FF1F4E3203003B
:10158000E18EFF1F3D8EFF1F3378022B13D00D49D4
:10159000A82303FB0511D1E90E0100220A4B2CF010
:1015A000C7F918B1FF2D04D0002005E06020FF2509
:1015B00094E6602092E6612005468FE602B0BDE821
:1015C000F08700BFF88EFF1F00407F4008B54FF442
:1015D000CC70FFF73AF9002126F0FAFD4FF4CC70F9
:1015E000FFF733F9012126F0C5FD0A20BDE80840C8
:1015F00026F064BF0B79037130B58B6883600B46AE
:1016000000F11A0413F80C2F027300F10D0213F805
:10161000015F02F8015B9442F9D1CB69C36130BD2F
:1016200010B5042894BF044603242146084822F03C
:10163000BDF9032C074A084B15BFF0214FF4A071E8
:101640001180118014BF4FF4A072F0221A8010BDD7
:101650005CC6FF1F0888FF1F4488FF1F2DE9F0416B
:10166000044690B003200F46FFF7DAFF012C25D186
:10167000974B98481B6804930499974E974DFFF732
:101680003FF997499348FFF731F9002332785C1C02
:10169000DBB29A420FD9A822022102FB0353D3E9FD
:1016A0000E238C480091FFF72FF98D498948FFF7E9
:1016B0001DF92346EAE78B498648B4E0022C40F046
:1016C000B480894B1B78FF2B40F0AF80804E874958
:1016D00033680293029B0A689A1A854B18784EF673
:1016E000602343439A4202D9FF2F00F0A5800024D3
:1016F000804B04AA03F1080C1546186859689646F1
:10170000AEE80300083363457246F6D1186899883D
:10171000DFF804829B79CEF80000AEF804108EF852
:10172000063098F80030FF2F18BF3B4630338DF855
:101730001930BCB170496748FFF7D8F898F8001025
:101740006448FFF7D7F86D496248FFF7CFF829469C
:101750006B4820F02BF808B16A4900E06A495D48FF
:10176000FEF71FFF69481FF090FE98B929466448AC
:1017700020F010F8132300282A46614908A808BF62
:1017800001241FF0C3FF08A96048FFF733FF08A832
:101790001FF038FEFCB15E495C484F4DFFF7A6F8DC
:1017A00000242B78E1B2994204F101040FD2002207
:1017B00008A819F067FB08A9544828F00FFC08A8EE
:1017C00028F051FD46495148FFF790F8E9E74549AF
:1017D0004E48FEF7E6FE4D481FF057FE28B333682B
:1017E0000893089949483C4E3C4DFFF789F83C491D
:1017F0004648FFF77BF8002332785C1CDBB29A4244
:101800000FD9A822022102FB0353D3E90E233F483C
:101810000091FFF779F832493C48FFF767F8234613
:10182000EAE730493948FEF7BCFE3A4B1878FFF733
:10183000F7FE10B0BDE8F08133680393364D039B8B
:101840000B602B780133DBB2092B00D900232B70FE
:101850002978DFF8D8804FF4D070FEF789FF2F4841
:1018600022F0C0F909224FF6E0738DE80C00322116
:101870001F230122294824F0C9FA0121274822F018
:101880003CF90124002302223621244888F8004034
:1018900023F00CFC0021214822F035F920491F4893
:1018A000FFF724F829781D48FFF724F81D4A1E4940
:1018B000B2F90020B1F900101848002323F0F6FB1C
:1018C0000021164822F01FF9002388F800300FE7A6
:1018D00058D8FF1F8C8AFF1F2AC4FF1FF88EFF1FD6
:1018E000D8200300272103000F88FF1F30C5FF1FEA
:1018F00064C5FF1F9A200300772003008B2003009C
:1019000038D5FF1F92230300662B0300F4C4FF1F8A
:101910008F2003002A88FF1F4788FF1F5CC6FF1F18
:101920009D2403004488FF1F0888FF1FCEC5FF1FAA
:101930002DE9F04F814689B06848694D694F884666
:10194000002122F0E0F80121644822F0D6F80320BB
:10195000FFF766FE0B2444F2082301930094BC2396
:10196000012246215D4824F051FA46F22C330193BE
:1019700000940F2301223721584824F047FA00230E
:1019800002223B21554823F091FB57495348FEF76B
:10199000ADFF2C782CB1FF2C08BF3C78013CA4B2E1
:1019A00000E0FF24514A0392702606FB09264644B4
:1019B00046F22C3A337E4948A34214BF53464FF4B3
:1019C000FC634FF00B0B0193012233234B21CDF825
:1019D00000B024F01BFA002302224D213F4823F0DF
:1019E00065FB3B780822E1B204A819F04BFA04A980
:1019F0003A4828F0F3FA04A828F035FC327E2B7818
:101A00003648CDF800B09A4214BF53464FF4FC63F9
:101A1000019301223323832124F0F8F900230222C9
:101A200085212E4823F042FB3B782978082204A820
:101A300019F028FA04A9294828F0D0FA04A828F0B7
:101A400012FC2C78FF2C06D0264B1B78013B9C42C5
:101A500003D0013402E0002400E0FF24039A1F4871
:101A6000702303FB0929C84446F22C3698F8183035
:101A70000B25A34214BF33464FF4FC63019300953A
:101A800033230122BB2124F0C1F900230222BD210E
:101A9000124823F00BFB3B780822E1B204A819F0AE
:101AA000F1F904A90D4828F099FA04A828F0DBFB05
:101AB0008DE860000F230122F321084824F0A6F9E5
:101AC00000230222F721054823F0F0FA08490348D1
:101AD000FEF70CFF09B0BDE8F08F00BF5CC6FF1F2A
:101AE000A0C5FF1F2AC4FF1FA9200300B8BCFF1F09
:101AF000AB200300013808B5052810D8DFE800F056
:101B0000050305090709522104E0062102E0D2215C
:101B100000E0C6210648BDE8084025F033BCD221CC
:101B2000034825F02FFC034B00221A7008BD00BFAC
:101B300014C5FF1FF08EFF1F10B5074A0023702148
:101B400001FB0324D8B294F858401CB10133112B87
:101B5000F6D1FF2010BD00BFB8BCFF1F38B5074D40
:101B60000024281990F858301BB1FF2200211FF0E3
:101B700027F87034B4F5EE6FF3D138BDB8BCFF1F51
:101B800010B58CB01B49684628F0ADFB5323009A72
:101B9000194904A81FF0BAFD04A91848FFF72AFD47
:101BA00004A81FF02FFC00242046FEF74EFE01344F
:101BB00002461349114828F048FAB4F5BE7FF3D124
:101BC00010490E48FEF792FE4FF4C8742046FEF707
:101BD0003CFE013402460A49084828F036FAB4F5BA
:101BE000167FF3D105481FF044FC684628F03BFB04
:101BF0000CB010BDAD20030038D5FF1FF4C4FF1F8B
:101C00005E200300BE2003000D4B03600B790371BF
:101C10008B6883600B7B037303460A4A30B543F835
:101C20000D2B01F1190401F10D0252F8045B43F888
:101C3000045BA242F9D112781A70CB69C36130BD3E
:101C40007C920300608303001B4B73B501220446A2
:101C5000014600201A7019F0EDF810B1174B1B78EF
:101C6000DBB9174B1B782BB32146012019F0E2F8A2
:101C700000B32146022019F0DDF8D8B90121204631
:101C800019F0C4F80F4A1378013313700E4B1B6818
:101C900001930E4B019A1A600CE00D4B14201D6845
:101CA00028F0F9FC0646FEF795FE3146284620F05E
:101CB00087FFD6E702B070BDFBB8FF1F4388FF1F48
:101CC0002DC5FF1FAEC7FF1F58D8FF1F28D5FF1F08
:101CD000A4D7FF1F2DE9F347384EA82202FB006767
:101CE0008246D7E90E4500293ED097F89130FF2B68
:101CF00008D002FB0361D1E90E01D7E926232BF0BE
:101D00002BFED0B1D7E91689204642464B462946DC
:101D10002BF022FE30B9D7E91223204629462BF0BA
:101D200011FE50B100220023404649462BF0F6FD3B
:101D300018B95046FFF788FF16E0A82303FB0A6393
:101D400093F8A12082B193F8A2206AB11C4A1D48E1
:101D5000126801921C4A019912680078891A64225B
:101D600010FB02F2914222D8A82707FB0A67D7E9A5
:101D70001423204629462BF0F9FD10B1C7E914457C
:101D800019E0D7E91089204642464B4629462BF0F8
:101D9000CFFD30B900220023404649462BF0BEFD5E
:101DA00048B1A82303FB0A66C6E9104503E00022F8
:101DB00083F8A220D8E702B0BDE8F087F88EFF1FB5
:101DC00058D8FF1F2DC5FF1F28D5FF1F73B5144618
:101DD00003EB430203EB8203CA1805B200230C2075
:101DE0008DE809000E46052312B229460B4824F05F
:101DF0000DF8FF2C0FD004EB440204EB82020B2100
:101E00004FF6E07332448DE80A0012B205232946EA
:101E1000024823F0FBFF02B070BD00BF5CC6FF1F8D
:101E2000022938B50346084605D1FF222C21FFF7C9
:101E3000CDFF002038BD1D4A1D491278A82404FB9F
:101E4000021494F86840012C14BF0B240D24013CAB
:101E500003B918B3A34203DB01280CD100241EE010
:101E600020B95C1EE4B2042C0AD114E0012804D18C
:101E70005C1CE4B202E00028F3D01C46042C0CD019
:101E8000072C0CD1A82505FB0212516840F6FF7201
:101E9000914204D008B9013C00E00134E4B222468A
:101EA0002C210220FFF792FF204638BDA0C5FF1F5E
:101EB000F88EFF1F2DE9F0430B88FF2B89B00546F4
:101EC0000C4617460CD14888092809D8874B8A88C0
:101ED000C0B21870864B1A70FFF7A2FB002001E118
:101EE0002389844E092B0ED1834A142303FB052337
:101EF00001221A7440F2AB10FEF7A7FC7F4B18705A
:101F00001B78A38154E00B2B3CD16389092B04D1AE
:101F10007B4B7C4A1B78DBB205E00A2B0AD1784B5D
:101F2000794A1B78DBB21278934211D00023A38147
:101F3000E28113E00B2B05D1714B1B78FF2B65D091
:101F4000002364E00C2B09D16D4B1B78FE2BF6E7C8
:101F50000122A2816D4A9BB21380E3816C4B93F8FE
:101F60000080B8F1FF0F0FD0654B1A78642A0BD8A8
:101F700018782BF0F5F9674BA82202FB0838C8E95E
:101F80000E0101E0052B13D13A78002A40F09F8022
:101F900070236B43F2544FF0700808FB05684FF054
:101FA000000988F8089038462CF043FC08F80090A7
:101FB000702303FB05666389ADF818300125A389FA
:101FC000ADF81A3006A9E38986F858503046ADF8C6
:101FD0001C30FEF7DAFC0020A3886288218802907A
:101FE000207A0190E088009030461EF025FE23897B
:101FF000112B0ED10320FEF728FC474B1B788342A0
:102000005BD908A92A4601F80C0D51E00123A381F0
:10201000A4E70B2B2FD163890E2B14D13F4F3B78B4
:1020200003F0F002A37B13433B70397840F2C510F4
:10203000FEF79EFB3B7803F00F033384384B1B788D
:1020400003F00F0315E00F2B37D1344FE2893B78B3
:1020500003F00F0343EA0213DBB23B70397840F21E
:10206000C510FEF785FB3B781B0933842C4B1B788E
:102070001B0973841FE005AF7BB92A4A10680590DD
:102080000E3434F8021FFF29DAB204D0F9540133B8
:10209000042BF6D11A46394614E0072B0DD12846F9
:1020A000FEF7D3FBFF2808D08DF814002A463946E6
:1020B0003046FEF771FC284614E008A9238A01F88F
:1020C0000C3D01223046FEF767FC01200AE038464D
:1020D0002CF0AFFB02467020394600FB05602CF067
:1020E000C5FB58E709B0BDE8F08300BF2A88FF1F91
:1020F0001288FF1FB8BCFF1F1CB9FF1FF18EFF1F06
:102100000BB9FF1FF8B8FF1FEEC9FF1FC6C5FF1FA1
:102110000D88FF1FF88EFF1F2AC4FF1FDE8EFF1FD2
:10212000DD8EFF1F081E03002DE9F04FB14DDFF8D3
:10213000CCA2002687B00C4600F1FF3900F1BF08A1
:102140003746AB4619F8013F3B2B40F07081092F11
:1021500004D10F2E40F296800F2695E02EB37B1E01
:10216000172B22D8DFE813F0180024004F00590085
:10217000630070007A00840021009F00A900B30072
:10218000BE00C800D200DC00E600F400FE0008013A
:1021900013011D012B014C011022002102A82DF07A
:1021A00041FAA82303FB045358600023202235E1A1
:1021B0001022002102A82DF035FAA823C0B203FB9B
:1021C00004530228187201D1012208E003280BD021
:1021D000042801D1022202E0072803D10522864B00
:1021E0001A70E2E7082802D1834B1870DDE709284E
:1021F00001D10622F3E70A2801D10722EFE70B28D5
:10220000D3D10922EBE70A22002102A82DF00AFA15
:10221000A82303FB04535872C7E70A22002102A82F
:102220002DF000FAA82303FB04539872BDE70A229D
:10223000002102A82DF0F6F9A823003003FB045377
:1022400018BF0120D872B0E71022002102A82DF09B
:10225000E9F9A82303FB04531873A6E71022002111
:1022600002A82DF0DFF9A82303FB045318619CE7B3
:102270000A22002102A82DF0D5F9A82303FB04535C
:10228000187592E7002E90D0A8236343E8183246D1
:1022900002A9153001932CF0E9FA019B2B441E444E
:1022A0000023737581E7002102A82DF021F9A823EE
:1022B00003FB0453C3E90A0177E7002102A82DF0CC
:1022C00017F9A82303FB0453C3E90C016DE70A22A5
:1022D000002102A82DF0A6F9A82303FB045383F8DC
:1022E000680062E7002102A82DF002F9A82303FB91
:1022F0000453C3E91C0158E7002102A82DF0F8F8A7
:10230000A82303FB0453C3E91E014EE7002102A8E2
:102310002DF0EEF8A82303FB0453C3E9200144E7A2
:10232000002102A82DF0E4F8A82303FB0453C3E91D
:1023300022013AE70A22002102A82DF073F9A8230E
:10234000003003FB045318BF012083F890002CE7F2
:10235000002102A82DF0CCF8A82303FB0453C3E905
:10236000120122E7002102A82DF0C2F8A82303FBE6
:102370000453C3E9160118E70A22002102A82DF030
:1023800051F9A82303FB045383F891000DE70021C2
:1023900002A82DF0ADF8A82303FB0453C3E92601DE
:1023A00003E70A22002102A82DF03CF9A8230030FF
:1023B00003FB045318BF012083F8A000F5E60A22AE
:1023C000002102A82DF02EF9A82303FB04530028B6
:1023D00014BF0122002283F8A1201EBF9AF800300A
:1023E00001338AF80030A82303FB04B3002283F8EA
:1023F000A220DAE6F88EFF1F00B9FF1FBFC7FF1F3C
:102400000A22002102A82DF00DF9A823003003FBB9
:10241000045318BF012083F8A300C6E602A9CA54DA
:1024200001330F2BFAD10137FFB200262FE10A2B1F
:1024300004D00D2B02D0192F40F01F81A448A823EF
:1024400003FB040240F6FF755168A94241D1537A5B
:102450000BB9A04B15E0012B01D19E4B2EE0022BB6
:1024600002D19C4B9C7004E1032B02D1994BDC7090
:10247000FFE0042B02D1974B1C71FAE0052B02D12F
:10248000954B1C70F5E0062B01D1944BF9E7072B17
:1024900001D1934BF5E7082B01D1924BF1E7092BC2
:1024A00001D1914BEDE70A2B01D1904BE9E70B2BC2
:1024B00001D18F4BE5E70C2B02D18D4B5C70D8E03E
:1024C0000D2B01D18B4BDCE70E2B40F0D2808A4BD9
:1024D000D7E740F6FE75A94240F0B880117A062988
:1024E00040F0C780517A41B94FF420735360022302
:1024F000537293720026814F0AE001290DD14FF4E7
:10250000207369A7D7E9006753600523537291725E
:10251000C2E90A6700260027A9E0022902D14FF488
:10252000227313E003290DD14FF43073744F5360BD
:1025300000260123C2E90A67537293725CA7D7E9A8
:10254000006794E004290CD14FF460736D4F536021
:1025500000260123C2E90A675372937200266A4F6C
:1025600085E005290FD14FF4727353A7D7E90067AF
:102570005360002353720123C2E90A67937250A784
:10258000D7E9006773E0062903FB04030DD14FF47C
:1025900084625E4F5A60022200265A720122C3E909
:1025A0000A679A7200265A4F4DE05A7A072A04D1D8
:1025B0004FF484625A6003222BE0082A0DD14FF4B5
:1025C0008462504F5A60042200265A720122C3E9E5
:1025D0000A679A7200264C4F35E0092A0AD14FF457
:1025E00090625A6004225A7201229A722EA7D7E989
:1025F000006724E00A2A06D14FF4B1625A6004222F
:102600005A72012217E00B2A0DD14FF4B1625A60C1
:102610000722404F5A7200260122C3E90A679A72C4
:1026200000263D4F0FE00C2A23D14FF494625A60EC
:1026300006225A72022224A7D7E900679A72C3E9D8
:102640000A6700260027C3E90C6712E040F6FD7315
:1026500099420ED14FF4B1632E4F536000260723E9
:10266000C2E90A6753722C4F012393720026C2E914
:102670000C67A82303FB040410E0A3F12102592AEC
:1026800005D806AA3244013602F8103CF6B2C1451C
:102690007FF458AD0E4AA82303FB0424606807B0FA
:1026A000BDE8F08FAFF30080000000A09999D93FFA
:1026B0000000000000F08BC0000000C07268E93F1D
:1026C00000000040DF6759C000000040E17A843F0D
:1026D000F88EFF1F01B9FF1F4988FF1F4688FF1FA3
:1026E0000788FF1F0B88FF1F0D88FF1F4888FF1FEB
:1026F0003F88FF1F0288FF1F0E88FF1F0000D03F8A
:1027000000001C400000E83F000048C00000E03F1F
:10271000000049C00000F03F00004EC02DE9F04F1E
:102720000246BDB072B6532304A8A1491EF0EEFFC5
:1027300004A81EF0AAFE30B19E4FDFF8ACA24FF005
:102740000008B946CEE062B69B499C48FEF7CEF839
:1027500027E1A826DFF874B299496643BD19002322
:1027600058468BF800302CF05CF82B7A062B06F1DB
:10277000100640F0BF803E440536EB7A01962A7D74
:102780000092904922460CA82CF000F80CA958465B
:102790002CF020F8A82303FB04948B4994F86820BC
:1027A0000CA82BF0F3FF0CA988482CF013F8D4E9FF
:1027B0001C012BF043F90CAB0822012125F0D0FAC3
:1027C0000CA982482CF006F8814980482CF002F8C8
:1027D000D4E91E012BF032F90CAB0822012125F0BF
:1027E000BFFA0CA979482BF0F5FF794977482BF00F
:1027F000F1FFD4E920012BF021F90CAB08220121D3
:1028000025F0AEFA0CA971482BF0E4FF70496F482F
:102810002BF0E0FFD4E922012BF010F90CAB0822D9
:10282000012125F09DFA0CA968482BF0D3FF6849D7
:1028300066482BF0CFFF94F8902066490CA82BF047
:10284000A5FF0CA961482BF0C5FFD4E912012BF0BC
:10285000F5F80CAB0222012125F082FA0CA95B48A5
:102860002BF0B8FF5A4959482BF0B4FFD4E91601B0
:102870002BF0E4F80CAB0222012125F071FA0CA92F
:1028800052482BF0A7FF94F891204F490CA82BF049
:102890007DFF0CA94D482BF09DFFD4E926012BF0BC
:1028A000CDF80CAB0222012125F05AFA0CA94748B9
:1028B0002BF090FF94F8A31094F8A13094F8A02086
:1028C00000910CA844492BF061FF0CA93F482BF064
:1028D00081FF3E4904A8FEF709F804A81EF02BFD6D
:1028E00008F101089AF800305FFA88F4A3423FF635
:1028F00030AF4FE06A6839490CA82BF047FF0CA9AC
:1029000058462BF067FF297B6B7A2A7A0291E97A85
:102910000191A97A00910CA831492BF037FF0CA93D
:1029200058462BF057FF2A692C490CA82BF02EFF94
:102930000CA958462BF04EFF2A7D26490CA82BF0F7
:1029400025FF0CA958462BF045FFBA190532254939
:102950000CA82BF01BFF0CA958462BF03BFFD5E928
:102960000A012BF06BF80CAB0822012125F0F8F9D5
:102970000CA958462BF02EFF154958462BF02AFF7C
:10298000D5E90C012BF05AF80CAB0522012125F0FA
:10299000E7F9FBE604A81EF0CEFC04A81EF069FDD2
:1029A00062B604A81EF02EFD3DB0BDE8F08F00BF5A
:1029B00038D5FF1FF88EFF1FC02003008C8AFF1F31
:1029C000D7200300DA20030017210300EBC6FF1F06
:1029D000D8200300182103001C210300F920030064
:1029E00000210300102103002AC4FF1FF0B5354B5E
:1029F0001C7891B007460E46002C60D008230A22AE
:102A000031496846FDF76EFD0622694604A827F0A5
:102A100021FE2E4908A827F066FC08A904A827F083
:102A2000F6FD054608A827F01EFC04A827F01BFCAD
:102A300065B906232A46694608A827F0EBFD08A9D0
:102A4000684627F0C5FC08A827F00DFC204904A81B
:102A500027F049FC694604A8FDF741FF1D4B1B7890
:102A6000012B0CBF1C491D4904A8FDF73AFF049D2A
:102A70001B4901232A4608A81EF048FE9FB11EB13B
:102A80001848FFF74BFE0AE008A81EF0DFFC30B143
:102A900008A81EF064FCC0B227F0C6F8F4E708A846
:102AA0001EF0E7FC02E02846FFF738FE08A81EF0FB
:102AB000A9FC04A827F0D7FB684627F0D4FB2046E2
:102AC00011B0F0BD33D5FF1F34C5FF1F4D260300E5
:102AD00028210300A8C6FF1F2E2103003321030075
:102AE00038D5FF1F382103002DE9F0438DB00E4685
:102AF0001746984608AC544D0C2800F28280DFE857
:102B000000F0071B232B333B434B535B636B73007A
:102B10004E49204627F0E7FB46F22C33029314205F
:102B20002823009300FB065001943C23424639467B
:102B300017F0F8FF204682E00DF11009434948469E
:102B400027F0D1FB424956E00DF110093F494846B4
:102B500027F0C9FB3F494EE00DF110093B494846BB
:102B600027F0C1FB3C4946E00DF1100937494846C2
:102B700027F0B9FB39493EE00DF1100933494846C9
:102B800027F0B1FB364936E00DF110092F494846D0
:102B900027F0A9FB33492EE00DF110092B494846D7
:102BA00027F0A1FB304926E00DF1100927494846DE
:102BB00027F099FB2D491EE00DF1100923494846E5
:102BC00027F091FB2A4916E00DF110091F494846EC
:102BD00027F089FB27490EE00DF110091B494846F3
:102BE00027F081FB244906E00DF1100917494846FA
:102BF00027F079FB2149204627F075FB4FF4FC6351
:102C00000BE00DF110091149484627F06CFB1C49F7
:102C1000204627F068FB4FF6E07303931420282327
:102C2000009342463C23394600FB06500294CDF8FF
:102C3000049018F01CF8204627F015FB484627F0B2
:102C400012FB0DB0BDE8F0831CB9FF1F4721030044
:102C500051210300572103005F2103006721030076
:102C600072210300762103007E21030087210300E7
:102C70008D210300952103009B210300A321030064
:102C8000AB21030038B50D460B49044627F02BFB5A
:102C90000DB90A490AE0092D01D1094906E00A2DBA
:102CA00001D1084902E0072D03D10749204627F04A
:102CB00097FB204638BD00BFB3210300B7210300B6
:102CC000BB210300BF210300C3210300F7B5002A85
:102CD00046F22C360C4618BF4FF4FC668A1C0623BD
:102CE000411C054600930196032312B209B2134812
:102CF00023F08CF86B1D04F108011BB2621C09B2B1
:102D000000910196194612B20C4821F089F927B2B8
:102D1000AB1D09341BB224B23A4619468DE8500067
:102D2000064821F07DF9EB1D1BB28DE850003A46B4
:102D30001946024821F074F903B0F0BD5CC6FF1FCC
:102D40002DE9F34146F22C330D4604464FF6E0716F
:102D5000002A0CBF1A460A46671C09236E1C07345A
:102D600024B236B24FF00008019200932AB201B2A9
:102D70003FB21048073523F049F82DB223463246BA
:102D800039468DE840010B4821F04AF92346324686
:102D900021468DE82001074821F042F98DE8200105
:102DA0003B4632462146034821F03AF902B0BDE8DD
:102DB000F08100BF5CC6FF1FF0B5032087B0FEF7AF
:102DC0002FFC00214C484D4E20F09DFE01214A4829
:102DD00020F093FE484820F005FF00240C238DE8E6
:102DE000180022460F232146434823F00FF833787A
:102DF000032B4BD140F2AD10FDF727FD002845D045
:102E00003F4F3D886D083E3DEDB2E30229199BB26C
:102E10000134009300220C23C9B23748A4B223F036
:102E2000F9F8202CF1D1398849080C204FF4784367
:102E30001E398DE8090000223C2309B22E4822F0F9
:102E4000E5FF3C8864083D34E4B20025EB02611BD9
:102E50009BB2009300220C23C9B22748013523F00E
:102E6000D9F8202DF2D13C8826496408053C02A8F7
:102E700027F039FAA4B205230093234802AB0222BB
:102E8000214618F065FB02A827F0EDF91F4C3078B9
:102E9000FEF7C6FB23780B2B2CD01D4B1A78003283
:102EA00018BF012201211420FFF74AFF194B01210D
:102EB0001A782320FFF70AFF0A2246F22C338DE806
:102EC0000C00012211460D230B4822F09FFF002326
:102ED00002220521084822F0E9F82378092B05D9B8
:102EE000022200231146044822F0E0F8217802482B
:102EF000FDF700FD07B0F0BD5CC6FF1F2A88FF1F6D
:102F00000888FF1FCB210300B8BCFF1F0A88FF1FE2
:102F10002DC5FF1F4388FF1F07B5002A0CBF4FF4C4
:102F200078434FF4FC630193072300930AB2042310
:102F300001B2034822F06AFF03B05DF804FB00BF52
:102F40005CC6FF1F012808B503D0022803D104493D
:102F500002E0044900E004490448FDF7C7FC08BD4D
:102F6000DE210300D6210300E52103005CC6FF1F1C
:102F70002DE9F84306460F46DDE9080190469946DB
:102F80002AF0B0F80022002304460D462AF0C6FCC1
:102F9000E8B942464B46304639462AF0A3F8DDE907
:102FA0000A2306460F46DDE90C012AF09BF802468B
:102FB0000B46304639462AF049FA22462B462AF07B
:102FC0006FFBDDE90A232AF08FF8BDE8F883DDE91D
:102FD0000A01BDE8F883FFFF2F4B37B501221A70B5
:102FE00000242E4B054621462D481C7022F0E2F8A5
:102FF000FFF7E2FE012D07D12A4B224623F81420C9
:103000000134112CFAD11BE0022D19D1264B244892
:10301000B3F900304FF6FF7201920C220092214664
:1030200022F0F4FE23460F22DC211D4822F03EF858
:1030300021461B4820F067FD1C491948FDF756FC46
:103040004FF6FF71164820F05EFD194B1B78042BDC
:103050001FD1134820F0C6FD0321114820F04DFD7B
:10306000002314220A210E4822F020F84FF6FF71A7
:103070000B4820F048FD0F490948FDF737FC0A21AD
:10308000074800233C2222F011F80B490448FDF7C1
:103090002DFC03B030BD00BF4288FF1F0DB9FF1FDC
:1030A0005CC6FF1F2EC4FF1F0888FF1FED21030011
:1030B000DAC7FF1FF2210300FD21030073B504B23C
:1030C0000DB20023164621462A460E4821F0EEFF97
:1030D0000D4B1B7803F0FF0293B90A23214601929E
:1030E00000932A461E23074822F090FE074B05480E
:1030F0001A783241D30754BF05490649FDF7F6FB5C
:1031000002B070BD5CC6FF1FCEC5FF1FECC4FF1F21
:1031100013220300162203002DE9F34107B20FFA30
:1031200081F800231446394642461A4821F0BEFF72
:10313000194B1B785BBB194A194D115D2B5D9942E8
:1031400004D0631CD25CEB5C9A4202D1154B1B7815
:10315000EBB100260A238DE8480042463946282371
:103160000C4822F053FE295D0A483346102226F00F
:1031700079FF01340C490748FDF7B8FB295D054884
:103180003346102202B0BDE8F04126F06BBF02B01A
:10319000BDE8F0815CC6FF1FCEC5FF1FFAC9FF1F47
:1031A000ECC4FF1F4288FF1F4D2603002DE9F04F9E
:1031B0004E4F4F4D4F4B00268DB080460C463E7013
:1031C000F2B2052A18D8DFE802F0030817170D122B
:1031D0002978C80710D501210DE0297889070BD57A
:1031E000022108E02978C80606D5032103E02978E2
:1031F000890601D5042139701978DFF8F8B0002963
:1032000040F074813C48297890F800E0DFF8E090C5
:103210008EEA0101314111F0010F824640F03D81FB
:1032200036490978002940F03881013604F10A0254
:10323000072E92B201D01446C2E79BF8003003F08B
:10324000FF06002B40F0528108F11E073FB215B275
:1032500033462A4639462A4821F028FF99F800309B
:103260001B0607D5254B1B7803F0FF02002B40F00F
:103270001B8116469BF8002002F0FF03002A40F055
:1032800035810FFA88FB1E482A46594621F00EFF69
:1032900099F8010066B12AF0DBFC1A492AF02CFDEE
:1032A00019492AF01FFC2AF07DF806460F4631E046
:1032B000C0EBC0006523A0F56070584340F2EB13EB
:1032C00090FBF3F02AF05CF80022002306460F463C
:1032D0002AF02EFBE0B900220C4B304639462AF08A
:1032E00045FBB8B10026094F14E000BFE4C7FF1F3B
:1032F000ECC4FF1FCEC5FF1FFAC9FF1F4288FF1F86
:103300005CC6FF1F96434B3F9643CB42000059409B
:103310000026002799F801209AF801309A4240F0DF
:10332000D280744B1B78002B40F0CD8004F1140147
:10333000022289B24046FFF7EFFE04F11E0104228B
:1033400089B24046FFF7E8FE6B4D04F1280189B2CF
:1033500006224046FFF7E0FE2978FF292DD0674B73
:103360001B788B4229D9664E6248A82707FB016E5D
:10337000DEE90E23007807900120069005200590D5
:103380004FF0000C04F13C00CDF824C080B24FF6A1
:10339000FF7CCDF820C00490CDF80C800291DEE9CE
:1033A0001801CDE90001574819F00AFC2B7807FBFA
:1033B0000363D3E90E01C3E918016978FF292ED010
:1033C0004E4B1B788B422AD94D4E4A48A82707FB03
:1033D000016EDEE90E23007807900120069005209B
:1033E00005904FF0000C04F14600CDF824C080B2E7
:1033F0004FF6FF7CCDF820C00490CDF80C800291F0
:10340000DEE91801CDE900013E4819F0D9FB3A4B3D
:103410005B7807FB0363D3E90E01C3E918010120C0
:10342000FDF713FAFF2861D0344B1B7883425DD936
:103430002B7883425AD0304B5B78834256D0304E43
:103440002C4FA82505FB00614FF0000ED1E90E239B
:1034500050343F78CDF824E04FF6FF7ECDF820E0E1
:1034600007974FF0050E0127A4B2CDF814E0069798
:103470000494CDF80C800290D1E91801CDE9000147
:10348000204819F09DFB3846FDF7DFF905FB006089
:10349000D0E90E23C0E9182328E0214640460B93CB
:1034A000FFF70CFE0B9BC0E60A23019600932A4609
:1034B00019233946144822F0A9FC14491248FDF793
:1034C00015FA0126D6E64FF000090A238DE8080216
:1034D0002A461E2359460C4822F098FCCDF800904D
:1034E00032463B460848FDF70FFA1FE70DB0BDE82E
:1034F000F08F00BF4288FF1F2888FF1F2AC4FF1FCC
:10350000F88EFF1FB8BCFF1F5CC6FF1F77270300A4
:103510002DE9F04F9E4B9F4C1B7813F0FD0087B0B8
:1035200001D1207014E09C4A1278C82A15D9DB0713
:1035300013D59A4B187880B9994B1B78FF2B0CD177
:10354000984B05221A70984A137843F001031370C0
:10355000904B187007B0BDE8F08F944B1A78012A91
:103560001D4629D01B78042B16D1914B914A5B78CC
:1035700012789A4210D9904AA82101FB0323D3E97B
:103580000E678E4B586829F00DFF02460B463046F9
:1035900039462AF0E1F978B92B78042B05D1844B10
:1035A000844A1B7812789A4208D82A787F4B022ADC
:1035B00016D01A78042A15D10020C9E77E4AA8211E
:1035C00001FB0323D3E90E677C4B186829F0EAFE60
:1035D00002460B46304639462AF0BEF90028E4D0B0
:1035E0006420B5E71A78052A14D01A78062A13D071
:1035F0001A78072A12D01A78082A11D01B78092BBA
:1036000040F0C2806E4B6B491A78097891429A4615
:1036100008D8B9E050209BE73C2099E7282097E79D
:10362000142095E71B78DFF890B1A82101FB03B3C4
:10363000D3E90E679AF8003001FB03B3D3E91245D2
:103640009AF8003001FB03B122462B46D1E916015E
:1036500029F048FD00220023804689462AF05EF9C1
:1036600090B922462B463046394629F03BFD0022D0
:10367000544B29F0EBFE42464B462AF011F800224B
:10368000002329F031FD01E0002000212AF0B6F9E5
:10369000C6B2092E75D89AF800109AF80030DFF8F3
:1036A0002881A82707FB01B107FB03B3D3E9122345
:1036B000D1E9160129F016FD0022424B29F0F0FF56
:1036C0009AF8003007FB03B3D3E90E23CDE90023BA
:1036D0009AF8003007FB03BBDBE9122304460D46D2
:1036E0003046CDE9022329F04BFE22462B4629F035
:1036F000ADFE824618F806008B4629F031FE06F131
:103700000109064648460F4629F03AFE22462B4656
:1037100029F09CFE52465B4629F0E4FC002200237F
:1037200018F80980CDE904012AF0F8F820BBDDE99A
:103730000223DDE9000129F0D5FC52465B4629F061
:10374000D1FC044640460D4629F00AFE32463B466F
:1037500029F0C8FC02460B462046294629F076FE91
:10376000DDE9042329F09CFF02460B46304639462A
:1037700029F0BAFC06460F46304639462AF016F9BB
:1037800003E0114B987AE3E62078C0B2E0E600BF90
:10379000AFC7FF1FBCC4FF1F2CC5FF1FE18EFF1F5B
:1037A0000F88FF1FE4C7FF1FECC4FF1FF18EFF1F30
:1037B0002888FF1F2AC4FF1FF88EFF1F98C5FF1F10
:1037C00029C4FF1F0000244084C5FF1F244B33F889
:1037D000102044F208239A423AD00FD81F2A2FD043
:1037E00001D8B2B339E0B2F5FC6F23D040F2FF73D9
:1037F0009A4232D1FF22114600202CE04FF6C043FE
:103800009A4221D009D8B2F5784F16D04FF61F034F
:103810009A4222D1FF2200211CE04FF6E0739A4227
:1038200005D04FF6FF739A4217D1FF2211E0002214
:10383000FF2107E00022FF210CE00022114605E0F5
:10384000FF220021084606E00022A521FF2002E019
:10385000A5221146104623F0B8BE0020704700BFD5
:103860001488FF1FF8B50E4B1B780546BBB10D4FF2
:103870000024FF2D0ABF07EB440328465878FFF7C2
:10388000A5FFA6B2024631460748013423F06BFE7D
:10389000082CEED10448BDE8F84023F097BDF8BDF0
:1038A000FC87FF1F2F88FF1F14C5FF1F0D4B30B56E
:1038B0001B889B1A994285B011DA5408031B0A44ED
:1038C000044412B24FF6E07524B202928DE814005F
:1038D00003950AB21BB201B2034821F025FB05B0E3
:1038E00030BD00BF4488FF1F5CC6FF1F064B82B07F
:1038F0001A68009200991A680192019A521A82423B
:10390000F9D902B0704700BF58D8FF1F13B504465D
:103910001DF025FD8DF8060020461DF020FD8DF8D8
:103920000700BDF8060002B010BD13B504461DF037
:1039300016FD8DF8040020461DF011FD8DF80500E0
:1039400020461DF00CFD8DF8060020461DF007FDF9
:103950008DF80700019802B010BDFFFFFFFFFFFFC9
:10396000F8B5234CA82303FB004408460D4629F074
:1039700007FDD4E9222329F069FD0646C5F57F70CD
:1039800003300F4629F0FCFC02460B463046394610
:1039900029F086FE26F0E4FFD4E9202306460F46F0
:1039A00029F054FD32463B4629F050FDD4E91E2350
:1039B00029F09AFB32463B4629F048FDD4E91C2306
:1039C00029F092FB02460B4600200A4929F068FEC6
:1039D00005A3D3E9002329F085FB29F0E7FF00B216
:1039E000F8BD00BFAFF300800000006066127140B8
:1039F000F88EFF1F0000F03F2DE9F047A54AA823ED
:103A000003FB00238AB05E7A042E05460F469246D9
:103A100000F2E480A04B985D23F0A2FF16F0FD0FAA
:103A200004B23ED140F28E339C423ADC40F27A330B
:103A30009C4202DDA0F1080432E040F266339C4271
:103A400002DDA0F10D042BE0B4F5517F02DBA0F103
:103A5000120425E0B4F5397F02DDA0F119041FE05E
:103A600040F276239C4202DDA0F1240418E040F2EB
:103A700062239C4202DDA0F1280411E0B4F5117F1D
:103A800002DDA0F122040BE0B4F50C7F02DDA0F111
:103A90001C0405E040F206239C4202DDA0F118045C
:103AA00024B2A82303FB05A3D3E90E234FF4CA7362
:103AB00073437A4AD058652101FB06014FF0650E29
:103AC00042F82140D1580131D150D158B94224BFD8
:103AD0000121D1500020002300210EFB06F6013306
:103AE0005FFA83FE774508D906EB030E52F82EE005
:103AF00010EB0E0041F10001F1E77A1E4FF0A8082B
:103B0000D31708FB05A82AF019FB29F069FC98F8DF
:103B10006830022B06460F460ED129F047FF01B24E
:103B20002846FFF71DFF29F02BFCD8E90A2329F0CE
:103B30008DFCD8E90C2332E0012B37D1D8E91C23C6
:103B4000CDE90423D8E92023D8E91E01CDE90223D9
:103B5000DDE9042329F0C6FA00220023CDE906019D
:103B600029F0DCFE00BBDDE90223D8E9220129F0BF
:103B7000B9FADDE90423804689463046394629F002
:103B8000B1FA02460B464046494629F05FFCDDE9A2
:103B9000062329F085FD02460B46DDE9020129F0E6
:103BA000A3FA06460F4601E0DDE902673C4B1B78AD
:103BB000032B04D14FF4D670FCF747FE88B9354A81
:103BC000A82303FB0525D5E90A233046394629F009
:103BD0003DFCD5E90C2329F087FA58E000200021AC
:103BE00055E030493048FCF781FE29462E48FCF765
:103BF00081FE2E492C48FCF779FE21462A48FCF725
:103C00007DFE022429492848FCF770FE32463B46D7
:103C100000942548FCF778FE24492348FCF766FE0B
:103C2000A82303FB05AA0094DAE91C231E48FCF72D
:103C30006BFE1E491C48FCF759FE0094DAE91E236E
:103C40001948FCF761FE19491748FCF74FFE00942C
:103C5000DAE920231448FCF757FE14491248FCF710
:103C600045FE0094DAE922230F48FCF74DFE0F4988
:103C70000D48FCF73BFE0E490B48FCF737FE0D4B99
:103C800009481B6809930999FCF74DFE97E70AB0AC
:103C9000BDE8F087F88EFF1FB0C7FF1F18CAFF1FCF
:103CA000DAC7FF1F1A2203008C8AFF1F4D2603006C
:103CB0002422030058D8FF1F2DE9F04FA44DDFF850
:103CC000949289B005F105084FF0A80A15F8017F14
:103CD000A04C0AFB079696F890306BB14FF48E70AB
:103CE000FCF7B3FD01463846FFF786FEC6E90E0134
:103CF00001212878FDF7EEFFA845E7D1964E974DB4
:103D000032782B789A4219D2262023F029FE377870
:103D100040F21D13C0F1D8005843A82606FB074601
:103D200000F6FC0029F02CFBD6E90A2329F08EFBD3
:103D3000C6E90E0101213846FDF7CCFF884B1A7801
:103D4000FF2A9B464ED0874B2E7893F80080B045D3
:103D500048D20120FCF779FD8642814642D90320F2
:103D6000FCF773FD86423DD9A82606FB0047D7E93C
:103D70000E0100227C4B29F0F9FD002800F09E8006
:103D8000744806FB0900D0E90E01D7E90E2329F09B
:103D900087FC29F033FEC0B229F05AFF7349019025
:103DA00029F0AAFF724902904FF000090F680391B1
:103DB000CA4606FB08461BF80A0029F049FF804660
:103DC000014602982AF054F900285ED10AF1010355
:103DD0005FFA83FABAF1050FEDD9B9F1000F01D0FE
:103DE000039B1F60634B93F800B0BBF1010F20D120
:103DF000614B93F800A02B78534539D9A82303FBD6
:103E00000A43D3E90E895D4B186829F0CBFA0646C0
:103E10000F4602460B464046494629F09DFD0028C4
:103E200065D0574B1A78012A61D083F800B0594603
:103E300074E0BBF1030F04D1514F3B78C3B90121AA
:103E400007E0BBF1020F13D14D4F3B78012B0FD18F
:103E500000214C4B3970187824F08CF94A4B387893
:103E60001E7829F07DFAA82303FB0646C6E90E0159
:103E7000464B1E78FF2E00F0DB800520FCF7E5FCAA
:103E80002D78A84207464ED3D2E04149019829F047
:103E900033FF014640462AF0EBF8002896D00AF19D
:103EA000010029F06DFAC6E90E013A4B1B68059333
:103EB000059F4FF001094FF0060A87E7D7E90E0189
:103EC0000022294B29F03EFD48B9324B284A1B6895
:103ED0000693069B12689B1AB3F57A7F82D9A826AF
:103EE00006FB084600220023C6E90E237AE7A82332
:103EF00003FB0A4ADAE90E233046394629F02CFD45
:103F000010B11F4B1A783AB91F4B1E782B78B34269
:103F1000AED91B4B1878A4E700211970194B1878FB
:103F200024F028F9F0E70420FCF78FFC854233D910
:103F3000A82303FB0747D7E90E8903FB0040494646
:103F400003FB0644D0E90E23404629F0CBF861E09C
:103F500000B9FF1FF88EFF1F0788FF1F2AC4FF1F2D
:103F60002CD5FF1F4888FF1F000008403333933FC4
:103F700024D5FF1FB0C5FF1F14CAFF1FB8C7FF1FFE
:103F80001188FF1FDF8EFF1F4988FF1F0B88FF1F4F
:103F90009A99593F58D8FF1F40F21D10FCF755FC65
:103FA000012845D1244A254B12681B680792079ABD
:103FB00003F5FA739A423BD90520FCF746FCA82585
:103FC00005FB0045074600220023D5E90E0129F034
:103FD000A5FCDFF86CA060B90021DAF800002AF037
:103FE0001FF830B1D5E90E0129F028FDCAF800000C
:103FF0001EE0A82505FB0747DAF8000029F0D2F9F2
:10400000D7E90E8902460B464046494629F06AF830
:1040100005FB0644D4E90A2329F018FAD4E90C2355
:1040200029F060F8C4E90E0101213046FDF752FE87
:1040300009B0BDE8F08F00BF58D8FF1FD88EFF1F12
:10404000EC8EFF1F10B572B60C4B41241C7003F8A8
:10405000010C073B8020187018780006FCD5084B2F
:104060001B788B54074B0A441B785370064B1B7804
:104070009370064B1B78D37062B610BD07000240E8
:104080000B0002400A000240090002400800024002
:1040900073B50F490F4801AEFCF728FC00223146EA
:1040A0000F20FFF7CFFF4FF4C67500242846FCF71A
:1040B000CCFBA5F5C6730135F35C83421CBF01340C
:1040C000E4B2B5F5C87FF1D1204602B070BD00BFA3
:1040D0002B2203008C8AFF1FF0B595B02C22002103
:1040E00009A823F037FBA94901A826F0FCF84FF4F2
:1040F000C6750A272846FCF7A8FB0928044608D8F5
:10410000A34901A8FCF7EDFBA14901A8FCF7E9FBD5
:1041100022E0632820D89E4901A8FCF7E2FBB4FB0B
:10412000F7F60A22F1B205A826F010F905A901A8B0
:10413000FCF7D5FB05A826F096F807FB16410A22E6
:10414000C9B205A826F002F905A901A8FCF7C7FB2A
:1041500005A826F088F803E0214601A826F0C4F956
:104160000135B5F5C87FC5D12C22002309A901A8C6
:1041700026F026FA09A822F0ECFC1021054622F0D0
:104180005DF8044628462AF0F9F9202221468148A4
:104190002AF00EFA80B9804905A826F0A4F805A9EE
:1041A0004FF4FC627D4816F0E3FB05A826F05BF8AF
:1041B00001214FF48B7067E0794901A826F010F9CE
:1041C0004FF4C6750A272846FCF73FFB092804462A
:1041D00008D86F4901A8FCF784FB6D4901A8FCF7DA
:1041E00080FB22E0632820D8694901A8FCF779FB0D
:1041F000B4FBF7F60A22F1B205A826F0A7F805A944
:1042000001A8FCF76CFB05A826F02DF807FB16416A
:104210000A22C9B205A826F099F805A901A8FCF759
:104220005EFB05A826F01FF803E0214601A826F052
:104230005BF90135B5F5C87FC5D12C22002309A94A
:1042400001A826F0BDF909A822F083FC102105463B
:1042500021F0F4FF044628462AF090F92022214656
:104260004C482AF0A5F9A8B94E4905A826F03BF814
:1042700005A94FF4FC62494816F07AFB05A825F021
:10428000F2FF01214FF48D70FCF772FA20462AF0FC
:1042900075F975E0444901A826F0A2F84FF4C675F7
:1042A0000A272846FCF7D1FA0928044608D83849D5
:1042B00001A8FCF716FB364901A8FCF712FB22E027
:1042C000632820D8324901A8FCF70BFBB4FBF7F6B2
:1042D0000A22F1B205A826F039F805A901A8FCF7D1
:1042E000FEFA05A825F0BFFF07FB16410A22C9B256
:1042F00005A826F02BF805A901A8FCF7F0FA05A8F7
:1043000025F0B1FF03E0214601A826F0EDF80135C4
:10431000B5F5C87FC5D12C22002309A901A826F034
:104320004FF909A822F015FC1021054621F086FF5F
:10433000044628462AF022F92022214615482AF070
:1043400037F980B9194905A825F0CDFF05A94FF423
:10435000FC62124816F00CFB05A825F084FF022130
:104360004FF4E77090E7124905A825F0BCFF0B4811
:104370004FF4784205A916F0FBFA05A825F073FF63
:1043800001A825F070FF15B0F0BD00BF3922030071
:10439000EB240300C8C4FF1F5722030058B9FF1FB6
:1043A0007822030096220300B4220300D2220300E5
:1043B000F922030038B546F22C3112481FF0A3FB56
:1043C000012110481FF099FB0F490E48FCF78EFAA7
:1043D0004FF4C6742046FCF738FA0928054601D880
:1043E0000A4902E0632803D809490648FCF77EFA27
:1043F000294604480134FCF77DFAB4F5C87FE9D1B9
:1044000038BD00BF5CC6FF1F07230300732D0300E8
:10441000EB2403002DE9F041074688B068B9C34B8F
:10442000C34AB3F90030019012880D3A12B20092DB
:1044300001460D22BF4821F0E9FCBF4B00221A7053
:10444000BE4B00221A60BE4BFF221A703FB93B469A
:10445000DC222821B74820F029FEFFF7ABFFB92462
:10446000052646F22C3300258DE8500002931E22CB
:10447000E6232821AF4821F021FD8DE85000E623F6
:104480001E2204AC2821AB48029520F02BFBAD493D
:10449000AD4E204625F027FF0F2323222D21009328
:1044A000AA480295DC23019416F03CFB204625F037
:1044B000DAFE29469F481FF026FB01219D481FF088
:1044C0001CFB2B46272232219A4820F0EFFD701961
:1044D000143516F0B7F9B5F5027FF8D10025192685
:1044E0009B49204625F0FFFE282337228721994843
:1044F00002950194009616F015FB204625F0B3FEB8
:104500009549204625F0EFFE28233722B421934811
:1045100002950194009616F005FB204625F0A3FEB7
:104520008F49204625F0DFFE28233722E1218D48E0
:1045300002950194009616F0F5FA204625F093FEB8
:104540008949204625F0CFFE282355228721874818
:1045500002950194009616F0E5FA204625F083FEB8
:104560008349204625F0BFFE28235522B4218148E7
:1045700002950194009616F0D5FA204625F073FEB8
:104580007D49204625F0AFFE28235522E1217B48B6
:1045900002950194009616F0C5FA204625F063FEB8
:1045A0007749204625F09FFE2823732287217548EE
:1045B00002950194009616F0B5FA204625F053FEB8
:1045C0007149204625F08FFE28237322B4216F48BD
:1045D00002950194009616F0A5FA204625F043FEB8
:1045E0006B49204625F07FFE28237322E12169488C
:1045F00002950194009616F095FA204625F033FEB8
:104600006549204625F06FFE28239122B421634896
:1046100002950194009616F085FA204625F023FEB7
:104620005F49204625F05FFE282337222D215D4873
:1046300002950194009616F075FA204625F013FEB7
:104640005949204625F04FFE282355222D21574851
:1046500002950194009616F065FA204625F003FEB7
:104660005349204625F03FFE282373222D2151482F
:1046700002950194009616F055FA204625F0F3FDB8
:104680004D49204625F02FFE282337225A214B483A
:1046900002950194009616F045FA204625F0E3FDB8
:1046A0004749204625F01FFE282355225A21454818
:1046B00002950194009616F035FA204625F0D3FDB8
:1046C0004149204625F00FFE282373225A213F48F6
:1046D00002950194009616F025FA204625F0C3FDB8
:1046E0004FF023083A49204625F0FDFD4423AF2230
:1046F0002D21384802950194CDF8008016F012FA69
:10470000204625F0B0FD3449204625F0ECFD442339
:10471000AF227621314802950194CDF8008016F041
:1047200001FA204625F09FFD5AE000BF0888FF1FD0
:104730004488FF1F5CC6FF1F0088FF1FD0C5FF1FF6
:104740000188FF1F272103001CB9FF1F58B9FF1F55
:1047500070260300E4B9FF1F24230300F8B9FF1FEC
:10476000782603000CBAFF1F7C26030020BAFF1F27
:10477000592A030034BAFF1F3428030048BAFF1F28
:10478000FF2403005CBAFF1F9422030070BAFF1FCE
:104790001023030084BAFF1FEB24030098BAFF1F05
:1047A0008A240300ACBAFF1F99210300D4BAFF1F6B
:1047B000122C0300FCBAFF1F12230300C0BAFF1F14
:1047C000DD2A0300E8BAFF1F2598030010BBFF1F76
:1047D00092230300A8B9FF1F142303006CB9FF1F25
:1047E0001549204625F07FFD144802950194CDF827
:1047F00000804523AF22BF2116F094F9204625F012
:1048000032FD0FB90E4902E0012F11D10D492046AA
:1048100025F069FD4FF6E07302930B480194009672
:10482000282391222D2116F07DF9204625F01BFD2D
:1048300008B0BDE8F08100BF1C23030080B9FF1F52
:10484000232303007C26030094B9FF1F2DE9F043C6
:10485000A14D89B006460F4690460024281914340D
:1048600015F0F0FFB4F5027FF8D19C4B9C48002571
:104870001D709C4B00221A609B4BB9241D701E2298
:1048800046F22C334FF00509114602938DE81002D1
:104890008C2321F013FB1E2211468C238DE810027D
:1048A0008F48029504AC20F01DF99049204625F070
:1048B0001AFD23220F23114600938D48029582236F
:1048C000019416F02FF9204625F0CDFC29468448A6
:1048D0001FF019F9012182481FF00FF92B462722FA
:1048E00028217F4820F0E2FBB8F1000F02D1CDF87B
:1048F000008001E00223009332463B4678480026C0
:104900001925FCF701F87B49204625F0ECFC28230B
:1049100037222321784802960194009516F002F977
:10492000204625F0A0FC7549204625F0DCFC282314
:1049300037225021724802960194009516F0F2F841
:10494000204625F090FC6F49204625F0CCFC28231A
:1049500037227D216C4802960194009516F0E2F80A
:10496000204625F080FC6949204625F0BCFC282320
:1049700055222321664802960194009516F0D2F83C
:10498000204625F070FC6349204625F0ACFC282326
:1049900055225021604802960194009516F0C2F805
:1049A000204625F060FC5D49204625F09CFC28232C
:1049B00055227D215A4802960194009516F0B2F8CE
:1049C000204625F050FC5749204625F08CFC282332
:1049D00073222321544802960194009516F0A2F800
:1049E000204625F040FC5149204625F07CFC282338
:1049F000732250214E4802960194009516F092F8C9
:104A0000204625F030FC4B49204625F06CFC28233D
:104A100073227D21484802960194009516F082F891
:104A2000204625F020FCB8F1010F1FD14349204654
:104A300025F059FC28239122232141480296019414
:104A4000009516F06FF8204625F00DFC3D492046F4
:104A500025F049FC3C4802960194009528239122B8
:104A60007D2116F05FF8204625F0FDFB37492046F2
:104A700025F039FC00261923912200935021282388
:104A800002960194324816F04DF8204625F0EBFBD3
:104A900023253049204625F026FC3E23AF22294617
:104AA0000296019400952C4816F03CF8204625F01B
:104AB000DAFB2A49204625F016FC3E23AF22672167
:104AC000029601940095264816F02CF8204625F011
:104AD000CAFB09B0BDE8F0831CB9FF1F0088FF1FA7
:104AE0005CC6FF1FD0C5FF1F0188FF1F27210300E1
:104AF00058B9FF1F70260300E4B9FF1F24230300E9
:104B0000F8B9FF1F782603000CBAFF1F7C260300AC
:104B100020BAFF1F592A030034BAFF1F34280300AC
:104B200048BAFF1FFF2403005CBAFF1F9422030052
:104B300070BAFF1F1023030084BAFF1F262303004F
:104B400098BAFF1F28230300C0BAFF1FEB240300FD
:104B5000ACBAFF1F922303006CB9FF1F1C23030094
:104B600080B9FF1F10B5074C20461FF03BF82046C8
:104B700001211EF0C2FF20464FF6FF71BDE8104034
:104B80001EF0C1BF5CC6FF1F2DE9F04190B0044686
:104B9000FFF7E8FF0021AE48AE4E1EF0B4FFAE4B6B
:104BA0001878FCF73DFD3278012A33D10A234FF4FF
:104BB000FC668DE8480032211F23A548A74D21F04F
:104BC00025F9002302223821A14820F06FFAA449D8
:104BD0009F48FBF78BFEA349A348FBF787FE002401
:104BE0002B78E1B2994204F101040FD2002208A807
:104BF00016F048F908A99C4825F0F0F908A825F016
:104C000032FB9A499848FBF771FEE9E7964825F090
:104C100005FAC0E0022A03D1954B1B7813B9A2E034
:104C2000092C76D80A234FF6E0758DE8280001227A
:104C30001F233221864821F0E9F88E4B84481D78E5
:104C400002220023362120F031FAFF2C18BF25461E
:104C500089497F48FBF74AFE29467D48FBF74AFE13
:104C6000864B1B680393864B039A1A60854B04ACF2
:104C700003F10802A04618685968274603C708339D
:104C800093423C46F7D118689A889B793860BA807D
:104C9000BB7130357C488DF819501CF0F6FB60B9BB
:104CA00013234246794908A81CF030FD08A976482C
:104CB000FCF7A0FC08A81CF0A5FB73481CF0E5FB62
:104CC000044600B367497048644DFBF70FFE0024AB
:104CD0002B78E1B2994204F101040FD2002208A816
:104CE00016F0D0F808A9684825F078F908A825F04A
:104CF000BAFA5E496448FBF7F9FDE9E7644962489E
:104D0000FBF74FFC47E063495748FBF74AFC347018
:104D100041E0032A12D10A234FF6E0748DE818000F
:104D200001221F2332214A4821F070F83321002349
:104D30000222474820F0BAF9574929E0042A15D140
:104D40000A204FF478438DE8090001221F23322105
:104D50003F4821F05BF83321002302223C4820F039
:104D6000A5F94E4914E0092C7FF65CAF0A2146F202
:104D70002C338DE80A0001221F233221344821F010
:104D800045F8332100230222314820F08FF94449AD
:104D90002F48FBF7ABFD434B1B78002B51D0424B08
:104DA0002B481C886408323421B2A4B20A224FF680
:104DB000E073671C02264FF478458DE80C003FB283
:104DC0000E23012221F022F8394600960C230822F6
:104DD0001F48019521F01AF83346394600960622FD
:104DE0001B48019521F012F8A71D04F10B014FF0AB
:104DF000040833460096062209B2154801953FB2D1
:104E000021F004F833463246394611480195CDF871
:104E1000008020F0FBFF062604EB08013B464246DB
:104E200009B20B48019500961FF0FAF8E31D04F152
:104E30000901019500961BB2424609B204481FF0D1
:104E4000EFF80320FCF7ECFB10B0BDE8F08100BFE9
:104E50005CC6FF1FDAC7FF1F2A88FF1F2AC4FF1F77
:104E60002A2303008F2003008C8AFF1FD820030011
:104E700033D5FF1F4788FF1F9D24030058D8FF1F0D
:104E800030C5FF1F9A200300F4C4FF1F38D5FF1F51
:104E9000272103002E2303003C23030042230300A9
:104EA00048230300BCC7FF1F0888FF1F2DE9F041FE
:104EB0003B4C07462046FBF780FD3A4A012313701E
:104EC0002372394B394A00261E70394B10781E70F8
:104ED000384B1978884215461C4612D2DFF8E0801C
:104EE000022198F8000023F073F998F80000324B83
:104EF00032491E6022284FF0030228BFFF2023F012
:104F000099F96A7823789A420FD22D4C0221607861
:104F100023F05EF96078284B2A49002222285A6043
:104F200028BFFF20032223F085F9274B274D0024BB
:104F30001C70274B2E681C70264B14201C7025F00B
:104F4000AAFB8046FBF75AFD414630461DF038FE6D
:104F5000A7F16403012B07D814202C6825F09BFBD4
:104F60000546FBF755FD13E01B4B38461C70FFF759
:104F70000BFE1A4B1878FCF753FB194B1B78042BCC
:104F80000CD014202C6825F086FB0546FBF72CFD81
:104F900029462046BDE8F0411DF012BEBDE8F08173
:104FA00054C4FF1F4288FF1FC8C7FF1F3F88FF1F51
:104FB00032D5FF1F2AC4FF1F10B9FF1FD9050000FB
:104FC000BDC7FF1FE9050000E9C6FF1FA4D7FF1FEB
:104FD000D4C5FF1FCEC5FF1FEAC6FF1F2A88FF1FCB
:104FE000DAC7FF1F37B54FF6E074002808BF00246A
:104FF0000546FFF7B7FD154B1B780194032B4FF0C7
:105000000B0300934FF000024FF0140307D0AA21C6
:105010000F4820F0FBFE00230222AC2106E0E6212F
:105020000B4820F0F3FE00230222E821084820F07C
:105030003DF8012D07D1002105481EF064FD05490A
:105040000348FBF753FC03B030BD00BF2A88FF1FA5
:105050005CC6FF1F2A2303002DE9F0438D4F8E4CC1
:105060003B78032B87B0054609D00C210022B4F908
:1050700000308A488DE80600114620F0C7FE032064
:10508000FCF7CEFA44F208260C22B4F9003083482B
:105090008DE844000022114620F0B8FEFFF762FDC3
:1050A0003DB1032D00F0F080012D4FF478460BD870
:1050B00001E046F22C360B23009301962E230122A9
:1050C0000521764820F0A2FE754902A825F00BF9CB
:1050D00005230093032202AB1921724816F038FA17
:1050E00002A825F0C0F815F0FD0F08D10B2300939E
:1050F00001962E2301223721684820F087FE6A4955
:1051000002A825F0F0F805230093032202AB4B21FF
:10511000644816F01DFA02A825F0A5F8012D73D1F8
:1051200000215E481EF0EFFC604B1A78012A1E46F3
:1051300007D14FF6FF7159481EF0E5FC4FF4784354
:1051400001E04CF218634FF00B0901220193A821F2
:105150002A235248CDF8009020F058FE4FF0050861
:10516000534902A825F0BFF802AB0322BD214D48E8
:10517000CDF8008016F0ECF902A825F074F80021B3
:1051800046481EF0C0FC3378012B56D0FCF7D4FC07
:105190004CF21866FF2814BF4FF4FC63334601221B
:1051A00001936F2134233D48CDF8009020F02EFE6E
:1051B000404902A825F097F802AB03228B21394819
:1051C000CDF8008016F0C4F902A825F04CF83B7821
:1051D0003248CDF80090032B18BF4FF4FC662B2308
:1051E0000122D721019620F011FE334902A825F0B3
:1051F0007AF82C48CDF8008002AB0322ED2116F09E
:10520000A7F902A825F02FF84FF6FF7123481EF0EA
:105210007AFC032D16D121880B2046F22C3332392B
:105220008DE8090009B22D2301221C4820F0EEFD73
:10523000248822491E3CA4B215E04FF6FF7117489E
:105240001EF061FC218815480B2246F22C333239BE
:105250008DE80C0009B22D23012220F0D7FD24880F
:1052600017491E3CA4B202A825F03DF8052300937F
:10527000032202AB21460B4816F06AF902A824F07B
:10528000F2FF07B0BDE8F0834FF6FF7103481EF050
:105290003AFCC0E72A88FF1F0888FF1F5CC6FF1F73
:1052A0004E230300B8BCFF1FED2103001288FF1F2F
:1052B000562303005B23030064230300BA2A030080
:1052C0006B2303002DE9F0437E4B1878A7B000282C
:1052D00000F0F5807C4F7D483988002301937C4B9A
:1052E0001B88423B1BB2653900932822652309B213
:1052F00020F08CFD0123774A774916A81CF006FAA6
:10530000FFF730FC08230DEB03000A227349FBF77B
:10531000E9F8062202A912A825F09CF970491EA8F6
:1053200024F0E1FF1EA912A825F071F904461EA879
:1053300024F099FF12A824F096FF64B906232246B0
:1053400002A91EA825F066F91EA902A825F040F8BA
:105350001EA824F088FFDFF89C81FF24002501228D
:1053600016A91EA81CF02EFA1EA81CF08EF80646E0
:105370001EA8002E00F081801CF045F8014606A80A
:1053800024F0B1FF1EA81CF040F8814600286DD122
:1053900054490AA824F0A7FF0AA906A825F037F95E
:1053A000002816DB01234A4606A90EA825F032F98B
:1053B0004D4912A824F097FF12A90EA825F027F94D
:1053C000B0FA80F612A824F04EFF0EA8760924F059
:1053D0004AFF0AA824F047FF002E47D198F8002082
:1053E000AB1A0C2B01DC954202D20135EDB23DE047
:1053F00003EB43023988354803EB820229325D39D9
:10540000334612B209B205F101091FF04FFE4946B9
:105410002E48FBF773FA35492C48FBF767FA06A9C3
:105420002A4824F0DBFD2F4912A824F05CFF12A9C2
:1054300006A825F0ECF83246034606A90EA825F08A
:10544000E9F80EA825F00DF9014602A825F08AF822
:1054500006460EA824F007FF12A824F004FF1EB190
:1054600098F800402C1BE4B25FFA89F506A824F0F6
:10547000FAFE1EA81BF0C6FF71E71BF0C3FF1C4B12
:1054800016A81D701BF0F5FFFF2C11D0398804EB16
:10549000440204EB82020A204FF4784328325E393A
:1054A0008DE8090012B25F2309B208481EF0F8FD2A
:1054B00002A824F0D8FE16A81BF0A4FF204627B0AF
:1054C000BDE8F08333D5FF1F0888FF1F5CC6FF1FB0
:1054D0004488FF1F2821030038D5FF1F34C5FF1F54
:1054E0004D260300702303001C24030074230300D3
:1054F00006B9FF1FE88EFF1F2DE9F0414E4B1978CA
:10550000A0B0064619B90A2224F020FF8FE001233B
:105510004A4A4B494B4F10A81CF0F8F8FFF722FB02
:105520000024012210A918A81CF04CF918A81BF09F
:10553000ACFF054618A8002D6DD01BF064FF014696
:10554000684624F0D0FE18A81BF05FFF80460028B4
:105550005AD13D4904A824F0C6FE04A9684625F0A6
:1055600056F8002816DB01234246694608A825F0B4
:1055700051F836490CA824F0B6FE0CA908A825F06D
:1055800046F8B0FA80F50CA824F06DFE08A86D0965
:1055900024F069FE04A824F066FE002D34D12C49C5
:1055A0000CA824F0A0FE0CA9684625F030F80546AA
:1055B0000CA824F058FE002DACBF0121FF210720CC
:1055C0003970FBF7D5F8234B1A78234B1B7813441B
:1055D0009C4217D11C490CA824F085FE0CA96846F2
:1055E00025F015F8002203466946304625F012F8EA
:1055F0000CA824F038FE684624F035FE18A81BF0ED
:1056000001FF11E00134E4B2684624F02CFE18A832
:105610001BF0F8FE85E71BF0F5FE10A81BF029FF34
:105620000E49304624F05FFE10A81BF0EBFE30461A
:1056300020B0BDE8F08100BF33D5FF1F2821030053
:1056400038D5FF1FA8C6FF1F702303001C240300CA
:1056500077230300A0C5FF1FE88EFF1FEB24030084
:105660002DE9F0438B4C8C4E2288338891B00A216F
:105670000025653B0A3A8DE822001BB212B20121D7
:105680008046864820F0C2FB228884480A3A2B468E
:1056900012B201211FF00AFD814B1B7843B98149E9
:1056A0007E48FBF723F94FF47A7022F007FFEDE014
:1056B00072B6FFF757FA7C4B02AD03F1100E2A4683
:1056C000186859682F4603C7083373453D46F7D11C
:1056D00018689B883860BB807449532308A808F178
:1056E00030088DF818801CF011F808A81BF0CDFECA
:1056F0000546002800F09C806D4B6E4A1B7812789E
:105700006D496E4C08A824F0A0FC04F5EE67002655
:10571000A04694F85830002B7DD094F827300B2BFE
:1057200005D1A38B093B9BB2022B40F2A380B4F9B5
:10573000101008A8FBF7E2F8614908A8FBF7D6F8B3
:10574000B4F9121008A8FBF7D9F85D4908A8FBF7CF
:10575000CDF8B4F9141008A8FBF7D0F8584908A8F8
:10576000FBF7C4F8B4F9161008A8FBF7C7F85449BA
:1057700008A8FBF7BBF894F8271008A8FBF7BAF8BD
:105780004F4908A8FBF7B2F8A18B08A8FBF7B6F8B9
:105790004B4908A8FBF7AAF8E18B08A8FBF7AEF87D
:1057A000474908A8FBF7A2F8218C08A8FBF7A6F840
:1057B000434908A8FBF79AF8217E08A8FBF79AF856
:1057C0003F4908A8FBF792F894F82730ABB94FF09F
:1057D0007009012509FB068994F82430AB4213D9DE
:1057E00009EB050308A8197EFBF784F80135344955
:1057F00008A8FBF77BF8EDB2EEE70B2B01D0052BE9
:1058000002D12378002B38D12E4908A8FAF7C9FE17
:1058100008A81BF090FD7034A74206F101067FF442
:1058200078AF08A81BF087FD08A81BF022FE1CE03B
:1058300022880A3A034612B2012118481FF036FCAA
:1058400033882288154801950A21653B0A3A009160
:105850001BB212B2012120F0D9FA1B490F48FBF705
:1058600045F84FF4FA6022F029FE62B608A81BF052
:10587000C9FD0BE00023E38359E7214608A8FBF7A5
:1058800035F80F4908A8FBF731F8BDE711B0BDE8BE
:10589000F08300BF4488FF1F0888FF1F5CC6FF1FFE
:1058A00033D5FF1F95230300C223030038D5FF1F04
:1058B0001288FF1F2A88FF1FA1230300B8BCFF1F07
:1058C000D820030027210300AE2303002DE9F04F69
:1058D000C24EA3B0934604AF32883B610A3A00231C
:1058E00012B28A4680461946BD4897F8A0901FF02C
:1058F000DDFBFFF737F907F118001BF075FDB8481D
:105900001DF0ECFF824580F2AE81B5481DF0E9FF45
:105910000A38834580F2A78101234246B14907F145
:1059200058001BF0F3FE07F1580107F11800FBF7D0
:1059300061FE1BF0AAFD044607F158001BF062FD52
:105940002CB94246A849A64824F07FFB90E107F114
:10595000180107F15800FCF757F907F15800FDF757
:10596000D5FF044607F158001BF04CFD44F64253A6
:105970009C4240F03F8107F1180107F15800FCF705
:1059800043F907F15800FDF7D0FF07F158001BF06D
:1059900039FD07F1180107F15800FCF735F907F157
:1059A0005800FDF7C2FF07F158001BF02BFD07F16F
:1059B000180107F15800FCF727F907F15800FDF727
:1059C000B4FFF86007F158001BF01CFD07F1180147
:1059D00007F15800FCF718F907F15800FDF7A5FF8B
:1059E00007F158001BF00EFD07F1180107F15800F0
:1059F000FCF70AF907F15800FDF797FF054607F194
:105A000058001BF0FFFC07F1180107F15800FCF7E4
:105A1000FBF807F15800FDF788FF786107F158009F
:105A20001BF0F0FC07F1180107F15800FCF7ECF847
:105A300007F15800FDF76AFF044607F158001BF014
:105A4000E1FC012C40F0D68007F1180107F1380085
:105A5000FCF7DAF807F13800FDF758FF182811D1E4
:105A600007F1180107F15800FCF7CEF807F15800CC
:105A7000FDF75BFFB0FA80F407F1580064091BF0F2
:105A8000C1FC00E0002407F138001BF0BBFC002C37
:105A900000F0B080C7F808D0ADB2BC8ABAF1000FF0
:105AA00011D1BBF1000F0ED1504B1A8833881B1B4C
:105AB0000221521B0A3B92FBF1F293FBF1F31FFA16
:105AC00082FA1FFA83FB3B697C612E467BB1484B0F
:105AD000702000FB093090F82530428A018A029339
:105AE00090F82730019300942B461BF0A5F805F1A0
:105AF000010909EB490929F0030339483B611DF00D
:105B0000EDFE5544854205DD35481DF0E7FECAEB44
:105B1000000086B232481DF0E4FE0BEB040585421E
:105B200006DD2F481DF0DDFECBEB000083B27B616C
:105B300006EB4605EB1D23F00703ADEB030DABB2FF
:105B4000FA687B603B69013C564403FB0429B3B20D
:105B50000DF110080024FB607B69A6B2B34239D96D
:105B600007F118001BF067FC484504D0494607F1CF
:105B700018001BF057FC7A68414607F118001BF02B
:105B80004CFC0BEB060292B20092FB6814485146A3
:105B900020F024FA0026B54214DD08EB0603104875
:105BA00099785B780902DB0001F4784103F4FC6327
:105BB0000B4318F80610033643EAD1011DF064FFC9
:105BC000B6B2E8E706481DF06BFF3B690134C3EB52
:105BD0000909C1E7D7F808D03FE000BF4488FF1F9C
:105BE0005CC6FF1F38D5FF1FD82303000888FF1F9E
:105BF000B8BCFF1F3288234B0B204FF6E0710B3AE5
:105C0000B3F9003012B28DE8030000211E4820F0E5
:105C1000FDF84FF478411C481DF075FF41461A48C5
:105C2000FAF764FE19491848FAF760FE4146184829
:105C30001BF0BCFD4FF4FA7022F040FC154A7023B3
:105C400003FB0922938B01339BB2FD2B938304D872
:105C50004A465946504600F021F807F118001BF05B
:105C600008FC012404E00C490748FAF73FFE002431
:105C700007F118001BF0C6FB20467C37BD46BDE887
:105C8000F08F00BF0888FF1F5CC6FF1FF2230300D0
:105C900038D5FF1FB8BCFF1FE52303002DE9F04FE7
:105CA000774B1C78A3B081468A469046002C00F0C2
:105CB000E280744B7449702505FB023502A8AF8B56
:105CC00024F011FB95F82730052B01D16F4902E034
:105CD0000E2B03D16E4902A824F082FB95F82730E1
:105CE000052B05D1284628F0A4FD012800F2BA8032
:105CF000FFB2FF2F19D10498013024F0CEFC049A92
:105D0000044601460023013202A824F059FC049BFA
:105D1000234400225A702046CDF8008001235246C9
:105D20004946FFF7D3FD044698E0DDF808B059492D
:105D300001235A4612A81BF0E9FC0026012212A9F1
:105D40001AA81BF03FFD1AA81BF09FFB0446002871
:105D50007BD0594606A824F0C6FA1AA81BF053FBBC
:105D6000014606A8FAF7BDFD1AA81BF04EFB002855
:105D700064D149490AA824F0B6FA0AA906A824F071
:105D800046FC00280CDB45490EA824F0ACFA0EA90D
:105D900006A824F03CFCC4430EA8E40F24F063FAE8
:105DA0000AA824F060FA002C48D1BE4241D10898DC
:105DB000013024F072FC089A01460132064623465F
:105DC00006A824F0FDFB089B33441AA85C701BF066
:105DD00050FB12A81BF04DFB2B4906A824F000FB3A
:105DE0001AA81BF010FB014606A8FAF77AFD0898DE
:105DF000033824F052FC089A234607460146033A2A
:105E000006A824F0DDFB089A3946033A284621F01B
:105E100007FC012352464946CDF800803046FFF783
:105E200055FD044606A824F01EFA1AA81BF0EAFA4B
:105E300011E01AA81BF01DFB0136F6B206A824F0EB
:105E400012FA1AA81BF0DEFA78E71AA81BF0DAFAA1
:105E500012A81BF00EFB12A81BF0D4FA02A824F023
:105E600002FA08E0294602A8FAF73BFD0A4902A80F
:105E7000FAF737FD3FE7204623B0BDE8F08F00BFBB
:105E800033D5FF1FB8BCFF1F2721030007240300E1
:105E90000D24030038D5FF1F152403001A24030026
:105EA00073B51C4B1C4A1D481D4D1E4E00241C7012
:105EB0001D4BB3F90030019412880C3A12B20092D3
:105EC00021460C221FF0A2FF184B1878FBF7A8FB05
:105ED000174B01221A7095F85830E2B26BB195F861
:105EE000273013B926F8143003E0052B0CD00E2B05
:105EF0000AD0002128461AF051FE0134112C05F178
:105F00007005E8D102B070BD698A288AFFF7C6FE25
:105F1000F3E700BFCEC5FF1F4488FF1F5CC6FF1F0D
:105F2000B8BCFF1F2EC4FF1F0888FF1F2A88FF1F51
:105F30004288FF1F2DE9F04FBE4FBF4E3A8833888D
:105F4000DFF854939FB000240D46653B0A210A3ABE
:105F500080468DE812001BB212B20121B7481FF033
:105F600055FF3A88B5480A3A234612B201211FF07C
:105F70009DF8FEF7F7FDB24B99F800001C70B14B8D
:105F80001C70FBF74DFBB8F10A0F40F09E803A8879
:105F9000B6F80090AC4BAD4916AD243A4FF00B0B60
:105FA00092B24FF0050A4FEA5909284683F800B02B
:105FB000049224F098F92B46049ACDF800A04946A3
:105FC000A34815F0C5FA284624F04DF93A88A149AE
:105FD0001A3A4FF01A0992B22846049224F083F933
:105FE000049A0294214628230195CDF800909A48FE
:105FF00014F098FD284624F036F933883A889749FA
:10600000293B1A3A9BB292B228460493059224F097
:106010006AF9059A0499029428230195CDF8009015
:106020008F4814F07FFD284624F01DF933883A8804
:10603000022044F20821703B0C3A8DE803001BB2A9
:1060400012B233217D481FF0E1FE864B1878338869
:106050003E3B22460093FA213223FAF7AAFB3F88FF
:1060600004901A3FBFB28049284624F03CF94346C9
:106070003A46BDF8101002940195CDF800907B4887
:1060800014F050FD284624F0EEF831886B48CDF826
:1060900000B046F22C333239019301222D2309B28C
:1060A0001FF0B4FE368872491E3EB6B2284624F070
:1060B0001AF9CDF800A02B4603223146644815F0AA
:1060C00047FA284624F0CFF8AFE06A4B1C78002C42
:1060D00000F0AB80684B09AA03F110071646186858
:1060E0005968144603C40833BB422246F7D11868E6
:1060F0009B882060A38008F1300831465F488DF806
:1061000034801BF047FB28B930238DF834305C4BCA
:1061100001221A7001233246584916A81BF0F6FADC
:10612000032089F80000FBF77BFA16A81BF0ADF9F5
:10613000044600286DD0534F454E00244FF01408FC
:1061400008FB047014F07EFB702303FB046301342E
:106150000022112C83F85820F2D14B4B0FAA03F1E7
:106160001806904618685968144603C40833B342A9
:106170002246F7D100261868206037463446B146DB
:1061800016A81BF063F900283ED016A81BF0E7F80C
:106190005FFA80FA15B1504623F046FDBAF13B0F85
:1061A00014D1072C06D81EAB2344013403F8609C9D
:1061B000E4B2F6E706A828F04DF91EAB03EB460360
:1061C000013623F83C0CF6B20024D9E7BAF10D0FE2
:1061D00002D0BAF10A0F10D17EB1092E384606AAB4
:1061E000414694BF8DF818908DF82090FBF762FE21
:1061F00000263844C7B23446C2E71EAB23440134FC
:1062000003F860ACE4B2BBE716A81BF032F9012436
:1062100008E01E490948FAF769FB32461C491D4847
:1062200023F013FF16A81BF0EDF820461FB0BDE8C1
:10623000F08F00BF4488FF1F0888FF1F5CC6FF1F48
:106240000DB9FF1FC5C5FF1FFD87FF1F1E240300DB
:10625000B8BCFF1FA920030058B9FF1FAB200300E3
:106260006CB9FF1F70C5FF1F4D26030080B9FF1FCB
:106270006B23030033D5FF1F5924030038D5FF1FBC
:106280000A88FF1F1CB9FF1F0C1E030028240300EF
:106290003F2403008C8AFF1F2A88FF1FFFFFFFFF98
:1062A0002DE9F04F8B469FB00646002840F024832E
:1062B0000146BB48BB4DDFF880A31DF024FC012143
:1062C000B7481DF01AFCB84BB548B3F90030019639
:1062D0002A880C3A12B21AAC314600920C222827B6
:1062E0001FF094FDB149204623F0FDFF3C233A46C0
:1062F00050210296AE480194009714F013FC2046FA
:1063000023F0B1FFAB49204623F0EDFF3E233A4690
:106310009A210296A8480194009714F003FC2046A5
:1063200023F0A1FFA549204623F0DDFF3E23E22113
:1063300002963A46A2480194009714F0F3FB2046D7
:1063400023F091FF9AF800309E49A84612AE16AD90
:106350002046002B39D04FF4FC6923F0C4FF3C23C6
:106360005A2205219848CDF808900194009714F01E
:10637000D9FB204623F077FF9249284623F0B3FF4C
:106380000A229AF80010B1FBF2F10EA823F0DEFF0A
:106390000EA9304624F011F88C49304624F0BEF89E
:1063A0000146204624F009F84B46224629468648F5
:1063B00014F014FB204623F056FF304623F053FF21
:1063C0000EA823F050FF28460DE023F08CFF46F284
:1063D0002C3302937C48019400973C235A220521D8
:1063E00014F0A0FB204623F03EFF794B79491B783F
:1063F000204623B123F077FF4FF4FC6303E023F042
:1064000072FF46F22C330293282300935A223C2336
:1064100050217148019414F085FB204623F023FF9E
:106420006E4B1B78012B06D16D49204623F05BFF94
:106430004FF4FC631BE0022B01D16A4902E0032BFD
:1064400006D16949204623F04EFF4FF6E0730EE077
:10645000042B06D16549204623F045FF4FF47843CD
:1064600005E06349204623F03EFF46F22C330293B9
:1064700028235A229A2100935E4801943E2314F067
:1064800051FB204623F0EFFE4CF218695A492827A9
:10649000204623F028FF3E235A22E2215748CDF818
:1064A00008900194009714F03DFB204623F0DBFE9A
:1064B0005349204623F017FF3C2305218C225148E5
:1064C000CDF808900194009714F02CFB204623F09F
:1064D000CAFE4D4B4D491B7820462BB123F003FFDC
:1064E0004FF6E073029303E023F0FDFECDF8089031
:1064F0003E238C22E22100974548019414F012FBC0
:10650000204623F0B0FE4349284623F0ECFE4CF22F
:10651000186941492827204623F0E5FE3C23BE2286
:1065200005213E48CDF80C9002940195009714F097
:106530009EFB204623F097FE284623F094FE384920
:10654000204623F0D0FE50213C238C223548CDF844
:1065500008900194009714F0E5FA204623F083FE9A
:1065600040F21B10FAF771F92F490A2800F28480D3
:10657000DFE800F06E060B10646982828282780088
:10658000284623F0B0FE294970E0284623F0ABFEF0
:1065900027496BE0284623F0A6FE264966E000BFA7
:1065A0005CC6FF1F4488FF1F0888FF1F6F2403007D
:1065B00030B9FF1F7724030044B9FF1F8224030072
:1065C00058B9FF1F8C2403006CB9FF1FE525030099
:1065D0004388FF1F9224030080B9FF1FDAC7FF1F03
:1065E00099240300A12403003C2303004223030059
:1065F000A824030094B9FF1FAF240300D0B9FF1FE4
:10660000B9240300A8B9FF1FBCC7FF1FC2240300A1
:1066100034BAFF1FCB240300F42803000CBAFF1F79
:10662000D124030070BAFF1FD9240300E224030021
:10663000E7240300ED2403002DC5FF1F284623F0A7
:1066400052FE974912E0284623F04DFE95490DE091
:10665000284623F048FE9449204623F044FE4CF29D
:10666000186312E0284623F03EFE9049204623F0AE
:106670003AFE4FF4FC6308E0284623F034FE8C49D0
:10668000204623F030FE4FF6E07303932823502179
:10669000BE220093874802943C23019514F0E7FA48
:1066A000204623F0E0FD284623F0DDFD824B8349A0
:1066B0001B78012B04D1284623F015FE804905E004
:1066C000022B09D1284623F00EFE7749204623F0FD
:1066D0000AFE4CF218630AE0032B18D1284623F077
:1066E00002FE7849204623F0FEFD40F2FF7303933B
:1066F00028230093BE223C239A21734802940195DB
:1067000014F0B5FA204623F0AEFD28460FE02046EF
:1067100023F0E9FD46F22C330293282300936A48C4
:1067200001943C23BE229A2114F0FCF9204623F068
:106730009AFD664B1B880BB36549304623F0D3FDA9
:106740006449284623F0CFFD6349204623F0CBFD62
:106750004FF4784304932823BE22E22100935F483C
:1067600003943C230295019614F01CFA204623F072
:106770007AFD284623F077FD304643E0584B1B78DE
:10678000022B0AD15249284623F0ADFD514920463B
:1067900023F0A9FD4FF6E07325E003F0FD02012A86
:1067A0000AD14B49284623F09EFD4A49204623F052
:1067B0009AFD4FF4FC6316E0042B0AD149492846A0
:1067C00023F091FD4349204623F08DFD40F2FF73F5
:1067D00009E03F49284623F086FD3E49204623F044
:1067E00082FD46F22C33039328230093BE223C23E0
:1067F000E2213A480294019514F039FA204623F038
:1068000032FD284623F02FFDB8F800203648083A1C
:10681000002312B201211EF049FCFDF7CBFD082335
:106820000A2232493046F9F75DFE062231462846F3
:1068300023F010FF2E49204623F055FD214628461F
:1068400023F0E5FE0746204623F00DFD284623F001
:106850000AFD67B906233A463146204623F0DAFEA0
:106860002146304623F0B4FD204623F0FCFC46F2DE
:106870002C311D481DF047F9B8F800201A48083A95
:10688000002312B2C8211EF011FC1A491648FAF76B
:106890002DF83146144823F0A1FB01F034BE00BFAF
:1068A000F1240300F9240300BD2D0300012503009A
:1068B000AB210300BCB9FF1FAFC7FF1F09250300B1
:1068C000A92D03008F2103005CBAFF1FCA8EFF1F92
:1068D00010250300A52603005529030048BAFF1F11
:1068E0006CC5FF1F162503005CC6FF1F34C5FF1FC4
:1068F0004D2603001A250300431E012B45F28D810E
:10690000DFF80C83B8F800400328A4F165091FFAEA
:1069100089F940F0CF800027DFF8F8820197B8F8B6
:106920000030B3480D3B1BB200930D2223B2394611
:106930001FF06CFA32463B468221AD481EF0B6FB92
:106940001AADAC49AA48F9F7D1FF4FF01A0AAA4983
:10695000284623F0C8FC64230E224946A748029724
:106960000195CDF800A014F0DDF8284623F07BFC5B
:10697000B8F80080A249A8F11A081FFA88F828463A
:1069800023F0B1FC4246642349469E480297019594
:10699000CDF800A014F0C6F8284623F064FC4FF6AA
:1069A000FF719348DFF874821DF0ADF832463B4624
:1069B00082218F481EF07AFB8E498D48F9F796FFA9
:1069C0002A260797904B9DF81C701B78711EBB42BE
:1069D00089B203D80021052000F029BC2FB98B4AC9
:1069E0003B4612784846FBF7F1F9A4F15E0B4FF6EF
:1069F000FF717F481FFA8BFB0FFA86FA1DF083F8B0
:106A0000002352460FFA8BF179481EF04FFBD8F85D
:106A1000042040F6FF739A4214D198F80930032BF2
:106A200010D8A4F157015246002309B270481EF055
:106A30003DFB3946032014F0FDF931460246584625
:106A4000FCF76AFA724B3946B3F800A0012014F043
:106A5000F1F9AAF1140A1FFA8AFA024631465046A1
:106A6000FCF76EF96A4B3946B3F800A0002014F029
:106A7000E1F9AAF10A0A1FFA8AFA0246314650469B
:106A8000FCF724F9604B0B221B783946284614F09A
:106A9000F9F92946564823F0A1FA284623F0E3FBEA
:106AA000079B01330D360D2B0793B6B208F1A808EA
:106AB00088D18FE7042840F0B3800025554E01951A
:106AC00033884B48544F423B1BB20FFA89F1009375
:106AD000282264231FF09AF94D4B32881B884448C2
:106AE00001951A21643B1A3A00911BB2294612B251
:106AF0001FF08CF932883E48DFF80C910A3A2B4699
:106B000012B201211EF0D2FA4FF6FF7138481CF084
:106B1000FAFF3D782A26CB463B780C33AB42C5F2D0
:106B20007C8099F80030AB4245F27780A4F15E0892
:106B30004FF6FF712E481FFA88F80FFA86FA1CF0FC
:106B4000E2FF002352460FFA88F129481EF0AEFA00
:106B5000324AA82303FB052340F6FF72596891428D
:106B600013D15B7A032B10D8A4F1570152460023AE
:106B700009B21F481EF09AFA2946032014F05AF968
:106B8000314602464046FCF7C7F9214B2946B3F887
:106B90000080012014F04EF9A8F114081FFA88F8BB
:106BA000024631464046FCF7CBF8194B2946B3F86C
:106BB0000080002014F03EF9A8F10A081FFA88F8B6
:106BC000024631464046FCF781F89BF800300B2224
:106BD00029461AA814F056F91AA9054823F0FEF917
:106BE00001351AA80D3623F03EFBEDB2B6B293E79D
:106BF0005CC6FF1F6F240300252503001CB9FF1F7F
:106C00002825030030B9FF1F2AC4FF1FA0C5FF1F9E
:106C10000888FF1F4488FF1FE88EFF1FF88EFF1FA4
:106C2000052840F0A5820025C34A01951288C34873
:106C3000DFF848930D3AA4F1660312B21BB200923A
:106C400029460D221FF0E2F84FF6FF71BB48BC4CFD
:106C50001CF059FF0121B9481CF04FFFB949B74852
:106C60001CF0A6FF31462B462422B448B64E1EF037
:106C70001DFA99F8003021780F221AA814F002F9B1
:106C80001AA9AE4823F0AAF91AA823F0ECFAAB48E7
:106C90001CF0A8FF4CF21861A8481CF034FF2B46EA
:106CA0002D220D21A5481EF001FAA849A348F9F7A5
:106CB0001DFE2B462D225F21A0481EF0F7F9A449A6
:106CC0009E48F9F713FE23789C48A8274FF0020846
:106CD000CDF8008007FB0363D3E91023F9F714FE16
:106CE0004FF6FF7195481CF00EFF2B463A220D21FE
:106CF00092481EF0DBF997499048F9F7F7FD2B46CB
:106D00003A225F218D481EF0D1F991498B48F9F75D
:106D1000EDFD2378CDF8008007FB0363D3E9122350
:106D20008648F9F7F1FD4CF2186184481CF0EBFE3F
:106D30002B4647220D2181481EF0B8F986497F482D
:106D4000F9F7D4FD2B4647225F217C481EF0AEF9AF
:106D50007F497A48F9F7CAFD2378CDF8008007FB10
:106D60000363D3E914237548F9F7CEFD4FF6FF719D
:106D700072481CF0C8FE2B4654220D216F481EF0AD
:106D800095F976496D48F9F7B1FD2B4654225F21FC
:106D90006A481EF08BF96E496848F9F7A7FD237819
:106DA000CDF8008007FB0363D3E916236348F9F7A6
:106DB000ABFD2B466E220D2160481EF077F9684925
:106DC0005E48F9F793FD2B466E225F215B481EF06B
:106DD0006DF95F495948F9F789FD2178284614F083
:106DE00029F8FCF7AFF82178284614F023F86D2134
:106DF00002465120FBF76AFF2B467B220D214F48AC
:106E00001EF054F957494D48F9F770FD2B467B2287
:106E100033214A481EF04AF953494848F9F766FDBC
:106E20007B222B463D2145481EF040F94F4B4348FD
:106E30001978F9F75FFD2B467B2247213F481EF06A
:106E400035F94B493D48F9F751FD2B467B225F212F
:106E50003A481EF02BF93E493848F9F747FD2178AA
:106E6000012013F0E7FFFCF76DF82178012013F003
:106E7000E1FF7A2102465120FBF762FF237807FBEE
:106E8000036340F6FF7259689142B04625D15B7AA0
:106E9000032B22D82B4688220D2128481EF006F904
:106EA00034492648F9F722FD88222B465F212348E2
:106EB0001EF0FCF826492148F9F718FD2178032037
:106EC00013F0B8FFFCF73EF82178032013F0B2FF6F
:106ED000892102465120FCF71FF8002395220D213D
:106EE00016481EF0E3F824491448F9F7FFFC002384
:106EF00095225F2111481EF0D9F815490F48F9F77E
:106F0000F5FC217899F80030A82505FB01810022C5
:106F100091F891101AA813F0B5FF1AA9074823F0A9
:106F20005DF81AA823F09FF90023A2220D2103483F
:106F30001EF0BCF824E000BF4488FF1F5CC6FF1FA2
:106F4000A0C5FF1FB8360300F88EFF1F2B250300D6
:106F50003325030037250300442503004C25030097
:106F6000592503008C2403005E250300BFC7FF1FC3
:106F70006025030062250300692503002AC4FF1F62
:106F8000AD49AE48F9F7B2FC0023A2225F21AB481D
:106F90001EF08CF8AA49A948F9F7A8FC237805FB4C
:106FA000038393F89120FF2A04D1A649A348F9F757
:106FB0009DFC06E002220092D3E926239F48F9F7C0
:106FC000A3FC0023AF220D219C489F4E9F4F1EF033
:106FD0006DF89F499948F9F789FC0023AF225F219A
:106FE00096481EF063F896499448F9F77FFC237899
:106FF000A82505FB038393F86800FBF7A3FF23781C
:1070000005FB038898F86830012B36D10023BC2299
:107010000D218A481EF04AF88E498848F9F766FC27
:107020000023BC225F2185481EF040F88449834834
:10703000F9F75CFC3B788148022405FB036300946C
:10704000D3E92023F9F760FC0023C9220D217B48F6
:107050001EF02CF880497948F9F748FC0023C92232
:107060005F2176481EF022F875497448F9F73EFC16
:107070003B78009405FB036573E0022B44F0CD855B
:107080000023BC220D216D481EF010F873496B4897
:10709000F9F72CFC0023BC22172168481EF006F8E3
:1070A00067496648F9F722FC3B786448082405FBE9
:1070B00003630094D3E91C23F9F726FC0023C922BB
:1070C0000D215E481DF0F2FF65495C48F9F70EFCA2
:1070D0000023C922172159481DF0E8FF5849574895
:1070E000F9F704FC3B78009405FB0363D3E91E2306
:1070F0005248F9F709FC0023BC2271214F481DF0CA
:10710000D5FF58494D48F9F7F1FB0023BC227B21FC
:107110004A481DF0CBFF4A494848F9F7E7FB3B785E
:10712000009405FB0363D3E920234448F9F7ECFB03
:107130000023C922712141481DF0B8FF4A493F4848
:10714000F9F7D4FB0023C9227B213C481DF0AEFF98
:107150003B493A48F9F7CAFB3B7805FB0365002336
:107160000093D5E922233548F9F7CEFB04F055BD4D
:10717000062840F08D8000253C4E019533882F482D
:10718000443B1BB21AAC282200930FFA89F1642306
:107190001EF03CFE3649204623F0A5F83423422257
:1071A00049460093334802956423019413F0BAFCD6
:1071B000204623F058F81A272F49204623F093F849
:1071C0006423AA2249462D4802950194009713F0A2
:1071D000A9FC204623F047F82949204623F083F8EC
:1071E00064230E224946274802950194009713F024
:1071F00099FC204623F037F8368823491A3EB6B268
:10720000204623F070F86423324649461F48029511
:107210000194009713F086FC204623F024F82C21DB
:1072200002202B465A46FAF7D1FD29460720FFF7E0
:1072300037F804F0F2BC00BF732503005CC6FF1FE3
:10724000332503007C250300F88EFF1FA0C5FF1F18
:1072500080250300872503008A2503007E2503007F
:107260002C230300ED540300182403004488FF1F5F
:107270009223030044B9FF1F8D250300D0B9FF1FDF
:10728000252503001CB9FF1F2825030030B9FF1F67
:10729000072829D161B9114A128801911A20A4F155
:1072A00064031A3A00901BB212B20D481EF0AEFDF4
:1072B00000210B481CF027FC0A4B1A78052A1AAC4F
:1072C0001D4604F091811A78062A04F08D811A78FF
:1072D000072A44F0AE8104F087B900BF4488FF1F3D
:1072E0005CC6FF1FEAC6FF1F092840F06F83FF2915
:1072F00040F0C2810025DFF878A3BF4EDFF874B3F9
:10730000FDF730FCB8F900300195BAF80020BB4811
:107310000D3A12B2009229460D221EF077FDB849AF
:10732000B6481CF045FC2B4624220521B3481DF02D
:10733000BDFEB449B148F9F7D9FAFDF713FCB248DC
:107340001AAC13F07FFAB14813F07CFAB04920462A
:1073500022F0C9FF34234222494601940093AD48EC
:107360000295642313F0DEFB204622F07CFFAA493D
:10737000204622F0B8FF7378A8483BF813300293F8
:107380001A276423792249460194009713F0CAFB17
:10739000204622F068FFA249204622F0A4FF642381
:1073A00049460E2201949F480295009713F0BAFBBC
:1073B000204622F058FFBAF800209B491A3A92B2B0
:1073C0002046079222F08FFF6423079A01944946D2
:1073D00096480295009713F0A5FB204622F043FF44
:1073E000BAF800909249A9F11A091FFA89F92046C2
:1073F00022F079FF13234A46294601948D480295CD
:10740000009713F08FFB204622F02DFFB8F8009074
:10741000BAF800208849A9F17D091A3A92B21FFAF8
:1074200089F92046079222F05EFF49461323079A06
:10743000019482480295009713F074FB204622F0D5
:1074400012FFB8F80030BAF800206C4844F2082E59
:107450000221A03B0C3A8DE802401BB212B2192166
:107460001EF0D4FCB8F80000963825F089FF002201
:10747000734B25F037FE80463078894625F070FF43
:1074800002460B464046494625F0E0FF00226D4B80
:1074900026F006F900226A4B25F026FE26F0AEFA09
:1074A000BAF800806849A8F11A081FFA80F91FFA93
:1074B00088F8204622F017FF0A23424649460194E5
:1074C00062480295009713F02DFB204622F0CBFE78
:1074D000FDF748FB2D2427B23A4600230D214748EB
:1074E0001DF0E4FD05F1010859494448F9F7FEF99A
:1074F00041464248F9F702FA06EB4503621E5B7803
:107500003E483BF8133001930923009312B20A233B
:1075100073211EF07BFC3A4600233F2137481DF0C3
:10752000C5FD16F8151035486423594345461F46D6
:107530000D34F9F7E3F9082DA4B2CCD1A22200232F
:107540000D212E481DF0B2FD42492C48F9F7CEF925
:10755000414B187825F004FF03230024672502938C
:10756000A223019302460B460494039400953B48E2
:1075700015F066FA2346AF220D2120481DF096FD36
:1075800037491E48F9F7B2F9364B187810FB07F067
:1075900025F0F6FE0526AF23019302460B46049420
:1075A0000394029600952D4815F04AFA2346BC2212
:1075B0000D2112481DF07AFD2B491048F9F796F974
:1075C000BC230193049403940296009500220023A7
:1075D000224815F035FA2346C9220D2107481DF02F
:1075E00065FD22490548F9F781F9234622462D21F8
:1075F0000220FAF7EBFBBCE12F88FF1F5CC6FF1FE0
:10760000B836030077240300A8B9FF1FBCB9FF1FD9
:107610009D25030044B9FF1FA225030094B9FF1F55
:10762000252503001CB9FF1F2825030030B9FF1FC3
:10763000A920030058B9FF1FAB2003006CB9FF1F3E
:107640000000394000005E404D26030080B9FF1F56
:10765000A8250300AD250300FC87FF1FB8BCFF1F52
:10766000B92503004188FF1FC5250300CB24030073
:107670004488FF1F1488FF1F012940F07A81C14D03
:107680002E78082E5ED8C04F963C17F8160000944E
:10769000192378220021F9F78CF8BC4EA3B281B2ED
:1076A000192206F1640013F033FBFDF75BFA2B7827
:1076B000B74803EB430203EB820200240A232D3276
:1076C0008DE8180012B21E233F211EF09FFB2B787D
:1076D000AF4803EB430203EB82022D3212B2234682
:1076E0003F211DF0E3FC2B78A94817F81310642301
:1076F00059431AACF9F702F9A649B6F88080B6F8F2
:107700008290B6F884A0B6F886B0204622F0EBFD51
:107710002B7807EB4307A04B7A7833F812300293AB
:107720004A465346414606F178000194CDF800B030
:1077300013F0F8F9204622F096FD06F18C00F9F7D7
:1077400011F988E0092E27D1944E963C30780094A8
:107750001923FF220021F9F72CF8A3B281B21922D4
:107760008F4813F0D5FAFDF7FDF92B78884803EB25
:10777000430203EB820200240A232D328DE8180015
:1077800012B21E2367211EF041FB307825F0E8FD80
:107790000494039403234EE00A2E21D1814F963C9A
:1077A00038780094192378220021F9F702F8A3B25F
:1077B00081B219227A4813F0ABFAFDF7D3F92B788E
:1077C0007348009603EB430203EB82022D32002440
:1077D00001941E2312B267211EF018FB387823E0B3
:1077E0000B2E38D1704E963C3078009419237822B5
:1077F0000021F8F7DEFFA3B281B21922684813F026
:1078000087FAFDF7AFF92B78614803EB430203EBEE
:1078100082022D320A2300248DE8180012B21E23A2
:1078200067211EF0F3FA30786423584325F0A8FD51
:1078300004940394052302932B7803EB430203EB98
:1078400082032D339BB201936723009302460B46BC
:10785000564815F0F5F82B780C2B40F08A804FF441
:10786000D470F8F7F2FF494C5149B4F88060B4F88D
:107870008270B4F88480B4F8869001281AAD0CBFE9
:107880004FF01F0A4FF4FC6A284622F02CFD3A46BE
:1078900043463146CDF808A0CDF8009004F17800B9
:1078A000019513F03FF9284622F0DDFC4149B4F878
:1078B0008690B4F88080B4F884A0B4F8826016A8EA
:1078C00022F011FD3C4B12A8197822F02CFD12A9D0
:1078D00016A822F01BFE4E4403360146B6B200271E
:1078E000284622F06AFD324653464146CDF80090C4
:1078F00004F18C000297019513F014F9284622F048
:10790000B2FC12A822F0AFFC16A822F0ACFCB4F82E
:107910009A30B4F89660B4F88080B4F88490B4F8E3
:1079200086A01E44254B12A8197822F0FCFC12A94F
:1079300016A822F042FD224916A822F0EFFD0336D8
:107940000146B6B2284622F038FD4B463246414643
:1079500004F1A00002970195CDF800A013F0E2F821
:10796000284622F080FC16A822F07DFC12A803F025
:10797000AABF1448F8F7F6FF1348F8F7F3FF04F02E
:107980004CB900BFA0C5FF1F2F88FF1F1CB9FF1FE8
:107990005CC6FF1FA22503001488FF1FFC87FF1F82
:1079A00080B9FF1F4188FF1F3E8EFF1FB8BCFF1F1D
:1079B000D1250300DB250300F08EFF1F2BC4FF1F22
:1079C000E1250300A8B9FF1FBCB9FF1F0A286FD12A
:1079D00000220C2044F2082311468DE8090023B24E
:1079E000AF481EF013FAFDF7BDF8002303228221F1
:1079F000AB481DF05BFBAB49A948F8F777FFB8F837
:107A00000010A7480B2646F22C3732392D230122CD
:107A100009B28DE8C0001EF0F9F9B8F80040A2499B
:107A20001E3C0525A4B21AA822F05DFC1AAB032265
:107A300021469E48009513F08BFD1AA822F013FCF6
:107A4000BBF1000F0CBF3B464FF47843012201937A
:107A500029462E23924800961EF0D8F994491AA878
:107A600022F041FC1AAB032219219048009513F033
:107A70006FFD1AA822F0F7FBBBF1000F0CBF4FF40B
:107A800078433B460122019337212E2384480096F8
:107A90001EF0BCF987491AA822F025FC83480095FE
:107AA0001AAB03224B2113F053FD1AA803F00BBFAE
:107AB0000B2804F0B2800C2840F0A68100267E4FEF
:107AC00001963B8876480D3B1BB20D220093314650
:107AD00023B21EF09BF94FF6FF7171481CF013F8AA
:107AE00001216F481CF009F874496D481CF060F8DA
:107AF0003346242205216A481DF0D8FA70496848A7
:107B0000F8F7F4FE66481CF06DF83A8864480A3AC3
:107B1000334612B205211AAC1DF0C8FA6949604813
:107B2000F8F7E4FE08230A2267492046F8F7DAFC52
:107B300021465B4822F052FA204622F094FB3A8814
:107B400057480A214FF478430B3A12B28DE80A00E5
:107B500016AD782331461CF0A3FA5C49284622F082
:107B6000C2FB40F29F10F8F770FE25F0F9FB0246C9
:107B70000B4600204FF0804122F070FF544B002252
:107B800025F064FC25F05AFF4FF028080146022238
:107B9000204622F02EFC3C23912205214D480396DD
:107BA00002940195CDF8008013F061F8204622F090
:107BB0005AFB284622F057FB4749204622F093FB08
:107BC00005213C232D22454802960194CDF80080E2
:107BD00012F0A8FF204622F046FB4FF4E570F8F7BC
:107BE00034FEBA463E493F4F48B1284622F07BFB5F
:107BF0003D49204622F077FB4FF4FC6308E028461D
:107C000022F071FB3849204622F06DFB46F22C33FE
:107C10005F2205210393CDF800803C2307F1640027
:107C20000294019513F023F8204622F01CFB28460D
:107C300022F019FB2D49284622F055FB2C492046FD
:107C400022F051FB4FF028084CF2186350215F22BC
:107C50000393284802943C230195CDF8008013F04B
:107C600006F8204622F0FFFA284622F0FCFA4FF4EC
:107C7000D870F8F726FE12AE83461F493046BBF196
:107C8000000F3FD022F02FFB1C49284622F02BFB8F
:107C90001B49204622F027FB4FF4FC6304933DE090
:107CA0005CC6FF1F82240300E7250300B8BCFF1F4A
:107CB000B5240300EC2503004488FF1FB8360300F9
:107CC000B9240300F325030034C5FF1F0626030073
:107CD00000405F4044B9FF1F1026030058B9FF1F42
:107CE000152603001CB9FF1F1D2603006C25030089
:107CF0003C26030094B9FF1F922803006829030063
:107D0000C92C030022F0EFFA3649284622F0EBFA9C
:107D10003549204622F0E7FACDF810B03C239122F5
:107D2000502102950196CDF8008003942F4812F05F
:107D300039FF204622F097FA284622F094FA30467E
:107D400022F091FA40F21910F8F77FFD2D239B22C3
:107D50000821FAF7C9FE2649204622F0C4FA002677
:107D600028235F2200939B213C2302960194214803
:107D700012F0D8FE204622F076FA4FF01A081E497B
:107D8000204622F0B0FA64230E224946029601945E
:107D9000CDF80080194812F0C5FE204622F063FAA3
:107DA000BAF8005016491A3DADB2204622F09BFAAF
:107DB0002A464946642302960194CDF80080114872
:107DC00012F0B0FE204622F04EFAFDF77BFAFB8956
:107DD0007989388919443246334689B2F9F7F6FF72
:107DE00003F01BBF6829030025260300A8B9FF1F65
:107DF0002E260300D0B9FF1F252503001CB9FF1F45
:107E00002825030030B9FF1F0D2840F00485FF2905
:107E100040F0DD83BC4D00242819143412F012FD0B
:107E2000B4F5027FF8D1B94BB94AB3F90030B9487B
:107E3000B94EBA4F0024019412880D3A12B2009242
:107E400021460D221DF0E2FF46F22C3503220223CB
:107E50008DE82C0005214FF49B738C22AD481EF059
:107E60002DF84FF6FF71AB481BF04DFE0121A948DC
:107E70001BF043FEAA49A7481BF09AFE2346242282
:107E80000521A4481DF012F9A649A248F8F72EFDD5
:107E9000A0481BF0A7FE29469E481BF034FE306820
:107EA000716832890EAB03C301201A80F8F7CDFC4C
:107EB0003B7883420CD99C4BA82202FB003000F196
:107EC00010030EAA53F8050F59681B7A03C21370EA
:107ED00016AC1AAD4FF0000894498DF84180204649
:107EE00022F001FA0EA9284622F0FDF928232D22BE
:107EF000052100938448CDF80C803C230295019421
:107F000012F0B5FE284622F0AEF9204622F0ABF979
:107F100030687168327A0EAB03C303201A70F8F729
:107F200094FC3B7883420CD97F4BA82202FB0030A3
:107F300000F110030EAA53F8050F59681B7A03C20B
:107F400013704FF000087A498DF84180204622F0E6
:107F5000CAF90EA9284622F0C6F928232D2250215D
:107F600000937448CDF80C803C230295019412F0E4
:107F70007EFE284622F077F9204622F074F9306818
:107F80007168327A0EAB03C304201A70F8F75DFCF7
:107F90003B7883420CD9644BA82202FB003000F1ED
:107FA00010030EAA53F8050F59681B7A03C2137009
:107FB0004FF0000860498DF84180204622F093F987
:107FC0000EA9284622F08FF928232D229B21009309
:107FD0005A48CDF80C803C230295019412F047FEDC
:107FE000284622F040F9204622F03DF930687168B9
:107FF000327A0EAB03C305201A70F8F726FC3B78E3
:1080000083420CD9484BA82202FB003000F1100338
:108010000EAA53F8050F59681B7A03C213704FF06C
:10802000000847498DF84180204622F05CF90EA9EE
:10803000284622F058F928232D22E62100934148B2
:10804000CDF80C803C230295019412F010FE2846D6
:1080500022F009F9204622F006F930687168327A78
:108060000EAB03C306201A70F8F7EFFB3B78834290
:108070000CD92D4BA82202FB003000F110030EAAF0
:1080800053F8050F59681B7A03C2137000272E4955
:108090008DF84170204622F026F90EA9284622F0DC
:1080A00022F9039728273C235A22052127480295C5
:1080B0000194009712F0DBFD284622F0D4F8204608
:1080C00022F0D1F830687168327A0EAB03C31A70AF
:1080D0001F4B20491E78012E204603D122F003F9C0
:1080E0001D4958E0022E03D122F0FDF81B4952E051
:1080F000032E03D122F0F7F819494CE0042E33D1B6
:1081000022F0F1F8174946E01CB9FF1F0888FF1F4D
:108110004488FF1F5CC6FF1F452603002AC4FF1FBB
:10812000B836030035260300F88EFF1F41260300F2
:108130000A26030044B9FF1F4F26030058B9FF1F4A
:10814000562603006CB9FF1F5D26030048BAFF1FC7
:108150003C8DFF1F622603006E260300722603007B
:10816000762603007A260300052E0FD122F0BBF8F5
:10817000B349284622F0B7F84FF4FC630393029505
:10818000019400973C239622314619E0062E08D12F
:1081900022F0A9F8AB49284622F0A5F84FF4FC6379
:1081A00007E022F0A0F8A849284622F09CF846F201
:1081B0002C3303930295019400973C2396220521CA
:1081C000A24812F054FD284622F04DF8204622F035
:1081D0004AF89F4B9F491B7812AE012B304607D1BE
:1081E00022F081F89C49204622F07DF89B4930E03E
:1081F000022B07D122F077F89749204622F073F836
:10820000974926E0032B07D122F06DF892492046CA
:1082100022F069F893491CE0042B07D122F063F89F
:108220008D49204622F05FF88F4912E0052B07D1D7
:1082300022F059F88849204622F055F8804908E094
:10824000062B0CD122F04FF88349204622F04BF840
:108250007C49284622F047F84FF4FC630BE022F0FB
:1082600042F87D49204622F03EF87749284622F020
:108270003AF846F22C33049328239622E621009301
:108280007A4803953C230294019612F08BFC284611
:1082900021F0E9FF204621F0E6FF304621F0E3FF20
:1082A000734BDFF8E4911A7899F80080FF2A4FF4B5
:1082B000CD709A464FF6E07718BF4FF4FC67F8F799
:1082C000C4FA804505D16B49204622F00CF8634979
:1082D0003EE040F29B10F8F7B8FA804505D16549B9
:1082E000204622F000F85E4932E04FF4CE70F8F7F5
:1082F000ACFA804505D15F49204621F0F4FF594989
:1083000026E040F29D10F8F7A0FA80455949204632
:1083100003D121F0E8FF54491AE0B8F1000F03D16E
:1083200021F0E1FF464913E0B8F1010F03D121F03C
:10833000DAFF44490CE0B8F1090F03D121F0D3FF73
:108340004D4905E0B8F10A0F07D121F0CCFF4B49A8
:10835000284621F0C8FF039708E021F0C4FF3A49FE
:10836000284621F0C0FF46F22C330393282396229F
:1083700050210093424802953C23019412F077FC6F
:10838000284621F070FF204621F06DFF9AF8013059
:1083900099F80180FF2B4FF4CD704FF6E07718BFAE
:1083A0004FF4FC67F8F751FA804505D1354920466E
:1083B00021F099FF29493EE040F29B10F8F745FA79
:1083C000804505D12F49204621F08DFF244932E018
:1083D0004FF4CE70F8F739FA804505D12949204687
:1083E00021F081FF1F4926E040F29D10F8F72DFA99
:1083F00080452449204603D121F075FF1A491AE02F
:10840000B8F1000F03D121F06EFF0D4913E0B8F170
:10841000010F03D121F067FF0A490CE0B8F1090F01
:1084200003D121F060FF144905E0B8F10A0F2DD106
:1084300021F059FF1149284621F055FF03972EE0FE
:10844000B7210300B32103008A28030030B9FF1FBE
:10845000E8C4FF1F7E260300672603006E26030084
:1084600072260300762603007A260300E4B9FF1F74
:108470003F88FF1F89260300BB210300BF210300A3
:108480000CBAFF1F91260300BDC7FF1F21F02BFF71
:108490006849284621F027FF46F22C33039328230E
:1084A0009B2196220093644802953C23019412F08C
:1084B000DEFB284621F0D7FE204621F0D4FE5F4B9C
:1084C0005F491F78012F304620D121F00CFF5D4914
:1084D000204621F008FF5C49284621F004FF4FF4B4
:1084E000FC630493282300930395029401963C2394
:1084F000C3220521554812F055FB284621F0B3FE52
:10850000204621F0B0FE304603F0DDB9022F07D13E
:1085100021F0E9FE4B49204621F0E5FE4C49DBE71E
:10852000032F07D121F0DFFE4649204621F0DBFE74
:108530004849D1E7042F07D121F0D5FE4149204613
:1085400021F0D1FE4449C7E7052F15D121F0CBFE1C
:108550003C49204621F0C7FE4049284621F0C3FE91
:108560004FF4FC630493282300930395029401962F
:108570003C23C3223946BDE7062F07D121F0B3FEC5
:108580003049204621F0AFFE3549A5E7072F07D136
:1085900021F0A9FE2B49204621F0A5FE31499BE799
:1085A000082F07D121F09FFE2649204621F09BFE8F
:1085B0002D4991E721F097FE2249204621F093FEB4
:1085C0001C49284621F08FFE46F22C3389E72749C3
:1085D000274B0A781B78DFF89C90501E98428846FB
:1085E00016D00AB9FF2B13D09A4217D099F8001071
:1085F0008A4201D1FF2B11D0501C834213D08A42F2
:1086000000D183B101398A4236D1FF2B34D10AE03F
:1086100044F208252E464FF4FC6731E044F2082569
:108620004FF4FC662BE044F208264FF4FC65374615
:1086300026E000BF8A28030020BAFF1FE8C6FF1FFC
:1086400099260300F52103006E26030034BAFF1FAC
:1086500072260300762603007A260300B721030062
:10866000B3210300BB210300BF210300A0C5FF1FEE
:10867000E88EFF1F2AC4FF1F44F208252E462F460E
:10868000DFF860A28A49BAF800B01AACABF11A0B55
:10869000204621F028FE1FFA8BFB02971A275A4624
:1086A0003323372183480194009712F03BFA204688
:1086B00021F0D9FDBAF800207F48113A002312B208
:1086C00039211CF0F3FC98F8001099F800300139BA
:1086D0000822C9B2204612F0D5FB2146764821F087
:1086E0007DFC204621F0BFFDBAF800B07049ABF127
:1086F0001A0B1FFA8BFB204621F0F5FD33235A4657
:10870000702102966D480194009712F00BFA2046F2
:1087100021F0A9FDBAF800206748113A002312B2EF
:1087200073211CF0C3FC99F8003098F8001008225F
:10873000204612F0A7FB21465F4821F04FFC20465F
:1087400021F091FDBAF8006059491A3EB6B22046B0
:1087500021F0C9FD32463323A921029558480194DE
:10876000009712F0DFF9204621F07DFDBAF80020D5
:108770005148113A002312B2AC211CF097FC98F832
:10878000001099F8003001310822C9B2204612F0D9
:1087900079FB2146484821F021FC204621F063FD69
:1087A000BAF8005047491A3D0026ADB2204621F0E4
:1087B0009AFD2A4633233146434802960194009796
:1087C00012F0B0F9204621F04EFDBAF800503F49B2
:1087D0001A3DADB2204621F086FD2A463323E22120
:1087E0003B4802960194009712F09CF9204621F034
:1087F0003AFDBAF8005037491A3DADB2204621F093
:1088000072FD02960194009727232A464FF48C713B
:10881000314801F09ABC142840F03984FF29DFF870
:10882000C8804FF0000600F032812D22631F0092B5
:1088300001961BB2C32205211F481DF0E7FA08EB81
:108840000600143611F0FEFFB6F5027FF7D123497A
:10885000234B0A781B78DFF89490501E9842884684
:1088600015D00AB9FF2B12D09A4216D099F80010F1
:108870008A4201D1FF2B10D0501C834212D08A4271
:1088800000D17BB1884233D1FF2B31D10AE044F2D1
:1088900008252E464FF4FC672EE044F208254FF4DD
:1088A000FC6628E044F208264FF4FC65374623E0D6
:1088B0004D26030080B9FF1F5CC6FF1F94B9FF1F40
:1088C000A8B9FF1FA9200300BCB9FF1FAB200300FC
:1088D000D0B9FF1F92230300F8B9FF1FA0C5FF1FE7
:1088E000E88EFF1F4488FF1F1CB9FF1F2AC4FF1F0B
:1088F00044F208252E462F46DFF82CA3BF49BAF8CC
:1089000000B01AACABF11A0B204621F0ECFC1FFAB8
:108910008BFB02971A275A4633233721B848019414
:10892000009712F0FFF8204621F09DFCBAF80020D5
:10893000B448113A002312B239211CF0B7FB98F861
:10894000001099F8003001390822C9B2204612F00F
:1089500099FA2146AB4821F041FB204621F083FCE7
:10896000BAF800B0A549ABF11A0B1FFA8BFB2046F1
:1089700021F0B9FC33235A4670210296A248019493
:10898000009712F0CFF8204621F06DFCBAF80020D5
:108990009C48113A002312B273211CF087FB99F80E
:1089A000003098F800100822204612F06BFA214699
:1089B000944821F013FB204621F055FCBAF80060E2
:1089C0008E491A3EB6B2204621F08DFC3246332342
:1089D000A92102958D480194009712F0A3F8204632
:1089E00021F041FCBAF800208648113A002312B267
:1089F000AC211CF05BFB98F8001099F800300131B5
:108A00000822C9B2204612F03DFA21467D4821F0E5
:108A1000E5FA204621F027FCBAF800507C491A3DBF
:108A20000026ADB2204621F05EFC2A4633233146B3
:108A3000784802960194009712F074F8204621F0CD
:108A400012FCBAF8005074491A3DADB2204621F02C
:108A50004AFC2A463323E22170480296019400978B
:108A600012F060F8204621F0FEFBBAF800506C4985
:108A70001A3DADB2204621F036FC029601940097D3
:108A800027232A464FF48C71664801F05EBB664B83
:108A900001961B885B480D3B1BB20D2200933146AB
:108AA00023B21DF0B3F94FF6FF7156481BF02BF8B7
:108AB000012154481BF021F85C4952481BF078F81A
:108AC0003346242205214F481CF0F0FA58494D48FE
:108AD0001AADF7F70BFF4B481BF084F855492846B1
:108AE00021F001FC544B16AC282719880A22204695
:108AF00021F02CFC2D223C230521404603960294B4
:108B00000195009712F0B3F8204621F0ACFB2846FF
:108B100021F0A9FB4949284621F0E5FB484B2046B6
:108B20001978FAF7AFF82D223C23502108F11400F0
:108B3000039602940195009712F099F8204621F0CF
:108B400092FB284621F08FFB3E49284621F0CBFBC3
:108B50003D4B2046197821F0E6FB2D223C239B213A
:108B600008EB0700039602940195009712F07FF836
:108B7000204621F078FB284621F075FB3349284632
:108B800021F0B1FB324B2046197821F0CCFB3C237D
:108B900008EB03002D22E62103960294019500972D
:108BA00012F065F8204621F05EFB284621F05BFBC1
:108BB000284A1378012B91460AD12749204621F0F3
:108BC00092FB2649284621F08EFB4FF4FC6355E0CA
:108BD000032B05D12049204621F085FB204906E0E2
:108BE000042B41D11F49204621F07DFB1B4928461B
:108BF00021F079FB40F2FF7340E000BF4D260300F7
:108C0000E4B9FF1F5CC6FF1FF8B9FF1F0CBAFF1FB6
:108C1000A920030020BAFF1FAB20030034BAFF1FB6
:108C20009223030048BAFF1F4488FF1FB836030091
:108C30009F260300AD260300EAC4FF1FB7260300EA
:108C40000AB9FF1FBC260300F8B8FF1FC7260300A0
:108C5000EEC9FF1F6CC5FF1FD22603007828030052
:108C6000D926030016250300A749204621F03BFB27
:108C7000A649284621F037FB4FF6E0735A2205211A
:108C8000039308F150003C2302950194009711F0E2
:108C9000EEFF284621F0E7FA204621F0E4FA9C4B4B
:108CA0001E7876B9314640F2CF10F7F761FD994949
:108CB000204621F018FB9549284621F014FB039625
:108CC0000FE0012140F2CF10F7F752FD9149204605
:108CD00021F009FB9049284621F005FB4FF4FC6385
:108CE000039328235A22502100938C4802953C2359
:108CF000019411F0BCFF284621F0B5FA204621F07E
:108D0000B2FA99F80030032B40F081808449204664
:108D100021F0E9FA002728268249284621F0E3FAC3
:108D20003C235A229B218048039702950194009688
:108D300011F09DFF284621F096FA204621F093FA83
:108D40007A49284621F0CFFA794B0A221988204621
:108D500021F0FCFA3C2387220521764803970294F0
:108D60000195009611F083FF204621F07CFA2846F9
:108D700021F079FA7049284621F0B5FA6F4B0A22A2
:108D80001988204621F0E2FA3C23872250216C48C2
:108D9000039702940195009611F069FF204621F097
:108DA00062FA284621F05FFA6649284621F09BFACC
:108DB000654B0A221988204621F0C8FA3C238722F5
:108DC0009B216248039702940195009611F04FFF92
:108DD000204621F048FA284621F045FA5C49284609
:108DE00021F081FA5B4B0A221988204621F0AEFA65
:108DF0003C238722E6215848039702940195009668
:108E000011F035FF204621F02EFA284617E053498D
:108E1000204621F068FA5249284621F064FA0023DE
:108E20000393282300935A223C239B213E4802951A
:108E3000019411F01CFF284621F015FA204621F07C
:108E400012FA4849484F204621F04DFA002644497D
:108E500028464FF0280821F046FA3C235A22E62102
:108E60000396424802950194CDF8008011F0FFFE70
:108E7000284621F0F8F9204621F0F5F946F22C3980
:108E80000A234FF0030B8DE80808B6224FF49B73BA
:108E900005213748CDF808901DF010F83346B72269
:108EA0002D2133481CF002F9FBF75CFE31493048B4
:108EB000F7F71CFD0722B7212520FAF7F7FCB721A9
:108EC000FA200722FAF7F2FC3E782B492046002EC2
:108ED00058D021F008FA2949284621F004FA4FF425
:108EE000FC630393C7223C23052102950194CDF82E
:108EF0000080234811F0BBFE284621F0B4F920463B
:108F000021F0B1F95CE000BFD22603008A280300FB
:108F100028C4FF1FDD2603007828030080B9FF1F47
:108F2000E4260300102503005CBAFF1F1824030089
:108F300066C5FF1F84BAFF1F182503003E8DFF1F63
:108F400098BAFF1FCD29030034D5FF1FACBAFF1F0D
:108F5000EB26030008B9FF1FC0BAFF1FF726030066
:108F600026550300FF260300B0C5FF1F70BAFF1F80
:108F70005CC6FF1F0627030036270300C92C030029
:108F800094B9FF1F21F0AFF9BC49284621F0ABF995
:108F90003C23C7220521BA48CDF80C9002950194D4
:108FA000CDF8008011F063FE284621F05CF92046E0
:108FB00021F059F931464FF4E870F7F7D9FB3E70CC
:108FC000B049284621F08FF9AF4B20461978F9F7C0
:108FD00059FE00262823C72250210093AB48039650
:108FE0003C230294019511F042FE204621F03BF90A
:108FF000284621F038F9A64A51681068128912AB48
:1090000003C3A4491A80A44B09781A78914202D26A
:10901000FF221A700DE0A14BA82101FB023310338F
:1090200012AA53F8050F59681B7A03C213708DF802
:1090300051609B49204621F056F9002712A92826A5
:10904000284621F050F93C23C7229B2195480397DD
:1090500002950194009611F00AFE284621F003F9CA
:10906000204621F000F99049204621F03CF98F4B31
:1090700002221968284621F0BCF903970295019451
:1090800000963C23C722E621894802F070B81628D2
:1090900040F08E82FF294FF0000440F04581854D5D
:1090A0002819143411F0CEFBB4F5027FF8D10A244C
:1090B0000025C02601944FF49B73302205217E4881
:1090C000029500961CF0FAFE4CF2186330220293CF
:1090D00001944FF49B730521774800961BF002FD25
:1090E0004FF6FF7174481AF00EFD012172481AF014
:1090F00004FD724970481AF05BFD2B464A22214656
:109100006D486F4C1BF0D2FF6E496B48F7F7EEFBD2
:1091100069481AF067FD022167481AF047FC237876
:10912000694AD25C5B4B1B789A424ED22726237841
:10913000DFF8949121782278584F19F80110DBB2AA
:109140000793237819F803304FF0A80808FB03733E
:1091500008FB017193F814A019F8023008FB03739F
:10916000D3E91223D1E9160123F0BCFF0022574BAB
:1091700024F096FACDE90801284624F001F90246C8
:109180000B46DDE9080124F061F9079B19F803306B
:1091900008FB0377D7E9122323F0A6FF24F04EFC47
:1091A0001AAB524601211EF0DBFD32B200231A2118
:1091B00041481BF07BFF01351AA93F48F7F796FBA2
:1091C00018360B2DB6B2B2D105E02078FF2100F59C
:1091D000F770F7F7CDFA03213748DFF80481DFF89D
:1091E000B490DFF800A11AF0E1FB46F22C313248CE
:1091F0001AF089FC002365220C212F481BF056FF32
:1092000033492D48F7F772FB00237A2210212A48B0
:109210001BF04CFF2F492848F7F768FB00238F22EB
:109220001E2125481BF042FF00212348F7F766FB6B
:109230000023A322102120481BF038FF26491E4896
:10924000F7F754FB0023B7220C211B481BF02EFF1D
:1092500022491948F7F74AFB07250024184B1A78CA
:10926000E3B29A4208D198F8013099F800209A4266
:109270003AD98AF8003037E0002737E02526030086
:1092800094B9FF1FB7260300DF8EFF1FA8B9FF1F89
:10929000452603002AC4FF1F14CAFF1FF88EFF1FB4
:1092A0006C250300BCB9FF1F76250300B8C7FF1F5C
:1092B000D0B9FF1F1CB9FF1F5CC6FF1FB8360300E3
:1092C000EAC6FF1F3E270300D08EFF1F0000244088
:1092D00050270300562703005B2703006027030085
:1092E000CF8EFF1FA0C5FF1F4FF4FC671AAE99F881
:1092F000003018F8011F0A22304611F0C3FD9F4AC2
:10930000142303FB042029468DE8C8004D223A238C
:109310003C3011F007FC0134304620F0A4FF3E350C
:10932000052CADB29AD108E05C2300930194F82398
:109330006422272192481CF069FD672441F2A205AE
:1093400022B215340095F1232A218D48A4B21CF0D5
:10935000BFFED02CF4D12A2441F2A20521B2183448
:109360000095542368228648A4B21CF053FEB4F53D
:10937000997FF3D1834C844E2378844DF25C2B7813
:109380009A4206D3BBF10B0FDFF820825FD902F0BF
:10939000B8BA22787E4F0B235A434FF00B08BA56C7
:1093A000642AC1BF227853430022FA54237808FB71
:1093B00003F34FF02A09FA566FF0530364325A430D
:1093C000C92392FBF3F2BC3292B24FF0010A237828
:1093D00008FB037313F90A30642B02F38A82694B8A
:1093E0006B491B7808FB031313F90A306433C2F28C
:1093F0008082237808FB03736FF0530113F90A305E
:1094000064334B43C92193FBF1F3BC33662B03DD7B
:10941000BC2BA8BFBC2300E0672399B207910FFAC9
:1094200089F109F118091FFA89F94FF478401BB244
:109430000190009312B20FFA89F351481AF0F0FD2F
:10944000B9F58D7F0AF1010A9CD0079ABFE723780E
:109450004C4FF25C2B789A4282F053823B784C4C12
:1094600047480B2505FB03430BEB4B0113F90B207E
:109470006FF0530364324FF478465A43C900C9234E
:1094800092FBF3F2BC320096032312B22A311BF096
:10949000BFFA4FF003090296152632233522F9212F
:1094A00037488DE840021CF009FD4FF6FF71344843
:1094B0001AF029FB374932481AF07AFB4A22002376
:1094C000FA212F481BF0F2FD3B782D4805FB0344A1
:1094D0001AAD14F90B10F7F711FA29481AF082FBAC
:1094E00000242D492846242720F0FDFE182364225D
:1094F0004FF49371019521480294009711F012FBEB
:10950000284620F0B0FE2549284620F0ECFE18231E
:10951000CC224FF49371019521480294009711F0E9
:1095200001FB284620F09FFE1E49284620F0DBFE66
:109530003C238C224FF49371019500931A480294B6
:10954000182311F0EFFA284620F08DFEB8F800201D
:109550000B480294183A8DE840024FF48A7312B215
:1095600011211CF0ABFC054D04F1C8002844143453
:1095700011F068F9642CF7D102F04FBB1CB9FF1F42
:109580005CC6FF1FEAC6FF1FD08EFF1F2AC4FF1F45
:10959000ABC6FF1FB83603002525030028250300AE
:1095A00030B9FF1F8B27030044B9FF1F4488FF1FFA
:1095B000182840F06283FF294FF0000440F08281B8
:1095C000B24D2819143411F03DF9B4F5027FF8D1E9
:1095D0000024AC250A2640F22B1330221421AC487B
:1095E00002948DE860001CF069FC4CF21863302294
:1095F0000293142140F22B13A5488DE860001BF064
:1096000071FA4FF6FF71A2481AF07DFA0121A048C5
:109610001AF073FA9F499E481AF0CAFA23464A2262
:1096200019219B481BF042FD9B499948F7F75EF9C9
:109630009A4A9B4910780B780891984292460BD22F
:1096400011781AA8082211F01DFC1AA9904820F0E0
:10965000C5FC1AA820F007FE8D481AF0C3FA0221B3
:109660008B481AF0A3F900231A22582188481BF0CE
:109670001DFD8C498648F7F739F927270026089AF7
:109680009AF800301278DFF814829A4240F2C580CE
:1096900000233AB216217E48834C1BF007FD98F850
:1096A0000030A82505FB03431B7D8BBB98F80010F9
:1096B00098F8003098F8002005FB014105FB0343B2
:1096C000D2B20792D1E91601D3E9122323F00AFDA1
:1096D0000022764B23F0E4FF80463046894623F093
:1096E0004FFE02460B464046494623F0AFFE079B1D
:1096F00005FB0344D4E9122323F0F6FC24F09EF981
:1097000024F0D6FC6A4902B21AA825F03FF880E09E
:1097100098F8003098F8001005FB034305FB014161
:109720001B7D012B98F8003098F8002005FB0343BF
:10973000D2B20792D1E91601D3E9122333D123F033
:10974000D1FC0022594B23F0ABFF804630468946BE
:1097500023F016FE02460B464046494623F076FEAD
:10976000079B05FB0344D4E9122323F0BDFC24F03E
:1097700065F90021054624F05DFC10B105F10040BB
:1097800000E028464B4924F0B7FA24F091FC0A2364
:1097900090FBF3F404FB1304284624F089FC2346D1
:1097A00002B2454932E023F09DFC00223F4B23F0FA
:1097B00077FF80463046894623F0E2FD02460B469D
:1097C0004046494623F042FE079B05FB0344D4E98B
:1097D000122323F089FC24F031F90021054624F0FE
:1097E00029FC10B105F1004000E02846334924F07F
:1097F00083FA24F05DFC642390FBF3F404FB130470
:10980000284624F055FC2E49234602B21AA824F01B
:10981000BDFF1AA91E48F7F769F8013618370B2E55
:10982000BFB27FF42CAF032119481AF0BFF846F2FB
:109830002C3117481AF067F900234D2217211448DC
:109840001BF034FC64211248F7F758F80023622219
:109850001A210F481BF02AFC50210D48F7F74EF84B
:109860000023A4221A210A481BF020FC14210848D6
:10987000F7F744F80023BA22202105481BF016FC14
:1098800000210348F7F73AF825E000BF1CB9FF1F95
:109890005CC6FF1FB83603006627030029C4FF1FFC
:1098A0002AC4FF1F72270300F88EFF1F0000244008
:1098B0006355030000002041792703000000C842DF
:1098C00082270300752300930194F8234D2227215A
:1098D0009A481CF09BFA502441F2A20522B2163499
:1098E0000095F1232A219548A4B21CF0F1FBD42C59
:1098F000F4D12A2441F2A20521B2183400956D2337
:1099000051228E48A4B21CF085FBB4F5997FF3D1A7
:109910008B4D2E46502716F8010B0097BE2364226C
:109920000021F6F746FF2A241FFA80F916F8010BEA
:109930000097BE2364220021F6F73BFF80B24F2838
:1099400003DDBE28A8BFBE2000E0502021B218349D
:10995000A4B21FFA80FA4FF4784800B20090CDF814
:10996000048023B20FFA89F274481AF059FBB4F557
:109970008D7F01D0D146D9E7ABF16503DBB2992BDE
:1099800000F2FA806F4B0BF13807FFB21B787A1E9A
:109990009A4216D00FB9FF2B13D09F4217D06A4AB4
:1099A0001278974201D1FF2B11D0791C8B4213D032
:1099B000974200D183B1013A974213D1FF2B11D1C5
:1099C0000AE044F2082426464FF4FC690EE044F213
:1099D00008244FF4FC6608E044F208264FF4FC64C7
:1099E000B14603E044F208242646A146DFF884810C
:1099F000B8F80020192005230025303A8DE8290009
:109A000012B2DB234F214D481CF058FA4FF0030CE3
:109A10004FF0000E94238DE808503C2218234FF499
:109A2000937146481CF04AFAB8F800A0464B1AADAC
:109A30000BF137011B780822C9B22846AAF1300A77
:109A400011F020FA1FFA8AFACDF808904FF01A099F
:109A5000524633234F213D480195CDF8009011F037
:109A600061F8284620F0FFFBB8F800A0364BAAF1B9
:109A7000300A1B780822394628461FFA8AFA11F064
:109A800001FA332352468721029631480195CDF8D9
:109A9000009011F047F8284620F0E5FBB8F8006088
:109AA000294B303E0BF139011B780822C9B22846F8
:109AB000B6B211F0E7F933233246BF2102942548AC
:109AC0000195CDF8009011F02DF8284620F0CBFB41
:109AD000B8F800402049303C284620F004FCA4B2ED
:109AE00000232246172102931C4801953323CDF809
:109AF000009011F017F8284620F0B5FBB8F80040A8
:109B00001749303C284620F0EEFBA4B20023224641
:109B1000F7210293134801953323CDF8009011F0FB
:109B200001F8284620F09FFB0F4810F08BFE0F48ED
:109B300010F088FE0E4800F0BCBD00BF5CC6FF1FE1
:109B400084C5FF1FE88EFF1F2AC4FF1F80B9FF1FB7
:109B500094B9FF1FA8B9FF1FA9200300BCB9FF1FBC
:109B6000AB200300D0B9FF1F1CB9FF1F30B9FF1F86
:109B700044B9FF1F4488FF1FBBF1C70F02F24D809D
:109B8000502315F80B0000936422BE230021F6F742
:109B900010FE0BEB4B01C90002B203232A31C0486F
:109BA000CDF800801AF034FF1521032335228DE80B
:109BB0000A00BB48CDF808802A23F9211CF07EF961
:109BC0004FF6FF71B64819F09EFFB649B44819F038
:109BD000EFFF00234A22FA21B1481BF067FA15F87B
:109BE0000B10AF481AACF6F785FEAD4819F0FAFF36
:109BF0000025AD492426204620F075FB18233C2281
:109C00004FF49371A94802950194009610F08AFFD1
:109C1000204620F028FBA649204620F064FB1823AC
:109C2000AC224FF49371A34802950194009610F072
:109C300079FF204620F017FB9F49204620F053FB78
:109C4000442364224FF4937100939C480295182397
:109C5000019410F067FF204620F005FB984810F0B3
:109C6000F1FD984810F0EEFD974810F0EBFD974895
:109C700010F0E8FD964800F01CBD152840F08882E1
:109C8000FF294FF0000440F06781884D28191434F3
:109C900010F0D8FDB4F5027FF8D1AC240A250026D7
:109CA00040F22B13302214217D488DE870001CF007
:109CB00005F94CF2186330220293142140F22B1361
:109CC00077488DE830001AF00DFF4FF6FF717448A9
:109CD00019F019FF0121724819F00FFF71497048FE
:109CE00019F066FF33464A2219216D481BF0DEF950
:109CF000784916A820F0F7FA774B1A78032A9A4683
:109D000017D176496648F6F7F1FD754B75491B7812
:109D1000097832461AA811F0B5F81AA9604820F05F
:109D20005DF91AA820F09FFA6F4916A820F058FB99
:109D300003E06E495A48F6F7D9FD594819F052FF29
:109D40000221574819F032FE00231A2253215448A9
:109D50001BF0ACF916A9524820F040F9272500273E
:109D60002AB2002316214E48614E1BF09FF90120B4
:109D7000F6F76BFDA82404FB006000225D4BD0E9E0
:109D8000160123F08DFC80463846894623F0F8FA08
:109D900002460B464046494623F058FB23F02EFE70
:109DA000013781B23E48F6F7A9FD18350B2FADB249
:109DB000D6D103213A4819F0F9FD46F22C31384842
:109DC00019F0A1FE9AF80030032B4FF04D024FF02E
:109DD000000340F09780434F31481A211BF066F989
:109DE0003B782F48012504FB03630095D3E9162334
:109DF000F6F78AFD002362221A2129481BF056F942
:109E0000397804FB0161D1E91289D1E91601424692
:109E10004B4623F067F90022374B23F017FB002253
:109E2000364B23F03DFC42464B4623F05DF900954E
:109E300002460B461A48F6F767FD0023A4221A21B2
:109E400017481BF033F9397804FB0161D1E9128915
:109E5000D1E9160142464B4623F044F90022284B33
:109E600023F0F4FA0022254B23F01AFC42464B461D
:109E700023F03AF9009502460B460948F6F744FDEF
:109E80000023BA221A2106481BF010F93B780095EE
:109E900004FB0364D4E912230148F6F735FD57E0CB
:109EA0005CC6FF1FB8360300252503001CB9FF1F41
:109EB0002825030030B9FF1F8B27030044B9FF1F7B
:109EC00080B9FF1F94B9FF1FA8B9FF1FBCB9FF1FBE
:109ED000D0B9FF1F8E2703006CC5FF1F9827030012
:109EE0002AC4FF1FFE87FF1FE4260300A6270300E6
:109EF000F88EFF1F0000244000005440000059402D
:109F000000003440172196481BF0D0F86421944893
:109F1000F6F7F4FC002362221A2191481BF0C6F8E0
:109F200050218F48F6F7EAFC0023A4221A218C481E
:109F30001BF0BCF814218A48F6F7E0FC2021884881
:109F40000023BA221BF0B2F800218548F6F7D6FCB0
:109F500016A820F088F908E0752300930194F823EF
:109F60004D2227217E481BF051FF502441F2A205CB
:109F700022B216340095F1232A217948A4B21CF0AC
:109F8000A7F8D42CF4D12A2441F2A20521B2183426
:109F900000956D2351227248A4B21CF03BF8B4F531
:109FA000997FF3D16F4B704D1A7807932E46032A91
:109FB00016F8012B6FF06C0714BF4FF065094FF4D2
:109FC00080797A4392FBF9F2BE3292B22A2416F8D3
:109FD000013B7B4393FBF9F3BE339BB24F2B03DD75
:109FE000BE2BA8BFBE2300E0502321B21834A4B278
:109FF0001FFA83FA4FF478481BB20093CDF804801F
:10A0000023B212B256481AF00BF8B4F58D7F01D086
:10A010005246DCE7BBF1FF0F01F0FF8515F80B207E
:10A020004F48CDF800806FF06C030BEB4B015A43A7
:10A03000C90092FBF9F2BE32032312B22A311AF0A0
:10A04000E7FC152203238DE80C00EF213423352291
:10A050004348CDF808801BF031FF4FF6FF714048B0
:10A0600019F051FD41493E4819F0A2FD00234A2252
:10A07000F0213B481BF01AF8079B15F80B401B78A2
:10A08000032B29D13A4B3B4A1B78A82101FB032122
:10A09000D1E91267D1E9160132463B4623F022F896
:10A0A00080462046894623F05BF902460B4640462F
:10A0B000494623F0CBF928A3D3E9002323F0F0FA93
:10A0C00032463B4623F010F80223009302460B462B
:10A0D0002348F6F719FC03E021462148F6F70AFC6D
:10A0E0001AAC1F4819F07EFD00252349242620467E
:10A0F00020F0F9F818233C224FF493711F48029581
:10A100000194009610F00EFD204620F0ACF81C499A
:10A11000204620F0E8F81823AC224FF49371194838
:10A1200002950194009610F0FDFC204620F09BF86B
:10A130001549204620F0D7F844231448009302958F
:10A140000194182364224FF4937110F0EBFC01F09A
:10A15000B9BB00BFAFF300800000000000E06F401B
:10A160005CC6FF1F6CC5FF1FBDC4FF1FB8360300D0
:10A17000FE87FF1FF88EFF1F252503001CB9FF1F58
:10A180002825030030B9FF1F8B27030044B9FF1FA8
:10A19000172840F0E480A04D00242819143410F052
:10A1A00051FBB4F5027FF8D10026AC240A258DE8D6
:10A1B000700040F22B13302214219848DFF8B4824B
:10A1C0001BF07CFE4CF2186330228DE830000293C5
:10A1D000142140F22B1391481AF084FC4FF6FF71C2
:10A1E0008E4819F090FC01218C4819F086FC8C49AE
:10A1F0008A4819F0DDFC33464A22192187481AF0B3
:10A2000055FF88498548F6F771FB844819F0EAFC48
:10A210003346BE22192181481AF048FF82497F48FF
:10A22000F6F764FB3346CB2219217C481AAC1AF0AE
:10A230003DFF7E49794816ADF6F758FB7C4920462C
:10A2400020F051F8282798F80010284620F06BF8E5
:10A250003C234D22192170480396029501940097E2
:10A2600010F005FD28461FF0FEFF20461FF0FBFF03
:10A270007049204620F037F898F80110284620F061
:10A2800052F83C234D2269216B48039602950194B4
:10A29000009710F0ECFC28461FF0E5FF20461FF069
:10A2A000E2FF6649204620F01EF898F80210284682
:10A2B00020F039F83C234D22B921614803960295DC
:10A2C0000194009710F0D3FC28461FF0CCFF2046E5
:10A2D0001FF0C9FF5B49204620F005F898F80310ED
:10A2E000284620F020F83C237F2219215648039667
:10A2F00002950194009710F0BAFC28461FF0B3FFB6
:10A3000020461FF0B0FF514920461FF0ECFF98F89F
:10A310000410284620F007F83C237F2269214C488E
:10A32000039602950194009710F0A1FC28461FF0B7
:10A330009AFF20461FF097FF464920461FF0D3FFA3
:10A3400098F8051028461FF0EEFF03960295019439
:10A3500000973C237F22B9213F4800F008BF0E2818
:10A3600040F0EE820026FF293C4FDFF80C91019669
:10A370001AAD40F0A2813B8828480D3B1BB20D224C
:10A380003146009323B21BF041FD4FF6FF71234885
:10A3900019F0B9FB0121214819F0AFFB20491F48F2
:10A3A00019F006FC3346242205211C481AF07EFED3
:10A3B0002B491A48F6F79AFA16AC184819F012FC0D
:10A3C000284920461FF08FFF254928461FF08BFFA4
:10A3D00028232D22502103960093234802953C23E5
:10A3E000019410F044FC28461FF03DFF20461FF06A
:10A3F0003AFF40F2AB10F6F728FA1C4B1C4E1870CF
:10A4000019781A46002901F075833378022B41F040
:10A41000C18301F06FBB00BF1CB9FF1F5CC6FF1FEB
:10A42000B8360300B9270300CA270300F727030043
:10A43000122803001828030030B9FF1F1E2803004C
:10A4400044B9FF1F2428030058B9FF1F2A2803001E
:10A450006CB9FF1F3028030080B9FF1F4488FF1F1D
:10A4600009250300F7260300E4B9FF1FF18EFF1F43
:10A47000AFC7FF1F2CD5FF1F2AC4FF1F1F78FFB2D5
:10A48000052F41F0A283A84928461FF02CFF4FF466
:10A49000FC6302932823009301953C232D22394627
:10A4A000A24810F03FFB28461FF0DDFE4FF00008E9
:10A4B00028279F4928461FF016FF3C235F220521CD
:10A4C0009C48CDF808800195009710F02BFB28469A
:10A4D0001FF0C9FE984928461FF005FF3C235F2264
:10A4E00050219648CDF808800195009710F01AFB8E
:10A4F00028461FF0B8FE924928461FF0F4FE3C2380
:10A50000912205218F48CDF808800195009710F021
:10A5100009FB28461FF0A7FE8B4928461FF0E3FEE3
:10A520003C23502191228948CDF80880019500975D
:10A5300010F0F8FA28461FF096FE337884497D4ED5
:10A54000022B204641F0F1821FF0CDFE81492846C2
:10A550001FF0C9FE4CF21863C3220521039306F1D4
:10A56000F0003C2302950194009710F080FB2846F0
:10A570001FF079FE20461FF076FE774B1B78002BEC
:10A5800041F0E982754920461FF0ADFE7449284626
:10A590001FF0A9FE4CF2186303932823C322502115
:10A5A000019400936F4802953C2310F060FB28460D
:10A5B0001FF059FE20466C4C1FF055FE99F80030F4
:10A5C00021780922284610F05DFC05237A220093A9
:10A5D00023212B46654810F0BBFF28461FF043FEA1
:10A5E000227899F800309A4219D2F28BB18B6048E8
:10A5F0001B32193112B2002309B21AF057FD5D4B1C
:10A60000186822F0CFFE22785B4BA82707FB0233A5
:10A6100002461B7D009356480B46F6F775F999F8EC
:10A62000003061780922284610F02CFC0523AC226A
:10A63000009323212B464D4810F08AFF28461FF037
:10A6400012FE627899F800309A421CD2B6F8462081
:10A65000B6F8441046481B32193112B2002309B231
:10A660001AF024FD434B586822F09CFE3E4B5A786A
:10A67000414BA82404FB023302461B7D00933C4857
:10A680000B46F6F741F96420FAF710FC3B4B3C48C7
:10A6900001221A7010F0D6F83A4810F0D3F83A4870
:10A6A00010F0D0F8394810F0CDF8394810F0CAF859
:10A6B000384810F0C7F801F0B0BA28230093C3223D
:10A6C0009A2305212A481BF0A1FB334B1A78334B00
:10A6D0001B78511E994215D00AB9FF2B12D09A420D
:10A6E00016D099F800108A4201D1FF2B10D0501CCF
:10A6F000834212D08A4200D17BB1884250D1FF2BD5
:10A700004ED10AE044F2082426464FF4FC684BE0A0
:10A7100044F208244FF4FC6645E044F208264FF466
:10A72000FC64B04640E000BF4C2803006CB9FF1F3A
:10A730006A2803001CB9FF1F7328030030B9FF1FEC
:10A740007B28030044B9FF1F8528030058B9FF1F69
:10A75000D2260300BD2D0300FAB8FF1F8E28030088
:10A760009628030020BAFF1F2888FF1FB8BCFF1FD0
:10A770005CC6FF1F98C5FF1FF88EFF1F4288FF1F92
:10A7800080B9FF1F94B9FF1FA8B9FF1FBCB9FF1FF5
:10A79000D0B9FF1FF8B9FF1FA0C5FF1FE88EFF1F2C
:10A7A00044F208242646A046B7F800A08D49284662
:10A7B000AAF11A0A1FF097FD1FFA8AFACDF808804D
:10A7C0004FF01A085246332337210195CDF8008007
:10A7D0008548DFF85CA210F0A5F928461FF043FD7C
:10A7E0003A888248113A002312B239211AF05EFCED
:10A7F0009AF8001099F80030013908222846C9B2A9
:10A8000010F040FB294679481FF0E8FB28461FF06E
:10A810002AFDB7F800B07349ABF11A0B1FFA8BFB96
:10A8200028461FF060FD5A46029633237021019599
:10A83000CDF800806E4810F075F928461FF013FD22
:10A840003A886A48113A002312B273211AF02EFC9A
:10A8500099F800309AF800100822284610F012FBF0
:10A86000294662481FF0BAFB28461FF0FCFC3E88D0
:10A870005C491A3EB6B228461FF035FD32460294B6
:10A880003323A9210195CDF800805A4810F04AF9E8
:10A8900028461FF0E8FC3A885448113A002312B2C7
:10A8A000AC211AF003FC9AF8001099F8003001313D
:10A8B00008222846C9B210F0E5FA29464B481FF095
:10A8C0008DFB28461FF0CFFC3C884B491A3C0026E4
:10A8D000A4B228461FF007FD2246332331460296D4
:10A8E0000195CDF80080454810F01CF928461FF06E
:10A8F000BAFC3C8842491A3CA4B228461FF0F3FC3B
:10A9000022463323E22102960195CDF800803D488E
:10A9100010F008F928461FF0A6FC3C883A491A3C7A
:10A92000A4B228461FF0DFFC02960195CDF8008006
:10A93000272322464FF48C71344810F0F3F81BE1C2
:10A94000102840F0EF81FD2940F21981FF2926D11E
:10A9500000252F4B01951B8824480D3B1BB20D226F
:10A960000093294623B21BF051FA4FF6FF711F489E
:10A9700019F0C9F801211D4819F0BFF825491B48F5
:10A9800019F016F92B462422052118481AF08EFBDF
:10A9900021491648F5F7AAFF144819F023F940F2A7
:10A9A0001B10F5F752FF1AAC0A2843D8DFE800F075
:10A9B000060D0F11424242424242130017492046FF
:10A9C0001FF091FC46F22C333AE0154904E015499A
:10A9D00002E0154900E0154920461FF084FC4FF4C1
:10A9E000FC632DE04D26030080B9FF1F5CC6FF1FEE
:10A9F00094B9FF1FA8B9FF1FA9200300BCB9FF1F0E
:10AA0000AB200300D0B9FF1F92230300F8B9FF1F4A
:10AA10004488FF1FB8360300D92403008A280300A6
:10AA2000E2240300E7240300ED24030001250300D2
:10AA3000A0C5FF1FA44920461FF055FC4FF6E07348
:10AA4000029328232D2205210093A04801943C2342
:10AA500016AD10F067F820461FF005FC9C4928460B
:10AA60001FF041FC002728269A4920461FF03BFC96
:10AA70003C235F2205219848039702940195009694
:10AA800010F0F5F820461FF0EEFB28461FF0EBFB18
:10AA9000924928461FF027FC914920461FF023FCCD
:10AAA0003C23912205218F4803970294019500963B
:10AAB00010F0DDF820461FF0D6FB28461FF0D3FB30
:10AAC000894928461FF00FFC854920461FF00BFCE2
:10AAD00005213C23C32285480397029401950096E3
:10AAE00010F0C5F820461FF0BEFB28461FF0BBFB48
:10AAF0004FF4D770F5F7A9FE7D4948B928461FF0F5
:10AB0000F2FB7C4920461FF0EEFB46F22C3308E0B6
:10AB100028461FF0E8FB774920461FF0E4FB4FF47E
:10AB2000FC63C32264210393734802943C23019580
:10AB3000009610F09CF820461FF095FB28461FF069
:10AB400092FB6E4928461FF0CEFB4FF48A70F5F752
:10AB50007CFE014620461FF0E6FB002303932823DA
:10AB600000936748029401953C23C3229B2110F077
:10AB70007EF820461FF077FB284600F0A4BE00298F
:10AB800044D1604B0A4643F82B200BF1010BBBF17B
:10AB9000080F4FF00004F6D1C823272250215A484D
:10ABA00000930194DC231BF031F9F9F7DBFF234616
:10ABB00028228C2154481AF079FA54495248F5F762
:10ABC00095FE234632228C214F481AF06FFA5049E5
:10ABD0004D48F5F78BFE3E4916A81FF084FB3D4912
:10ABE0001AA81FF080FB1F231AAA16A93A480FF0D3
:10ABF000F5FE1AA81FF037FB16A81FF034FB454BD3
:10AC000014221A70444B1C7001F007B801292DD191
:10AC100000233C4A194642F823100133082B4FF019
:10AC20000004F8D1C823272250213748009301940B
:10AC3000DC231BF0EBF8F9F795FF284916A81FF065
:10AC400052FB27491AA81FF04EFB23461AAA16A941
:10AC500024480FF0C3FE1AA81FF005FB16A81FF02A
:10AC600002FB284B02221A6100F0D7BF022940F0F4
:10AC7000D487244B244819610024C823272250215B
:10AC80008DE81800DC231BF0C1F8F9F76BFF1649BB
:10AC900016A81FF028FB12491AA81FF024FB234610
:10ACA0001AAA16A911480FF099FE1AA81FF0DBFA8C
:10ACB00016A81FF0D8FA194B1B681A93184B1A9A4A
:10ACC0001A6000F0AABF00BFAB2103001CB9FF1F30
:10ACD0009B280300903F030030B9FF1FA02803000A
:10ACE000A528030044B9FF1FA928030058B9FF1F76
:10ACF000E2240300AF2803006CB9FF1FB52803004E
:10AD000080B9FF1F1CC6FF1F5CC6FF1FBD280300C4
:10AD1000D5280300EAC6FF1F0188FF1F58D8FF1F70
:10AD2000E48EFF1F112840F043824FF00008B54B1E
:10AD3000CDF804801B88B4480D3B1BB20D22009354
:10AD4000414623B21BF062F84FF6FF71AE4818F08F
:10AD5000DAFE0121AC4818F0D0FEAC49AA4818F040
:10AD600027FF434624220521A7481AF09FF9A84946
:10AD7000A548F5F7BBFD16ADA34818F033FFA5496C
:10AD800028461FF0B0FA4FF48E70F5F75EFD1AAC4E
:10AD90000146282720461FF0C6FA50213C233A4698
:10ADA0009D48CDF80C800294019500970FF05FFF4D
:10ADB00020461FF058FA28461FF055FA4FF4D67077
:10ADC000F5F743FD12AE01289449304620D11FF01B
:10ADD0008AFA934928461FF086FA924920461FF0C6
:10ADE00082FA4FF4FC633A469B21049303943C237C
:10ADF0000295019600978C480FF0D4FE20461FF074
:10AE000032FA28461FF02FFA30461FF02CFA24E0C1
:10AE10001FF069FA824928461FF065FA81492046E9
:10AE20001FF061FA46F22C339B213A4604937E4888
:10AE300003943C230295019600970FF0B3FE204641
:10AE40001FF011FA28461FF00EFA30461FF00BFAD9
:10AE500041464FF4D670F5F78BFC40F2AD10F5F794
:10AE6000F4FC724928B120461FF03DFA4FF4FC6310
:10AE700004E020461FF037FA46F22C3328220092D5
:10AE8000052102936A4801943C230FF04BFE2046B3
:10AE90001FF0E9F9674920461FF025FA664B28277D
:10AEA00019784CF2186828461FF03DFA3C233A46C0
:10AEB000EB216248CDF80C800295019400970FF0C9
:10AEC000D6FE28461FF0CFF920461FF0CCF95C498A
:10AED00020461FF008FA4FF4D270F5F7B6FC014691
:10AEE00028461FF020FA3C235F2205215548CDF863
:10AEF0000C800295019400970FF0B9FE28461FF0D0
:10AF0000B2F920461FF0AFF94F4920461FF0EBF988
:10AF1000002350215F2202934C4801943C23009768
:10AF20000FF000FE20461FF09EF940F2AF10F5F73B
:10AF30008CFC4749C8B930461FF0D5F94549284629
:10AF40001FF0D1F9444920461FF0CDF946F22C33C9
:10AF50000493424803940295019600973C235F2294
:10AF60009B210FF01FFE20462EE030461FF0BBF95C
:10AF7000384928461FF0B7F940F2AF10F5F765FCE5
:10AF800001460AA81FF0CFF90AA90EA81FF015FA6A
:10AF900033490EA81FF0C2FA014620461FF00DFAF1
:10AFA0004FF4FC635F229B2104932C4803943C23C1
:10AFB0000295019600970FF0F5FD20461FF053F91A
:10AFC0000EA81FF050F90AA81FF04DF928461FF0EF
:10AFD0004AF930461FF047F940F21D10F5F735FCED
:10AFE00001282049304643D11FF07DF91E492846EB
:10AFF0001FF079F91D4920461FF075F94FF4FC63E5
:10B0000042E000BF4488FF1F5CC6FF1FB836030044
:10B01000EE280300FD28030030B9FF1F9D24030024
:10B02000062903008724030058B9FF1F0F290300D6
:10B0300080B9FF1F17290300FF87FF1F6CB9FF1F8F
:10B040001F29030094B9FF1F28290300A8B9FF1F77
:10B050002E290300352903008A280300BCB9FF1FED
:10B06000E52503003C29030041290300782803005B
:10B070001FF039F9414928461FF035F9404920466B
:10B080001FF031F946F22C33049328235F22EB2181
:10B0900000933C4803943C23029501960FF082FDF7
:10B0A00020461FF0E0F828461FF0DDF830461FF07C
:10B0B000DAF8354B354F1B78F3B9354928461FF080
:10B0C00012F9344920461FF00EF939880A22304619
:10B0D0001FF03CF946F22C33049328230093039687
:10B0E000029401953C23962205212B480FF05AFD2E
:10B0F00030461FF0B8F81FE03B882549284643B189
:10B100001FF0F1F8254920461FF0EDF84FF4784381
:10B1100007E01FF0E8F8224920461FF0E4F84FF45A
:10B12000FC63039328230093029401953C23962209
:10B13000052119480FF09BFD20461FF094F8284682
:10B140001FF091F8174920461FF0CDF8164B1978DB
:10B150000A22013128461FF0F9F80023039313480F
:10B1600002952823009301943C23962250210FF04E
:10B170007EFD28461FF077F8A4E300BF41290300B5
:10B180008A280300D0B9FF1F6CC5FF1FCA8EFF1F9E
:10B190001025030046290300E4B9FF1F4C290300D2
:10B1A000532903005C290300E5C7FF1FF8B9FF1FFF
:10B1B000122840F032850027B54B01971B88B5480F
:10B1C0000D3B1BB20D223946009323B21AF01EFE2E
:10B1D0004FF6FF71AF4818F096FC0121AD4818F00A
:10B1E0008CFCAD49AB4818F0E3FC3B46242205211A
:10B1F000A84819F05BFFA949A648F5F777FBA548D1
:10B2000018F0F0FC4FF4D970F5F75BFB16AD82B285
:10B21000A34912A81AAC23F0B9FAA2492846282655
:10B220001FF061F812A920461FF05DF83C232D2283
:10B23000052103979C480294019500960FF017FD95
:10B2400020461FF010F828461FF00DF84FF4DA7072
:10B25000F5F737FB924982B212A823F097FA934987
:10B2600028461FF040F812A920461FF03CF83C2366
:10B270002D22502103978E480294019500960FF0DD
:10B28000F6FC20461EF0EFFF28461EF0ECFF4FF4C0
:10B29000DB70F5F716FB824982B212A823F076FA2A
:10B2A000844928461FF01FF812A920461FF01BF8FA
:10B2B0003C232D229B2103977F4802940195009601
:10B2C0000FF0D5FC20461EF0CEFF28461EF0CBFF27
:10B2D0004FF4DC70F5F7F5FA714982B212A823F049
:10B2E00055FA764928461EF0FEFF12A920461EF0A8
:10B2F000FAFF3C232D22E621039771480294019521
:10B3000000960FF0B4FC20461EF0ADFF28461EF05C
:10B31000AAFF4FF4DD70F5F7D4FA614982B212A8A2
:10B3200023F034FA674928461EF0DDFF12A92046B3
:10B330001EF0D9FF3C235F22052103976248029447
:10B34000019500960FF093FC20461EF08CFF2846D6
:10B350001EF089FF4FF4DE70F5F7B3FA504982B260
:10B3600012A823F013FA594928461EF0BCFF12A96F
:10B3700020461EF0B8FF3C235F225021039754481B
:10B380000294019500960FF072FC20461EF06BFFB0
:10B3900028461EF068FF4FF4DF70F5F792FA404937
:10B3A00082B212A823F0F2F94A4928461EF09BFF08
:10B3B00012A920461EF097FF3C235F229B21039792
:10B3C00045480294019500960FF051FC20461EF06E
:10B3D0004AFF28461EF047FF4FF4E070F5F771FA78
:10B3E0002F4982B212A823F0D1F93C4928461EF019
:10B3F0007AFF12A920461EF076FF3C235F22E62149
:10B40000039737480294019500960FF030FC2046D0
:10B410001EF029FF28461EF026FF4FF4D870F5F7DE
:10B4200050FAB8424FF4D870C8BF4FF4FC67F5F734
:10B4300048FA1B4982B212A823F0A8F929492846E4
:10B440001EF051FF12A920461EF04DFF05213C239E
:10B450009122254803970294019500960FF007FC6E
:10B4600020461EF000FF28461EF0FDFE4FF4E2705D
:10B47000F5F7EBF901281D4928463BD11EF033FFB3
:10B480001B4920461EF02FFF4FF4FC633AE000BF3B
:10B490004488FF1F5CC6FF1FB83603006429030001
:10B4A0006F290300762903001CB9FF1F7E290300C2
:10B4B00030B9FF1F8629030044B9FF1F8E290300FE
:10B4C00058B9FF1F962903006CB9FF1F9E2903007E
:10B4D00080B9FF1FA629030094B9FF1FAE290300FE
:10B4E000A8B9FF1FB6290300BCB9FF1FBB29030081
:10B4F000C92C03001EF0F7FE684920461EF0F3FE3B
:10B5000046F22C3391225021039300963C2302945F
:10B51000019563480FF0ABFB20461EF0A4FE2846C1
:10B520001EF0A1FE5F4928461EF0DDFE00262827FA
:10B530005D4920461EF0D7FE3C23BE22052103961E
:10B5400002940195009759480FF091FB20461EF098
:10B550008AFE28461EF087FE554920461EF0C3FE8F
:10B560003C23BE22502102960194009751480FF0CF
:10B57000D9FA20461EF077FE4F4920461EF0B3FE52
:10B580003C23BE229B210296019400974B480FF06A
:10B59000C9FA20461EF067FE494928461EF0A3FE60
:10B5A000484920461EF09FFE3C23BE22E62103961A
:10B5B00002940195009744480FF059FB20461EF075
:10B5C00052FE28461EF04FFE4CF218613F4818F01C
:10B5D0009AFA3346E7220A213C4819F067FD3C49B4
:10B5E0003A48F5F783F918E32B78052B07D1394B47
:10B5F000002019780FF01EFC002840F056812B78AF
:10B60000062B04D02B78072B40F0518108E0314BFA
:10B61000012019780FF00EFC002840F04681F1E778
:10B620002C4B032019780FF005FC002840F03D81D9
:10B630003DE11A780A2A59D1274920461EF053FEC7
:10B64000002221461D480FF093F920461EF00BFE04
:10B65000224920461EF047FE46F22C3302931A235D
:10B660004946019400938322642317480FF05AFA45
:10B6700020461EF0F8FD1A4A00231370194A137071
:10B68000194B14201C681FF006F80546F5F7C0F9A1
:10B690002946204617F094FABFE200BF2526030092
:10B6A000F8B9FF1FC4290300CB2903000CBAFF1F00
:10B6B000CF29030020BAFF1FD5290300D0B9FF1FEF
:10B6C000A9280300E0290300E4B9FF1F5CC6FF1F9F
:10B6D000E4290300A0C5FF1F9425030027210300D0
:10B6E000D4C5FF1FCEC5FF1FA4D7FF1F1E78F6B21B
:10B6F000082E40F0D4808F4D8F49B5F80080DFF8D8
:10B700007CB2DFF88492A8F11A0820461EF0EBFD07
:10B710001A271FFA88F844F2082342461921029397
:10B7200086480194332300970FF0FCF920461EF061
:10B730009AFD2A888248DFF85482113A002312B217
:10B740001B2119F0B3FC9BF800304FF0A80A0AFB4C
:10B750000393324693F8911098F800300139C9B23A
:10B7600020460FF08FFB214675481EF037FC20461F
:10B770001EF079FD2A8870491A3A92B22046079243
:10B780001EF0B1FD4FF4FC63079A0293522133235C
:10B790006C48019400970FF0C5F920461EF063FD38
:10B7A0002A886748113A002312B2552119F07EFC0D
:10B7B0009BF8001098F800300AFB0191324691F88E
:10B7C000911020460FF05EFB21465D481EF006FCFE
:10B7D00020461EF048FD2A8857491A3A92B2204660
:10B7E00007921EF080FD44F20823079A02938B21F2
:10B7F00033235548019400970FF094F920461EF02A
:10B8000032FD2A884E48113A002312B28E2119F0D7
:10B810004DFC9BF800300AFB0399324699F89110D1
:10B8200098F800300131C9B220460FF02BFB2146B9
:10B8300043481EF0D3FB20461EF015FD2E884349D9
:10B840001A3E4FF00008B6B220461EF04CFD3246BC
:10B85000132341463E48CDF80880019400970FF02D
:10B8600061F920461EF0FFFC3A4B2D881E883A49AC
:10B870007D3E1A3DB6B2ADB220461EF034FD132314
:10B880002A4631463548CDF80880019400970FF0DC
:10B8900049F920461EF0E7FC3148FCF76EB81A78EB
:10B8A0003AB11B78022B11D103E02E4902E02E4958
:10B8B00000E02E4920461EF016FD002221462848B1
:10B8C0000FF056F820461EF0CEFCA6E1284920468F
:10B8D0001EF009FD0022214621480FF049F82046BC
:10B8E0001EF0C1FC2348F5F73DF8234B01221A70E6
:10B8F00093E1237808FB0373002103F80A10FDF796
:10B9000078BD1E4B93F800902378F35C09F1FF3269
:10B910009A4208D0B9F1000F3AD1194B194A1B7855
:10B92000D35CFF2B34D144F2082427464FF4FC6A41
:10B9300048E000BF4488FF1F4D26030094B9FF1F55
:10B940005CC6FF1F58B9FF1FA8B9FF1FA92003003D
:10B950006CB9FF1F0888FF1FAB20030080B9FF1FD1
:10B96000D0B9FF1FD5290300112A030022290300A3
:10B970008D250300E4B9FF1FD4C5FF1FA0C5FF1F1D
:10B98000EAC6FF1FD08EFF1FF88EFF1F2AC4FF1FBD
:10B990002378F35C4B4500F097802A78914500F0BE
:10B9A0008C802178715C09F101038B4200F09C804E
:10B9B000914500F08E80934200F0918044F208247B
:10B9C0002746A246B8F800B02B781AAE09F1FF312D
:10B9D00030460822C9B2ABF1180B0FF053FA1FFA28
:10B9E0008BFBCDF808A04FF0150A5A4633234A21A5
:10B9F0000196CDF800A08A480FF094F830461EF06A
:10BA000032FCB8F800B02B78ABF1180B4946304641
:10BA10001FFA8BFB08220FF035FA5A4602973323A0
:10BA200082210196CDF800A07E480FF07BF83046C9
:10BA30001EF019FCB8F800702B7809F10101183FCD
:10BA40003046BFB20822C9B20FF01CFA3A4633237F
:10BA50000294BA210196CDF800A073480FF062F865
:10BA600030461EF000FCB8F800407049183C002534
:10BA7000A4B230461EF037FC224633231121029532
:10BA80000196CDF800A06A480FF04CF830461EF041
:10BA9000EAFBB8F800406749183CA4B230461EF0F3
:10BAA00022FC02950196CDF800A033232246F22114
:10BAB00061480FF037F8FCF726BD604B60491B78F2
:10BAC000CB5CFF2B7FF46DAF44F208244FF4FC678E
:10BAD00077E75A495A480978415C29B16BE72378DE
:10BAE000F35CFF2B7FF46AAF44F208274FF4FC6449
:10BAF000BA4667E7534920461EF0F5FB52492846EF
:10BB00001EF0F1FB4CF218630393282300932D22BF
:10BB10003C2305214D48029501940FF0A8F82846D2
:10BB20001EF0A1FB2046FEF7BFBC032B09D11EF07F
:10BB3000DAFB474928461EF0D6FB40F2FF73FEF7BA
:10BB40000BBD1EF0D0FB434928461EF0CCFB4FF442
:10BB5000FC63FEF701BD022B0BD13F4920461EF0CE
:10BB6000C2FB3E4928461EF0BEFB4FF6E073FEF7CF
:10BB700013BD01214FF4D570F4F7FAFD3849204682
:10BB80001EF0B1FB334928461EF0ADFB4FF4FC63B9
:10BB9000FEF702BD1278334B012A06D132492846FE
:10BBA0001EF0A1FB4FF6E0732EE01A78022A01D1B5
:10BBB0002E491DE01A78032A01D12D4918E01A7880
:10BBC000042A7EF45BAC2B4912E01A78062A01D1D4
:10BBD00029490DE01A78072A01D1284908E01A7886
:10BBE000082A01D1264903E01B78092B06D12549F3
:10BBF00028461EF078FB4FF4FC6305E022492846F6
:10BC00001EF071FB4FF478430293282300930195B3
:10BC10003C232D220521FEF743BC1FB0BDE8F08F69
:10BC2000E4B9FF1FF8B9FF1F0CBAFF1FA9200300DA
:10BC300020BAFF1FAB20030034BAFF1FEAC6FF1F64
:10BC4000D08EFF1F8A280300532703006CB9FF1F03
:10BC50008F210300A92D030096280300C92C03009F
:10BC60008E280300F18EFF1F362803003B280300B7
:10BC700040280300472803005028030054280300ED
:10BC8000582803005C280300642803002DE9F04FC6
:10BC90008BB004ABB84E83E803003778BDF9104091
:10BCA000BDF91250AFB90DF11808B44940461EF065
:10BCB0001AFB23220F23009311468223B0480297D8
:10BCC000CDF804800EF02EFF40461EF0CCFAAD4BAE
:10BCD0001F700021AC4817F016FF0121AA4817F089
:10BCE0000CFF3178A84801EB4101490000232722CD
:10BCF000323119F0DBF9A54B1F7899462FB17B1C27
:10BD000089F800304FF0010801E04FF00A08A4B2B2
:10BD1000ADB201232A4621469D480EF09BFD38B363
:10BD20003378DFF854B2062B22D8DFF8B4A2994951
:10BD3000DAF8000022F07EF9D0B197499248F4F782
:10BD4000D5FD404621F084FFDAF8001021F0D4FF41
:10BD5000CAF80000384621F003FB02460B460020DB
:10BD60008E491EF07BFE02460B4600208C490AE2FB
:10BD700001232A4621468B480EF06CFD40B33378F0
:10BD8000DFF8F4B1062B23D8DFF854A28149DAF8A2
:10BD9000000022F04FF9D8B183497B48F4F7A6FDA3
:10BDA000404621F055FFDAF8001021F0A5FFCAF84F
:10BDB0000000384621F0D4FA02460B4600207749AD
:10BDC0001EF04CFE02460B4600204FF08041DAE1A7
:10BDD00001232A46214675480EF03CFD38B33378DE
:10BDE000DFF894B1062B22D8DFF8F4A16949DAF81C
:10BDF000000022F01FF9D0B16D496348F4F776FDD9
:10BE0000404621F025FFDAF8001021F075FFCAF84E
:10BE10000000384621F0A4FA02460B4600205F4994
:10BE20001EF01CFE02460B4600206249ABE10123D6
:10BE30002A46214660480EF00DFD38B33378DFF80E
:10BE400038B1062B22D8DFF898A15249DAF8000061
:10BE500022F0F0F8D0B159494B48F4F747FD40467D
:10BE600021F0F6FEDAF8001021F046FFCAF80000D3
:10BE7000384621F075FA02460B46002047491EF06D
:10BE8000EDFD02460B4600204D497CE101232A4688
:10BE900021464C480EF0DEFC38B33378DFF8D8B0DA
:10BEA000062B22D8DFF838A13A49DAF8000022F050
:10BEB000C1F8D0B144493448F4F718FD404621F0A8
:10BEC000C7FEDAF8001021F017FFCAF80000384664
:10BED00021F046FA02460B46002030491EF0BEFD16
:10BEE00002460B46002039494DE101232A462146EE
:10BEF00037480EF0AFFC68B13378DFF87CB0062B22
:10BF000008D8DFF8DCA02349DAF8000022F092F824
:10BF1000002867D101232A4621462E480EF09AFCBC
:10BF200000287AD03378DFF850B0062B75D8DFF8C8
:10BF3000B0A01849DAF8000022F07CF800286CD094
:10BF400025491148F4F7D2FC404621F081FEDAF889
:10BF5000001021F0D1FECAF80000384621F000FAA6
:10BF600002460B4600200D491EF078FD02460B46A6
:10BF700000201A4907E100BF0088FF1F27210300A6
:10BF800058B9FF1FE08EFF1F5CC6FF1F0188FF1F0F
:10BF9000E4B9FF1F003C1C4670260300000024404B
:10BFA0000000F03FF8B9FF1F242303000CBAFF1F65
:10BFB000782603000000084020BAFF1F7C260300FB
:10BFC0000000104034BAFF1F592A0300000014403B
:10BFD00048BAFF1F5CBAFF1FFF24030000001C408B
:10BFE000D0C5FF1FB949BA48F4F780FC404621F09C
:10BFF0002FFEDAF8001021F07FFECAF80000384664
:10C0000021F0AEF902460B460020B2491EF026FD93
:10C0100002460B460020B049B5E001232A462146DE
:10C02000AE480EF017FC38B33378DFF8FCB2062BBD
:10C0300022D8DFF8D8A2AA49DAF8000021F0FAFFE6
:10C04000D0B1A849A248F4F751FC404621F000FEC7
:10C05000DAF8001021F050FECAF80000384621F04E
:10C060007FF902460B4600209A491EF0F7FC024673
:10C070000B4600209C4986E001232A4621469B4826
:10C080000EF0E8FB38B33378DFF89CB2062B22D8E9
:10C09000DFF878A29249DAF8000021F0CBFFD0B1A6
:10C0A00093498B48F4F722FC404621F0D1FDDAF8A1
:10C0B000001021F021FECAF80000384621F050F9A6
:10C0C00002460B46002083491EF0C8FC02460B4680
:10C0D0000020884957E001232A46214686480EF071
:10C0E000B9FB78B199F80030844C43B98449784859
:10C0F000F4F7FCFB337801333370012300E0013B9C
:10C10000237063E37F4801232A46214600F5C87067
:10C110000EF0A0FB60B13378DFF80CB2062B07D825
:10C12000DFF8E8A16E49DAF8000021F083FF80B95A
:10C1300001232A46214674480EF08CFB00283AD091
:10C14000724B0021186821F06BFF074600283FD092
:10C1500031E06F495E48F4F7C9FB404621F078FDB5
:10C16000DAF8001021F0C8FDCAF80000384621F0C6
:10C17000F7F802460B46002056491EF06FFC0246B7
:10C180000B460020002121F08BFA0446DAF800006B
:10C190000D4621F007F90B4602462946204620F0BD
:10C1A000A3FF21F04BFC9BF80030CAF800000133DC
:10C1B0008BF800300AE301232A46214655480EF049
:10C1C00049FB002841D0544F3B780C2B4CD93CE024
:10C1D000524C237883F00103237027220346282141
:10C1E0003B4818F063FF257806AC4DB14C49384800
:10C1F000F4F77CFB4A4920461EF075F802970FE0E1
:10C2000008224CF218638DE80C0028210523272210
:10C210002F4819F0FBFD424920461EF064F80295B4
:10C2200019230093912228237D21374801940EF091
:10C2300079FC20461EF017F899F80030002B00F02A
:10C24000C5822E4A013B1370C0E201232A462146D3
:10C2500030480EF0FFFAA8B12F4B1A780D2A0FD0F4
:10C260001A780E2A0ED10BE000210520FAF718F8F3
:10C2700039780620FAF714F82A4B06221A70A5E23C
:10C280000E2070E001232A46214622480EF0E2FAF1
:10C2900040B1214B1A780E2A04D91A78112A01D8F4
:10C2A000142060E001232A4621461A480EF0D2FAF3
:10C2B00000283BD0184B1A78122A37D1194A14207B
:10C2C000107000221A70FF2152E000BF34280300D2
:10C2D0005CC6FF1F000024400000184070BAFF1F1A
:10C2E000003C1C46942203000000204084BAFF1F3B
:10C2F000102303000000224098BAFF1F0188FF1F8F
:10C30000262303001CB9FF1FC0BAFF1FD0C5FF1FA3
:10C31000EB24030080B9FF1FEAC6FF1FE08EFF1F5A
:10C3200028230300FD87FF1F0088FF1F01232A46E3
:10C33000214697480EF08EFA30B1964B1A78122AA1
:10C3400002D91A78182A0DD901232A462146904885
:10C350000EF080FA78B18F4B1A781C2A0BD91A7814
:10C360001E2A08D811208C4A1070FF221A701978E2
:10C37000F9F796FF2AE201232A46214687480EF064
:10C3800069FA08B133787BB9002327225921844800
:10C3900018F08CFE4FF47841814817F0B4FB8149C6
:10C3A0007F48F4F7A3FA11E27F4B1B7823B17F4A51
:10C3B000136803F100431360764C2378012B14D1EA
:10C3C0007B4B7C4A1B78A82505FB0325774B186817
:10C3D00020F0E8FFC5E9120100210520F9F760FF10
:10C3E0006D4B06221A700025C5E02378032B0CD173
:10C3F0006F4B704A1B78A82505FB03256B4B18680B
:10C4000020F0D0FFC5E91601E6E723780B2B0CD10D
:10C41000674B684A1B78A82505FB0325634B186802
:10C4200020F0C0FFC5E92001D6E723780C2B0CD102
:10C430005F4B604A1B78A82505FB03255B4B1868FA
:10C4400020F0B0FFC5E92201C6E72378092B0CD103
:10C45000574B584A1B78A82505FB0325534B1868F2
:10C4600020F0A0FFC5E92601B6E723780D2B08D1FF
:10C470004E4B51491B680B601520F4F7BAF90E2298
:10C4800060E02578EDB20E2D0CD1484B4A491B686F
:10C4900041F8043F1A20F4F7ACF93F4B1D70FF231D
:10C4A0002370A0E723780F2B22D1404D43492E68FB
:10C4B000304621F0DDFD20B90021304621F0B0FDED
:10C4C00008B13E4B2B6028683D4E21F017FE3080AE
:10C4D0003C481DF025FD33883B493A484FF47A72B9
:10C4E00092FBF3F2F4F72AFA317840F2CD1026E00D
:10C4F0002378102B10D12D4D3449286821F0B8FD38
:10C5000008B1324B2B60286821F0F8FD304BC1B2E6
:10C51000197040F2CB1012E02378112B15D1234D66
:10C520002A4E2868314621F0A3FD00B12E6028680C
:10C5300021F0E4FD274BC1B219704FF4E670F4F717
:10C5400017F91422144B1A70A9E72378114D122BF6
:10C5500009D1164B20491B680B6040F2D310F4F749
:10C5600048F914222DE12B78122B39D92B78182B6E
:10C5700040F2168134E0194B581914350EF062F967
:10C58000B5F5DC7FF7D1044B21781878F0E600BFD1
:10C5900080B9FF1FEAC6FF1FFD87FF1F6CB9FF1F91
:10C5A0005CC6FF1F64280300E08EFF1FD0C5FF1F7D
:10C5B000A0C5FF1FF88EFF1F98C5FF1F00007F4317
:10C5C000EAC4FF1FDCC7FF1FF90500000000C842D6
:10C5D000F8B8FF1FEEC9FF1FB8C7FF1F1CB9FF1F28
:10C5E00023787C4D192B1DD17B4D7C4E286831461C
:10C5F00021F03EFD00B12E602868794D21F07EFDCE
:10C6000081B2298040F22710C9B2F4F7B1F8754B16
:10C61000297814221A70FF232370734A734B1278FF
:10C620001B783EE02B781A2B1BD16B4D6B4E286884
:10C63000314621F01DFD00B12E6028686A4D21F0C1
:10C640005DFD81B229804FF49470C9B2F4F790F87F
:10C65000644B14221A70FF232370644B2A781B78D2
:10C660001DE02B781B2B21D15B4D5C4E2868314699
:10C6700021F0FEFC00B12E6028685C4D21F03EFDEB
:10C6800081B2298040F22910C9B2F4F771F8554BF4
:10C6900014221A70544AFF23237012782B785049C1
:10C6A0000978534801905348009023E02B781C2BC5
:10C6B00024D1494D494E2868314621F0D9FC00B1BA
:10C6C0002E6028684B4D21F019FD81B229804FF46E
:10C6D0009570C9B2F4F74CF8424B41494448097887
:10C6E00014221A70FF2323703F4A404B12781B78A4
:10C6F0000190009540481AF091FA74E62B781D2BB2
:10C700000AD1354B186821F0F9FC3C4B1A8880B2ED
:10C71000904213D100200EE02B781E2B16D12E4B09
:10C7200037491D68284621F085FC38B1284621F09C
:10C73000E5FC324B80B21880F4F764F8294B1122E3
:10C740001A70304AFF23237013704CE62B781F2B8E
:10C750007FF449AE204B2B4F1868DFF8888021F01A
:10C76000CDFC264B1A8880B290424FF000060ED1C5
:10C7700030461E80F4F746F8234B1E70142388F8C9
:10C780000030224B1E70FF232B703B702BE60323DF
:10C7900088F800302E70FF233B7029783046E7E59B
:10C7A0000D4B2E78186821F0A9FC194BC1B2F6B2D6
:10C7B00028781E4400F5877006F8131CF3F7D8FF9D
:10C7C0001722084B1A70FF232B700CE60BB0BDE844
:10C7D000F08F00BFEAC6FF1FD0C5FF1F00007F43D8
:10C7E00066C5FF1FFD87FF1F3E8DFF1F34D5FF1F4E
:10C7F0001388FF1F08B9FF1FD8C5FF1FCA8EFF1F70
:10C8000000401C460188FF1FA0C5FF1FE88EFF1FC8
:10C810002CD5FF1F2DE9F74F0120F4F716F8344E01
:10C82000A82303FB00660022324BD6E9160120F054
:10C8300037FFD6E90E8902460B4604460D464046B0
:10C84000494620F02DFF21F0D9F85FFA80F8B8F1C1
:10C85000090FDFF8A49045D8D6E90E2329462046D3
:10C86000CDE9002321F0CAF81FFA80FB0BFB08FA80
:10C87000504620F085FD064619F808000F4620F0C6
:10C880006FFDC84404460D4698F8010020F068FD8D
:10C8900022462B4620F026FC3246804689463B46FF
:10C8A000DDE9000120F01EFC02460B4640464946E9
:10C8B00020F0CCFD80460BEB0A00894620F060FD9D
:10C8C00032463B4620F00EFC02460B4640464946A7
:10C8D00020F0E6FE22462B4620F006FC21F08EF8E2
:10C8E000C0B201E099F80A0003B0BDE8F08F00BFC4
:10C8F000F88EFF1F00002440BDC4FF1F37B5002481
:10C900004FF4D8708DF800408DF801400194F3F792
:10C91000D8FF00283CD023492348F3F7E7FF4FF422
:10C92000E270F3F792FF0128054609D01F491E481F
:10C93000F3F7DCFF21464FF4E270F3F719FF2546C9
:10C940001B491948F3F7D2FF002404F1D900400035
:10C9500080B28DF80150F3F7B4FFE2B2019069465E
:10C96000144816F02DFA0134019A13490E481DF0AF
:10C970006CFB082CE9D14FF4D8708DF80050F3F718
:10C98000A0FF0E490190024607481DF05EFB03E040
:10C990000B490548F3F705FE6946064816F0D4F939
:10C9A00003B030BD1A2A03008C8AFF1F262A030019
:10C9B0002B2A030038C5FF1F352A03003B2A03003A
:10C9C000472A03002DE9F04F5D4B5E4A1B7889B082
:10C9D0004FF00B0B06935C4B1B780BFB03234FF0C4
:10C9E000000A00250793594B1AF80340069B9C4206
:10C9F00080F08280564BA82202FB0434D4E9160151
:10CA00000022544B20F04CFED4E90E8902460B461E
:10CA100006460F464046494620F042FE20F0EEFF13
:10CA20005FFA80F8B8F1090F5CD83946304621F03A
:10CA300005F8D4E90E3406464046CDE9023421F02B
:10CA400007F9314621F058F920F0ACFC3D4B0BFBC7
:10CA50000A34CDE9000114F9080020F091FC08F136
:10CA6000010780463846894621F0F2F8314621F028
:10CA700043F920F097FCDDE9002320F033FB00228E
:10CA80000023E457CDE9040120F048FF00BB204615
:10CA900020F076FC42464B4620F024FBDDE90023E3
:10CAA00006460F46DDE9020120F01CFB02460B465C
:10CAB0003046394620F0CAFCDDE9042320F0F0FDC1
:10CAC00002460B464046494620F00EFB804689460A
:10CAD000284620F067FC42464B4620F005FB20F03C
:10CAE000ADFF08E0079B93F90A0021F0B1F8014679
:10CAF000284620F0F9FF05460AF1010ABAF1050FB0
:10CB00007FF471AF144B28461C7821F0D1FA00B2A3
:10CB100010F1640F03DB6428A8BF642001E06FF00C
:10CB2000630020F02DFC0A4BA82202FB0433C3E96A
:10CB30000E01D3E90E0120F081FF09B0BDE8F08FAE
:10CB40002AC4FF1FABC6FF1FE88EFF1FD08EFF1F3A
:10CB5000F88EFF1F000024400288FF1FFFFFFFFF29
:10CB60002DE9F04F9A4B9B4C1A7889B0032A059314
:10CB700060D126887822B3B293FBF2F602FB163618
:10CB8000002E57D1944D954B2B6008236B71944B1D
:10CB9000DFF87C921B78022B0CBF022300234FF09E
:10CBA00001082B72404664236B7285F80480F3F70A
:10CBB0004CFEA82707FB0090D0E90E0120F01EFFD5
:10CBC000C0F30720A8724046F3F73FFE07FB009032
:10CBD000D0E90E0120F012FF2E73E8726E73AE736F
:10CBE000EE73009695E80F00F3F71CFF7D4A13786B
:10CBF0004344DBB21370137803F0FF020BB97A4B96
:10CC00001A702A6879497A487A4E1DF01EFA06F1A0
:10CC1000080716F8012F784975481DF016FAB74233
:10CC2000F7D1764B6A791B680793079B7449704864
:10CC30001DF00BFA734B1B78032B40F08380724B73
:10CC40001B78FE2B7ED1714E714D3178A82707FBE2
:10CC50000151D1E90E010022002320F087FE0028B7
:10CC600070D0FFF7AFFE8246FFF7D4FD367807FBA2
:10CC70000651D1E91289834642464B46D1E9160155
:10CC800020F030FACDE90201584620F069FB024657
:10CC90000B46DDE9020120F0D9FB4BA3D3E90023C9
:10CCA00020F0FEFC42464B4620F01EFA594B002273
:10CCB00020F0CCFB20F0A2FE80B220F0C9FF564944
:10CCC0008046504621F0CCF801464FF07E5020F0CF
:10CCD00009FF0146404621F00FF821F00FFA4F4BB3
:10CCE00080B218804E4B93F800804E4B1B78434522
:10CCF0000AD920F0A9FF484921F0B2F820F052FBF0
:10CD000007FB0857C7E90E01A82707FB0655414B4B
:10CD10000022D5E90E0120F099FB20F047FE424B9E
:10CD20001860424819F02EFF60B1414B1D78414B0D
:10CD30001888414B188020F013FB354B07FB053555
:10CD4000C5E90E01059B1B78012B07D123882821FB
:10CD50009BB293FBF1F201FB123333B340F2191093
:10CD6000F3F773FD092826D123884FF4FA619BB2AB
:10CD700093FBF1F201FB1233D3B12388C8219BB29C
:10CD800093FBF1F201FB123393B1238801339BB281
:10CD90002380238842F6E0619BB293FBF1F201FB12
:10CDA00012335BB90B4A138008E0F4F74DFAD5E76C
:10CDB000F3F77EFEE9E70028E7D0DEE709B0BDE83B
:10CDC000F08F00BFAFF300800000000000E06F4074
:10CDD000AFC7FF1FF28EFF1F74C5FF1F00D1CC1C11
:10CDE000F18EFF1F2CC5FF1FE18EFF1F582003008F
:10CDF0008C8AFF1F7BC5FF1F5E20030058D8FF1FD2
:10CE0000642003006CC5FF1F0BB9FF1FFE87FF1FC7
:10CE1000F88EFF1F000059400000C842ECC9FF1FF8
:10CE20000E88FF1F2AC4FF1FE8C9FF1FD8C5FF1FB8
:10CE30000D88FF1F6EC5FF1FC6C5FF1F70B50679A1
:10CE40000023DAB2964209D9DA000468A518A2587C
:10CE5000914203F10103F4D1287970BD002070BD27
:10CE60002DE9F04F884B1B78042B95B082460C4679
:10CE700016462BD11323854A85490CA814F046FC8D
:10CE80000CA98448F4F7B6FB0CA814F0BBFA81484F
:10CE900014F0FBFAB8B152467F497E481DF0D5F830
:10CEA000651EE71D15F8012F7C497A481DF0CDF865
:10CEB000AF42F7D17A4B7B491B680B930B9B7548AC
:10CEC00032461DF0C2F8734814F0D3FA5146764842
:10CED000FFF7B4FFBAF5307F064626D1734B1B78B7
:10CEE000DF0756D572490023E05CC8540133082B94
:10CEF0006F4AF9D16F4B002119701178CD0701D518
:10CF000001220DE01178880701D5022208E011788E
:10CF1000C90601D5032203E01278920601D5042246
:10CF20001A70654B01221A7033E0BAF5A86F30D140
:10CF3000624B1B78FF2B2CD1614B624A1B78127815
:10CF40009A4226D9E079604A00F00F010F2910D1EA
:10CF5000A82505FB0325AF7A27F00F0747EA101035
:10CF600020F00EFAC5E90E01E37947EA1317AF7214
:10CF70000BE0062909D1A82505FB032520F00F00A9
:10CF8000AB7A03F00F031843A87201210920F4F7CC
:10CF9000A1FEDFF834B116B10136F3B214E0DBF8CC
:10CFA00004309A4540F05781F6E793F80890B9F1BC
:10CFB000060F16D0B9F1070F16D122781B699342DC
:10CFC00014D0019B0133DBB20193019B3E4A3E4FDB
:10CFD0005D1EEDB2A82303FB05235A689245E4D0F9
:10CFE00039E14FF0010803E0C84601E04FF00008C6
:10CFF000A82606FB057600230022CDE90C23B37A90
:10D00000012B0AD1F37A13B9737AE2560EE0737AE0
:10D01000E25C0023CDE90C2371E0B8F1010F17D1D8
:10D02000022B08D1F37A1BB9737AE25ED317F1E7CA
:10D03000737AE25AEDE7042B61D1F37A13B9737A6C
:10D04000E258F3E7737AE3580C9300230D9356E00C
:10D05000B8F1000F3AD1022B07D1F37A13B9737AE2
:10D06000E25E08E0737AE35A09E0042B47D1F37AD1
:10D070001BB9737AE258D2BAD8E7737AE3585BBA2D
:10D080000C93CDF834803AE0DAC7FF1F3821030053
:10D0900038D5FF1FF4C4FF1F592003005E20030092
:10D0A00058D8FF1F64200300F0C9FF1FAFC7FF1F40
:10D0B000ECC4FF1FE4C7FF1FE18EFF1F2CD5FF1F2D
:10D0C0004888FF1F2AC4FF1FF88EFF1FB8F1040F06
:10D0D00015D1042B13D1727AA118A25C4B781206D9
:10D0E00042EA0342CB781A438B7842EA0322D317F1
:10D0F000CDE90C230C9820F055F9C6E90E01A826BD
:10D1000006FB0576327B3369FF2A22D1FF2B2DD116
:10D11000DDE90C0120F06CF980466079894620F049
:10D120001FF902460B4600204C491DF097FC0246B1
:10D130000B464046494620F0B3FA8046E0888946CF
:10D1400020F01EF902460B46404649461FF0CAFF32
:10D1500026E05BB1B9F1070F08D0DDE90C01002131
:10D1600018401FF0ADFF20F043F911E0B8F1040FB3
:10D170004FF0A80606D106FB05B6D6E90A23D6E984
:10D180000E0107E0DDE90C0120F032F906FB05B6DF
:10D19000D6E90A2320F05AF9D6E90C231FF0A4FFA0
:10D1A000A823C6E90E0103FB057797F86830012B29
:10D1B00041D1D7E90E23CDE90423D7E91C23CDE9DA
:10D1C0000223D7E92223D7E91E01CDE90623DDE9B1
:10D1D00002231FF087FF00220023D7E92089CDE931
:10D1E000080120F09BFBF8B9DDE90223DDE9040129
:10D1F0001FF078FF42464B4606460F46DDE9060122
:10D200001FF070FF02460B463046394620F01EF9EB
:10D21000DDE9082320F044FA02460B464046494621
:10D220001FF062FF804689460D4AA82303FB0523B1
:10D23000C3E90E890AE0022B08D1BDF93010284657
:10D24000F6F78EFB20F09CF8C7E90E010121284675
:10D25000F4F740FDB5E615B0BDE8F08F00002440BE
:10D26000F88EFF1FFFFFFFFF2DE9F04186B01AF097
:10D2700007FCD34AD3480023FF2151825372138203
:10D280001946C21819500833B3F5007F1171CD4A01
:10D29000F7D1CD4B402100261A60197133469351C6
:10D2A00091190836B6F5007F4FF000040B71F6D1E6
:10D2B00040F29F10F3F7C9FA20F052F802460B46ED
:10D2C00000204FF080411DF0C9FBBBA3D3E9002330
:10D2D00020F0BCF820F092FB234601462246009441
:10D2E000BA4815F09DFCBA48BA4ABB49046080258B
:10D2F00005711FF0DFFEB948B64AB74905710460F1
:10D300001FF0D8FEB648B34AB349057104601FF058
:10D31000D1FE40F2C710F3F798FAB24B18704FF4F1
:10D32000E470F3F792FAB04B187040F2C510F3F7BF
:10D330008CFAAE4B1870AE4814F056F8A54AAD49B9
:10D34000AB481FF0B7FEAC4814F04EF8A14AA9490B
:10D35000A9481FF0AFFEA94819F036FD9D4AA8491B
:10D36000A6481FF0A7FE40F29910F3F76EFAD223F9
:10D3700002460821A3481AF0E0F8964AA249A148BB
:10D380001FF098FE4FF4C870F3F75FFA054640F2BD
:10D390009110F3F75AFA0B210D220C238DE80E00A1
:10D3A00002462946FF239948994D16F047FA9948B5
:10D3B00015F0E4FD40F2A910F3F747FA964B187008
:10D3C00040F27710F3F741FA944B18704FF4CD7098
:10D3D000F3F73BFA287040F29B10F3F736FA6870C7
:10D3E0004FF4CE70F3F731FAA87040F29D10F3F7C6
:10D3F0002CFAE87040F2C310F3F727FA287140F2D4
:10D40000A510F3F722FA864B864D187040F2A7104C
:10D41000F3F71BFA844B187040F21710F3F715FA64
:10D42000824B187040F21510F3F70FFA804B18700A
:10D430000720F3F70AFA7F4B18704FF49070F3F758
:10D4400004FA287040F21F10F3F7FFF9687040F2F9
:10D45000CB10F3F7FAF9784B784D18704FF4E6706B
:10D46000F3F7F3F9764B187040F2C910F3F7EDF9C2
:10D47000744B187040F2CD10F3F7E7F9724B188037
:10D480004FF4E770F3F7E1F9704B187040F2CF10EA
:10D49000F3F7DBF96E4B001B18BF012018704FF437
:10D4A000E870F3F7D2F96B4B187040F2D110F3F734
:10D4B000CCF9694B18704FF4E970F3F7C6F9674B74
:10D4C000187040F2D710F3F7C0F928704FF4EC70E1
:10D4D000F3F7BBF9687040F2D910F3F7B6F9A8700A
:10D4E0004FF4ED70F3F7B1F9E87040F2DB10F3F7A9
:10D4F000ACF928714FF4EE70F3F7A7F9687140F2B8
:10D50000DD10F3F7A2F9A8714FF4EF70F3F79DF96E
:10D51000E87140F2DF10F3F798F928724FF4F070D9
:10D52000F3F793F9687240F2E110F3F78EF9A872FD
:10D530004FF4F170F3F789F9494B4A4D18704FF4E5
:10D54000F770F3F782F9287040F2EF10F3F77DF9E6
:10D5500068704FF4F870F3F778F9A87040F2F110A2
:10D56000F3F773F9E8704FF4F970F3F76EF9287177
:10D570004FF49570F3F769F93B4D288040F227107E
:10D58000F3F763F9394B074618804FF49470F3F7BB
:10D590005CF9374B8046188040F22910F3F755F9B3
:10D5A000344B354A1880354B35490490019300952A
:10D5B00068E000BFAFF30080000000008084FE4000
:10D5C00054C4FF1FE8C7FF1FF0C9FF1F38C5FF1F66
:10D5D000C0C7FF1FF887FF1FC1060000DCC7FF1F81
:10D5E000408EFF1FF9B8FF1FDD8EFF1FDE8EFF1F6D
:10D5F00044C5FF1F05140200F4C4FF1F408DFF1F28
:10D60000B96C020014C5FF1F057302005CC6FF1F42
:10D61000B0C7FF1FA2C5FF1F2BC4FF1FF08EFF1F47
:10D620002DC5FF1FBDC7FF1F70C5FF1F3C8DFF1F0E
:10D63000E8C4FF1FA8C6FF1FF8B8FF1FBDC4FF1F27
:10D64000EEC9FF1F0AB9FF1FEAC4FF1F6CC5FF1F09
:10D6500028C4FF1FB0C5FF1FDF8EFF1F14CAFF1FA6
:10D660000BB9FF1FD08EFF1F08B9FF1F66C5FF1F34
:10D670003E8DFF1F34D5FF1F6EC5FF1F1388FF1F90
:10D68000E8C9FF1F5F4B0594CDF80C8002975E48F8
:10D690005E4D19F0E9FA40F22110F3F7D6F8287040
:10D6A0004FF49170F3F7D1F8687040F22310F3F75C
:10D6B000CCF8A8704FF49270F3F7C7F8E87040F216
:10D6C0002510F3F7C2F828714FF49370F3F7BDF803
:10D6D000687140F25F10F3F7B8F84D4D28704FF4C1
:10D6E000B070F3F7B2F8687040F26110F3F7ADF87C
:10D6F000A8704FF4B170F3F7A8F8E87040F2631027
:10D70000F3F7A3F828714FF4B270F3F79EF868713D
:10D7100040F2FB10F3F799F83E4B3F4D18703F482D
:10D7200015F02FFC4FF48A70F3F78FF83C4B18700C
:10D7300040F2A110F3F789F83A4B18704FF48B7050
:10D74000F3F783F8384B187040F2AB10F3F77DF81D
:10D75000364B18704FF4D570F3F777F8344B1870D8
:10D760004FF4FE70F3F771F8287040F2FD10F3F7F4
:10D770006CF868704FF4FF70F3F767F8A87040F228
:10D78000FF10F3F762F8E8703046F3F75EF828719F
:10D7900040F20120F3F759F8687140F20220F3F7E4
:10D7A00054F8A87140F20320F3F74FF8E8714FF4F2
:10D7B0000170F3F74AF8287240F20520F3F745F8B4
:10D7C000687240F20620F3F740F8A87240F2072092
:10D7D000F3F73BF8174B1870174B2246E2521434FC
:10D7E000B4F5027FFAD1154B002203F5EE6123F860
:10D7F000662C23F8022C70338B42F8D106B0BDE8BA
:10D80000F08100BFECC9FF1FD8C5FF1F2CD5FF1F3B
:10D81000C8C5FF1FE8C6FF1F84C5FF1FD4C7FF1F71
:10D82000AAC6FF1F64C5FF1FAFC7FF1FF18EFF1FF2
:10D83000FAB8FF1F29C4FF1F1CB9FF1F28BDFF1F17
:10D840002DE9F041074688B08846002408EB040320
:10D8500004AA03F1100E164618685968154603C548
:10D86000083373452A46F7D132466946094819F00C
:10D870008DFC6D463A192B4603CBB34210605160C4
:10D880001D4602F10802F6D11034C02CDED108B0DA
:10D89000BDE8F081408DFF1F2DE9F04FCDB0064669
:10D8A000B4491CA81CF01FFD1CA930461CF0AFFE9B
:10D8B00004461CA81CF0D7FC74BB08230A22AE49FE
:10D8C0001CA8F2F70FFE1CA930461CF081FD1CA815
:10D8D0001CF0C9FC062231461CA81CF0BBFEA7495F
:10D8E00014A81CF000FD14A91CA81CF090FE04460E
:10D8F00014A81CF0B8FC1CA81CF0B5FC64B90623E5
:10D90000224631461CA81CF085FE1CA930461CF09E
:10D910005FFD1CA81CF0A7FC99491CA81CF0E3FCA7
:10D9200031461CA81CF0F2FD96491CF0F7FD01469B
:10D9300004A81CF042FD1CA81CF095FC049C924914
:10D9400014A80123224613F0E1FE14A813F09DFD54
:10D95000002867D114A813F08CFD22468B498C480F
:10D960001CF073FB86491CA81CF0BDFC31461CA8AA
:10D970001CF0CCFD87491CF0D1FD014604A81CF029
:10D9800015FD1CA81CF06FFC224601237E49049D56
:10D990001CA813F0BBFE1CA914A8F3F72BFE1CA8AF
:10D9A00013F030FD14A813F070FD0446002839D19F
:10D9B0002A46794D794976481CF047FB2A887848F1
:10D9C0000A3A234612B20A2117F070FB754B2A88D7
:10D9D0001B8873480B214FF6E075693B0B3A1BB26D
:10D9E00012B28DE82200214618F010FA4FF4784167
:10D9F0006B4816F088F86C491CA81CF074FC314682
:10DA00001CA81CF083FD014665481CF0E7FA1CA821
:10DA10001CF029FC14A813F02CFD4FF4FA601AF046
:10DA20004DFDBEE14FF48C70F2F70FFFFF284FF071
:10DA3000000405D121464FF48C70F2F799FEB0E155
:10DA40005A4B5B4A1C705B4B5B4D1C70FF23137081
:10DA500053709370D3701371584A2B701370584AD7
:10DA60006B701370574A1370574A1370574A1370EC
:10DA7000574A1370574A1370574A14A8137013F07B
:10DA800004FD039570B1DFF85CB1DFF854A12746BF
:10DA9000A0462546A14614A813F0D8FC80B1002F5B
:10DAA00032D076E14D491CA81CF01DFC1CAA0A21AD
:10DAB0003148F2F741FD1CA81CF0D5FB052742E1D7
:10DAC000B8F10A0F14D9002F40F06781444B1B783E
:10DAD000012B12D021461CA8F4F726FB81450CD05F
:10DAE000404B1B682DB203EBC50243F8350014719F
:10DAF00014A813F0BEFC1FB125E114A813F0B9FC63
:10DB0000002C00F01F81ACE014A813F028FCC0B278
:10DB10000D2807D19AF80020012A03D0B8F1320F5E
:10DB2000B9D90A204CAB03EB08020A2802F8C00C52
:10DB30005AD19AF80020012A00F08280402C00F28D
:10DB40008880B8F10A0F40F2858021461CA8F4F7BE
:10DB5000EBFA484509D0DBF800302AB203EBC201EA
:10DB6000013543F83200EDB20C710134E4B2814664
:10DB700070E000BF572A030034C5FF1F4D26030085
:10DB8000282103003321030038D5FF1F5B2A03003F
:10DB90008C8AFF1F2E2103004488FF1F792A03006F
:10DBA0005CC6FF1F0888FF1F882A0300AEC7FF1F3F
:10DBB00001B9FF1FBFC7FF1F3F88FF1F4988FF1F15
:10DBC0004688FF1F0788FF1F0B88FF1F0D88FF1F58
:10DBD0000288FF1F0E88FF1F4888FF1F9D2A030031
:10DBE000A8C6FF1FF0C9FF1FB8F1BF0F2BD19AF8CD
:10DBF0000020012A30D11CA96F48FFF721FEC02266
:10DC00006D491CA819F00CFD402C03D902274FF0D8
:10DC1000BF0840E721461CA8F4F786FA814509D0E1
:10DC2000DBF800302AB203EBC201013543F83200C1
:10DC3000EDB20C710134E4B281464FF0FF080BE005
:10DC4000B8F1BF0FD7D0B8F1C00F34BF00270327FA
:10DC500002E002274FF0000808F101035FFA83F8A1
:10DC600019E7039B1B78FF2B07D0544AA82101FB1F
:10DC700003239A7A0AB902229A72039B5A78FF2ADE
:10DC800007D04E4BA82101FB02339A7A0AB902222F
:10DC90009A7230461CF0E5FC014608A81CF08DFB8A
:10DCA00047490CA81CF01FFB0CA930461CF0AFFC28
:10DCB0000022034608A910A81CF0ACFC10A908A873
:10DCC0001CF086FB10A81CF0CEFA0CA81CF0CBFAB6
:10DCD0000A9B062B03D83B4908A8F2F702FE08234B
:10DCE0000A22394910A8F2F7FDFB10A908A81CF078
:10DCF0008EFC054610A81CF0B6FABDB13349344875
:10DD0000F2F7F4FD08A932481CF068F908A910A838
:10DD10001CF053FB0A2110AA2B48F2F70DFC10A8A7
:10DD20001CF0A1FA2B492A48F2F73BFC2A4B197840
:10DD300001B101214FF48C70F2F71AFD08A81CF014
:10DD400092FA2EE00427254C254822880A3A00231F
:10DD500012B20A2117F0AAF9224B22881B880B2045
:10DD60004FF6E071693B0B3A8DE803001BB212B22B
:10DD700000211B4818F04AF84FF47841184815F074
:10DD8000C2FE3B463246184915481CF05EF9002495
:10DD900007E0B8F10A0F7FF6ABAE14A813F069FBE9
:10DDA000D1E714A813F02EFB04A81CF05CFA20465F
:10DDB0004DB0BDE8F08F00BFEBC6FF1FF88EFF1F10
:10DDC000A52A03004D26030034C5FF1FA92A03001E
:10DDD0008C8AFF1FB62A030000B9FF1F4488FF1F6B
:10DDE0005CC6FF1F0888FF1FBF2A0300034B1B7878
:10DDF0000BB1FFF751BD1846704700BF33D5FF1F69
:10DE00002DE9F04F08208FB0F2F71FFDFF2808D052
:10DE100001211AF0DDF90820F2F717FD00211AF0B0
:10DE2000A9F98E4C8E4D21788E48F2F7C4FB2978E3
:10DE30008C48F2F7C0FB69788A48F2F7BCFB4FF4D4
:10DE4000CD70F2F702FD00211AF0C2F940F29B10EA
:10DE5000F2F7FBFC00211AF0BBF94FF4CE70F2F799
:10DE6000F4FC00211AF0B4F940F29D10F2F7EDFC39
:10DE700000211AF0ADF94FF4C870F2F7E6FC012169
:10DE80001AF0A6F94FF4C870F2F7DFFC01211AF07E
:10DE900071F94FF4CB70F2F7D8FC01211AF098F920
:10DEA0004FF4CB70F2F7D1FC01211AF063F94FF473
:10DEB000CA70F2F7CAFC01211AF08AF94FF4CA704D
:10DEC000F2F7C3FC01211AF055F94FF4D770F2F7BD
:10DED000BCFC012804D900214FF4D770F2F748FCAC
:10DEE0002078062808D9002140F21710F2F740FCEC
:10DEF0005A4B00221A7006E0042804D90538022182
:10DF0000C0B21AF065F9584C2078062807D90021CC
:10DF100040F21510F2F72CFC0023237006E00428D1
:10DF200004D905380221C0B21AF052F94F4C2378B7
:10DF3000322B06D91E2140F2A510F2F719FC1E2340
:10DF400023704B4E00254FF4CA780127B1464FF09D
:10DF5000650A08FB05F30124F7500AFB05FB4FF4A3
:10DF60008E70F2F772FC844206D20BEB040301348C
:10DF700049F82370E4B2F2E70135072DE9D1142006
:10DF8000F2F763FC3B4C3C4E20701920F2F75DFC2D
:10DF90003A4960701520F2F74AFC39491A20F2F725
:10DFA00046FC384940F2D310F2F741FC002404F556
:10DFB000167504F263272846F2F747FCA5F5167399
:10DFC0000135AF42F054F6D10B34372CEFD140F28B
:10DFD000C310F2F73AFCFF2802D000211AF0F8F83B
:10DFE0004FF4E370F2F731FC01211AF0F1F84FF42D
:10DFF000E570F2F72AFC04464FF4E3702CB9F2F70F
:10E0000024FC21461AF0B6F809E0F2F71EFC0121C3
:10E010001AF0B0F801214FF4E570F2F7A9FB1A4CA1
:10E020001A4922780F481CF010F82278A046BAB39B
:10E03000174B197864291D462CD94FF4FE7400271C
:10E0400040F2072620460021F2F792FBA4F5FE736A
:10E050000134B442EF54F5D122E000BF3C8DFF1FE4
:10E06000BDC7FF1F8C8AFF1FE8C4FF1F2DC5FF1F00
:10E0700018CAFF1F2888FF1FABC6FF1F98C5FF1FC8
:10E080009CC5FF1FB8C7FF1FAFC7FF1FDF2A0300D4
:10E0900084C5FF1F032A03D9AB49AC48F2F781FAC4
:10E0A000AB48AC4CDFF8249319F03CF940F2771000
:10E0B000F2F7CBFBA84B1870F3F71CFD082140F2D8
:10E0C000A9102170F2F754FB2178A14819F03BF90F
:10E0D0004FF4B370F2F7B9FBA04B187040F2651023
:10E0E000F2F7B3FB9E4B0646187040F2671440F2FD
:10E0F0006F172046F2F7A9FB09EB44056FF4337262
:10E10000AB18A5F2CE25187004F10800F2F79DFBBC
:10E110000134BC422870ECD131468D4819F05AFACE
:10E120000220F5F753FB00210246894819F01BFA3B
:10E13000874819F04BF90820F2F787FBFF2802D037
:10E1400001211AF017F8874C874E64201AF0B6F9AF
:10E150000021864817F072F8FF2320783370F3F718
:10E160005FFA227882497948824C1BF06EFF7F4823
:10E1700015F038FD40F20710F2F767FB7E4B187080
:10E180004FF48370F2F761FB7C4B003018BF012025
:10E1900018704FF4BC70F2F758FB0128207002D0C1
:10E1A000C31E012B02D8002323700CE002280AD1E1
:10E1B0004FF4D070F2F749FB714B092888BF002259
:10E1C000187088BF1A7022786E4960481BF03DFFB6
:10E1D0004FF4D370F2F739FB6B4902465B481BF0F2
:10E1E00034FF4FF4CB70F2F730FB684902465748D2
:10E1F0001BF02BFF40F29710F2F727FB6449024611
:10E2000052481BF022FF20226249634818F06EFD3D
:10E2100003244FF4CB70F2F718FB01465F4813F06C
:10E22000D3F918B15E4B01221A700AE064201AF08B
:10E2300045F9013C5B494548F2F7B3F914F0FF0496
:10E24000E7D1574B03931A78002A65D140F2951015
:10E25000F2F7FBFA012119F0BBFF4FF4D370F2F78C
:10E26000F4FA012840F2951005D0F2F7EEFA0121F8
:10E2700019F080FF0CE0F2F7E8FA4B4919F004FFBF
:10E2800040F29510F2F7E1FA484B19781AF022F8AB
:10E29000474C36484FF4784115F035FC012133489E
:10E2A00015F02BFC22883148093A002312B20121D3
:10E2B00016F0FCFE22883F4B2C48B3F900304FF695
:10E2C000E0710A240A3A12B201910094002117F079
:10E2D0009DFD39492548F2F709FB37491B48F2F7FC
:10E2E00060F90321214815F008FC0023142221467F
:10E2F0001E4816F0DBFE4FF6FF711C4815F003FCBC
:10E300002E491A48F2F7F2FA4FF4FA601AF0D6F8EA
:10E3100000232B4C15485BE02A490C48F2F741F9E1
:10E3200040F2AF10F2F791FA0028F1D026491B48CD
:10E3300013F030FA0028EBD0002300931A46194658
:10E340002148F7F7C3FAE3E7F22A03008C8AFF1F9C
:10E3500014C5FF1F2BC4FF1FF08EFF1F4188FF1F36
:10E36000FC87FF1F2A88FF1FFD87FF1F5CC6FF1F5A
:10E37000052B0300DAC7FF1FFF87FF1F4388FF1F1E
:10E380004788FF1F152B0300252B0300352B0300A7
:10E39000452B03005D3C0300408DFF1F38D5FF1F58
:10E3A00033D5FF1F552B0300001BB74870C5FF1F57
:10E3B0004488FF1F0888FF1F5E2B0300702B03009B
:10E3C000B8BCFF1F822B0300902B03002F88FF1F78
:10E3D000E2187033B3F5EE6FD060B949F8D1B9489F
:10E3E0000023C2181433B3F5027F5160F9D1002025
:10E3F000F2F72BFAB44BB54C1870B54BB54F013052
:10E400001870F6F7AFFB2288B7F90030AC4800254A
:10E410000A210A3A8DE8220012B2294617F0F6FCCA
:10E420002288A7480A3A2B4612B2052116F03EFE72
:10E43000A949A348F2F75AFA40F29510F2F705FA03
:10E44000012119F0C5FE4FF4D370F2F7FEF901284F
:10E4500007D040F29510F2F7F8F9012119F08AFE81
:10E4600014E0FF2540F29510F2F7EFF9294619F074
:10E4700031FF01201AF022F8013DF3D140F295104E
:10E48000F2F7E3F9954B197819F024FF2288B7F9D0
:10E4900000308B4800250A210A3A8DE8220012B28A
:10E4A000294617F0B3FC228885480A3A2B4612B257
:10E4B000052116F0FBFD8A498148F2F717FA012180
:10E4C000884814F027FEF3F781F8874A136805930C
:10E4D000864B0599196092469946DAF80030069302
:10E4E000069BD9F800209B1A632B3BD8142019F007
:10E4F000E5FF4FF4CC70F2F7A8F919F05BFE054682
:10E500000028EAD1228801904FF00A090A3A014610
:10E51000642312B26A48CDF8009017F077FC228885
:10E5200067480A3A2B4612B2052116F0BFFD704922
:10E530006348F2F7DBF96E496E48F2F732F86E493C
:10E540000AA81BF0D0FE0AAA49466C48F1F7F4FF6E
:10E550000AA81BF088FE4FF47A7019F0AFFF4FF055
:10E56000010A01E04FF0000AF5F792FD0546F8B107
:10E57000228853480B2100250B3A8DE822006423A2
:10E5800012B217F043FC22884D480A3A2B4612B2C9
:10E59000052116F08BFD4FF47841494815F0B3FA88
:10E5A00057494748F2F7A2F90A2019F087FFFBE71D
:10E5B00054495048F1F7F5FF2288B7F90030404838
:10E5C00001954FF00B090B3ACDF8009012B2294695
:10E5D00017F01CFC22883A480A3A12B22B46052151
:10E5E00016F064FD48493648F2F780F947490AA811
:10E5F0001BF079FE0AA8FFF7F9FB454B18700AA833
:10E600001BF031FEF6F7AEFA2288B7F900302C483D
:10E61000CDF800900B3A12B22946019517F0F6FB9F
:10E6200022882748DFF898900A3A2B4612B2052133
:10E6300016F03CFD37492248F2F758F93649204890
:10E64000F2F754F9228839881D480A3A43392B4693
:10E6500012B209B216F02AFD30491948F2F746F90C
:10E6600098F8003083B1194B1A881A4B1988490859
:10E670000A3A0F3909B248462B4612B216F016FD77
:10E6800027494846F2F732F926491A48F2F72EF997
:10E69000254A1378042B144606D124491548F2F76D
:10E6A00025F94FF4164107E0052B45D120491148C3
:10E6B000F2F71CF94FF4E1311E481BF079FB63E0DF
:10E6C0005CC6FF1F1CB9FF1FE5C7FF1F4488FF1F63
:10E6D0000A88FF1F0888FF1F992B030070C5FF1FC2
:10E6E000AD2B0300A2C5FF1F58D8FF1FD88EFF1FF8
:10E6F000BB2B03008C8AFF1F9D2A030034C5FF1F1C
:10E70000CD2B030092230300EC2B0300572A0300B8
:10E710002AC4FF1FFD2B0300043F0300062C030047
:10E72000142C03001B2C030000B9FF1F2D2C030029
:10E73000332C0300648AFF1F062B01D1B149B6E7D1
:10E74000072B05D1B049B148F2F7D0F8B049B3E78B
:10E75000092B0DD1AF49AD48F2F7C8F8AE4819F012
:10E7600015FF062019F07AFFAC4B00229A720BE0DD
:10E7700033B1AB49A548F2F7B9F84FF496419BE79E
:10E78000A849A248F2F7B2F82178A048DFF8208320
:10E79000A54FF1F710FF40F21B10F2F756F8A3490E
:10E7A00002469A481BF051FC0024E3B2A346013410
:10E7B00022469F49954802931BF047FC4FF4CD70C9
:10E7C000F2F743F818F8015F854217D040F29B102A
:10E7D000F2F73BF8854211D04FF4CE70F2F735F8DE
:10E7E00085420BD040F29D10F2F72FF8854205D0FC
:10E7F000012D03D9093D012D00F23F828D4B39785F
:10E800001B788B4240F239828048F2F773F802217C
:10E8100098F8000019F0DCFC874B002243F82B200D
:10E82000029B012B854B05D01878854922284FF093
:10E83000030204E05878834922284FF0030228BFDE
:10E84000FF2019F0F7FC98F800207F496F481BF073
:10E85000FCFB3A787D4BA82101FB0233002283F8B0
:10E860009020022C07F101079FD1794D2A78531E81
:10E87000072B2F4626D8774964481BF0E6FB2B78F8
:10E880005A1E032A05D874480344002113F8010CCA
:10E890000AE0581FC0B2012809D8002119F098FCDD
:10E8A000287805382146C0B219F092FC11E0DA1F31
:10E8B000012A07D8981CC0B2002119F089FC2878D9
:10E8C0000230EFE7FF2140F2FB10F1F74FFF00238A
:10E8D0003B70624D62494D48F2F708F82B7803F01F
:10E8E000FD02012A66D15F4B1A78642A05D93221CC
:10E8F00040F2CB101970F1F73BFF5B4B1A78642A9A
:10E9000005D964214FF4E6701970F1F731FF574FC4
:10E910003B88042B03DDFF2BA8BFFF2300E005236A
:10E920004FF4FA723B80524C92FBF3F3514A13704E
:10E9300022780A2A04D840F28363D340DB0705D447
:10E94000002140F2C9102170F1F712FF0121207857
:10E9500019F03EFC484B374A1B7892F8008043453B
:10E9600002D2464A137006E00520F1F76EFF80459B
:10E9700084BF424B18702B78042B0CD1404923489C
:10E98000F1F7B4FF20783F4919F07EFB0021207891
:10E9900019F0A0FC08E03B883B493C484FF47A72F0
:10E9A00092FBF3F2F1F7CAFF2278394917481BF0BE
:10E9B0004CFB0FE00BB9374902E0022B04D136497A
:10E9C0001248F1F7EEFD05E034491048F1F7E9FD92
:10E9D00000232B7032490D48F1F788FF314B1B782B
:10E9E000002B67D0304C3149227808481BF02DFBB2
:10E9F0002078012119F0ECFB0021207819F0BAFBF6
:10EA00005CE000BF3B2C0300412C03008C8AFF1FFD
:10EA10006EDC0200472C030006800100488EFF1FB9
:10EA2000502C0300552C03003F88FF1F5B2C030074
:10EA3000652C03002AC4FF1F10B9FF1FBDC7FF1FAD
:10EA4000D9050000E90500007A2C0300F88EFF1FAD
:10EA5000E8C6FF1F8B2C0300B0C7FF1F6CC5FF1F4C
:10EA60009C2C0300F8B8FF1FEEC9FF1FEAC4FF1F6C
:10EA70000AB9FF1F1388FF1F0B88FF1FFE87FF1FA8
:10EA8000AF2C030000907B46F9050000DCC7FF1F98
:10EA9000B42C0300DC2C0300C52C0300D02C030095
:10EAA000E72C0300B0C5FF1FDF8EFF1FF02C030013
:10EAB000BCC7FF1F7A497B48F1F773FD4FF4D17053
:10EAC000F1F7FFFE784B80B242F20F72904218804D
:10EAD0001C4601D82B7823B90020F1F793FE0023C0
:10EAE0002380724D724F2B680793079B3B604FF456
:10EAF0007A783378FF2B17D12B680893089B3C68F2
:10EB000040F2AF101C1BF1F7A0FE08FB00F084429E
:10EB100000F2BA804FF4CC70F1F797FE19F04AFB7F
:10EB2000002800F0B180E4E70021624816F042FBC3
:10EB3000039B1B786BB1604B1B7853B9BAF1000F84
:10EB400007D15E4B187801385146C0B2F7F7F2F999
:10EB500001E0002333700120F4F73EFA584B594E80
:10EB600000241C7096F82730052BE2B201D00E2B42
:10EB700004D196F85830002B40F089800134112CD4
:10EB800006F17006EED1504B50491A784548504C6A
:10EB90001BF05BFA40F29F10F1F757FE1EF0E0FB0E
:10EBA00002460B4600204FF080411BF057FF3AA36E
:10EBB000D3E900231EF04AFC0B460246454939487A
:10EBC0001BF043FAFDF79AFE4FF48A70F1F73DFE11
:10EBD0004149024620460BF0D7F92046F1F7EDFEF9
:10EBE000C4F804903D492F483D4CF1F77FFEFA22CE
:10EBF0003C493D48F1F7A2FE142026681BF04BFD6E
:10EC00008046F1F7FBFE4146304613F0D9FF142051
:10EC100024681BF040FD0646F1F7E6FE314620462B
:10EC200013F0CEFF4FF4CC70F1F70FFE0322212832
:10EC300088BFFF202D4919F0FDFA2D491948F1F739
:10EC4000B0FC2B680A930A9B2A4916483B60F1F7EF
:10EC50004DFE2B68099309991248F1F764FE0020D4
:10EC6000F4F7B4FD00210246234818F07CFC22484A
:10EC700018F0ACFB0FB0BDE8F08F20490948F1F760
:10EC800090FCFF233B70ECE50023337031E7718A81
:10EC9000308AF7F703F871E7000000008084FE4037
:10ECA000BD2D03008C8AFF1FCA8EFF1F58D8FF1F7F
:10ECB000D88EFF1F5CC6FF1FFD87FF1F0A88FF1F3E
:10ECC000CEC5FF1FB8BCFF1F64C5FF1F012D030089
:10ECD00054C4FF1F1B2D030038C5FF1F2C2D03003C
:10ECE000A4D7FF1F61CB0000C0C7FF1FF16E01005A
:10ECF000422D0300492D030014C5FF1F8A2803007D
:10ED00002DE9F04FA7B006AF07F1200381464FF47D
:10ED1000CC7083E80600F1F798FDB24DB7F92040BA
:10ED2000B7F922A0212888BFFF2019F07FF901231D
:10ED30002B70AD4BBB61187808B9F4F793FDA3B203
:10ED4000AA4C3B612368FB62A94BFA6A1A604FF434
:10ED5000E170F1F77AFD7C6140B10021F023009170
:10ED60001A463869F1F735FD03B210E04FF6C16677
:10ED70001AFB06F640F2411396FBF3F63B6906F5E3
:10ED8000A07603F101080FFA86FA0FFA88F3994882
:10ED9000FB6114F027FF984A1478FF2C934611D199
:10EDA000964909881839002351452B7006DCF9690A
:10EDB000182903DC0123137002F06FBD8BF80030BB
:10EDC00002F06BBD012C40F2A980162C04D88C4BAC
:10EDD000E340DA0700F14381884B1B88313B534500
:10EDE00078DCFA69132A75DC864E96F80080B8F153
:10EDF000FF0F40F03181844C2078F2F711FC86F847
:10EE00000080F2F7ABFE9BF800300B2B09D17F4B53
:10EE100040F2A7101978F1F7ABFC7D4B1A787D4BC7
:10EE20001A709BF80030022B06D17A4B1878013803
:10EE3000C0B2F6F715FC07E006D9764B1878013812
:10EE40000021C0B2F7F776F8734B10225A72734B59
:10EE50001B78042B03D101210846F3F7C7FD704B43
:10EE6000DFF8EC81DFF8EC916E4E01221A704FF062
:10EE7000000A6D4B504683F800A0F4F7ADF80A2065
:10EE800019F01CFB2078694CF2F7CAFB554694F840
:10EE90002730052B5FFA8AF202D00E2B42F01F8535
:10EEA00094F85810002902F03885618A208AF6F714
:10EEB000F5FE0AF1010ABAF1110F04F17004E6D16E
:10EEC0005B4BFF20187000238BF80030F5F7EEFF46
:10EED00002F0E3BC022C40F0C280534500F3C18035
:10EEE000FB69132B00F3BD80464E3378FF2B00F0F7
:10EEF000B8804E48702404FB03000122FF210CF06F
:10EF000069FBF2F72BFE0120F6F7A6F8F6F7C8FF2B
:10EF1000474AFF233370137002F0BFBC002C40F04F
:10EF20009E8001231370434A32481370424A3F4D7A
:10EF3000424E137014F056FEBC6195F8583097F8A5
:10EF4000189033B31FFA8AF80123BA8B414628463A
:10EF50000BF0ECFF18B12C4B1B78032B0DD03B6949
:10EF6000C3F1F0014246012389B228460BF0DEFFCF
:10EF700078B1254B1B78032B0BD095F82730092B44
:10EF800042F01D852E4B1B7803F0FD03012B02F090
:10EF90006C85BB690133112BBB6105F17005CCD1C8
:10EFA000002C42F07A84274A274B1078197888423F
:10EFB00015461C4606D2254B1878222828BFFF206C
:10EFC00019F034F86A7823789A4206D21F4B5878A1
:10EFD000222828BFFF2019F029F80020F6F73CF876
:10EFE00002F05BBCCEC5FF1FE08EFF1F58D8FF1F8D
:10EFF00028C5FF1F5CC6FF1FFD87FF1F0888FF1F76
:10F00000004561004A88FF1F2A88FF1F70C5FF1F47
:10F010000C88FF1F0A88FF1F54C4FF1FDAC7FF1F99
:10F020004288FF1F0BB9FF1FFBB8FF1FB8BCFF1FB3
:10F030000188FF1FD4C5FF1FE9C6FF1FDD8EFF1F1C
:10F04000AFC7FF1F3F88FF1F2AC4FF1FBDC7FF1F99
:10F05000F9B8FF1FB0C5FF1F022C3FF445AF142CB9
:10F0600033D8BD4BE340DE0708D5BC4B1B78FF2BE4
:10F0700004D1AAF138039BB22B2B09D90A2C24D135
:10F08000B74B1B88313B534547F3758602F005BCEF
:10F09000FB69132B19DCB34B00241C70AF4BFF2210
:10F0A0001A70B14A01231370B04A2B7002201370FA
:10F0B000F5F7D2FF03238BF80030F2F74FFD21461E
:10F0C0002046F7F7EDF802F0E8BB022C7DD1DFF81F
:10F0D0008C8298F80030FF2B41F0CE81AAF16E03AC
:10F0E0009BB2362B0CD8FB69132B09DCF2F724FDFD
:10F0F000FF28834604D09E4B1B78012B42F03786B5
:10F10000AAF1A7039BB22C2B14D8FB69132B11DC9B
:10F11000974B1A78012A14BF0122002201201A708D
:10F12000F5F79AFF934B18780138C0B2F6F798FAC2
:10F1300002F0B3BBAAF1D6039BB22D2B01F29C8146
:10F14000FB69132B01F39881894B1B78012B01F08C
:10F1500093810320F2F764FA0121874814F0CDFC73
:10F160000021854814F0CFFC844B1A78032A05D17E
:10F1700002221A704CF21863019308E0022A08BFB9
:10F1800004214CF2186218BF0321197001920B235D
:10F19000009301222B23D721774816F037FE7849B8
:10F1A00007F170001BF09FF805230093032207F17D
:10F1B0007003ED2173480CF0CBF907F170001BF0E0
:10F1C00052F8F6F76DFE02F068BB012C1BD0032C41
:10F1D00005F0FB87042C07F02581052C06F0FD8245
:10F1E000072C07F019810C2C07F004810D2C07F077
:10F1F0000781112C07F00A81122C06F08A84142C46
:10F2000016D106F0AFBCBAF1310F06F31383BAF191
:10F21000000F46F30F83FB69272B47F3B285012CC0
:10F2200006F00883032C05F0D487142C06F09E8486
:10F23000182C2BD1FB69322B10DD534BFA691B883C
:10F24000323B9A420ADA514B1A78FF2A06D1002142
:10F2500020461970F7F724F802F01FBBBC8B4C480E
:10F260001FFA8AF60123224631460BF0F3FA0028F2
:10F2700002F0E085454B1978FF2902F0DB85454A0D
:10F28000535C632B42F2EA8502F0D4BD162C3CD1CC
:10F29000FB69692B13DD3C4BFA691B881E3B9A42C4
:10F2A0000DDA3D4B1A78FE2A09D0384A0021117038
:10F2B0002046FE221A70F6F7F3FF02F0EEBABC8B7E
:10F2C00033481FFA8AF60123224631460BF0C2FA70
:10F2D000002802F0CA862D4B1978FF2902F0C58656
:10F2E0002E4D2F4B2A780B2000FB02325256632AF8
:10F2F00002F3BB862A7800FB023316205A5C0132E7
:10F300005A54F6F7CDFF02F0C8BA152C4CD1FB6960
:10F310001E4D322B09DD2B78FF2B06D10021204614
:10F320002970F6F7BDFF02F0B8BABE8B18481FFA75
:10F330008AF40123324621460BF08CFA002803F0B0
:10F3400063802978FF2903F05F80164A535C632BA2
:10F3500043F2A38003F058B8B6F217000188FF1FEC
:10F360000888FF1FBCC4FF1FD4C5FF1FE9C6FF1FCD
:10F370001288FF1F0A88FF1F5CC6FF1F2A88FF1F15
:10F3800064230300B8BCFF1F4488FF1FA0C5FF1FF4
:10F390001CB9FF1F84C5FF1FE88EFF1FEAC6FF1FB1
:10F3A000ABC6FF1FBDC4FF1F112C73D1B7F81C8063
:10F3B000C4481FFA8AF60123424631460BF04AFA46
:10F3C00050B34FF48E70F1F740FA0130C4B2292CDB
:10F3D00028BF022421464FF48E70F1F7C9F9BA49CB
:10F3E00007F160001AF07FFF214607F170001AF064
:10F3F0009AFF4CF2186307F1700207F16001B148FF
:10F400000BF0ECFA07F170001AF02DFF07F1600025
:10F410001AF029FF02F041BA012342463146AB48B7
:10F420000BF018FA002803F0A2804FF4D670F1F721
:10F430000CFA002843F09B80A54907F150001AF010
:10F4400052FFA44907F160001AF04DFFA24907F1ED
:10F4500070001AF048FF4FF4FC6307F1500107F108
:10F4600060020093994807F170030BF0FFFA07F16F
:10F4700070001AF0F8FE07F160001AF0F4FE07F1D0
:10F4800050001AF0F0FE01214FF4D670F1F770F938
:10F4900002F003BA172C40F09F80FB692C2B0EDC86
:10F4A0008E4A002313708E4A13708E4A1120FF215A
:10F4B00013708BF80000F6F7F3FE02F0EEB9B7F820
:10F4C0001C8089481FFA8AF60323424631460BF016
:10F4D000C1F9054670B1834B13221A7009238BF8CA
:10F4E0000030824B18781DF03BFF0022F5F7AEF993
:10F4F00002F0D3B903234246314672480BF0AAF911
:10F50000044670B1774B14221A7009238BF800302F
:10F51000764B58781DF024FF2A46F5F797F902F04C
:10F52000BCB903234246314671480BF093F970B1E0
:10F530006C4B15221A7009238BF800306B4B9878AE
:10F540001DF00EFF2246F5F781F902F0A6B903235C
:10F55000424631465D480BF07DF970B1614B162291
:10F560001A7009238BF80030604BD8781DF0F8FE34
:10F570000022F5F76BF902F090B9032342463146B9
:10F580005C480BF067F9044670B1564B17221A70AD
:10F5900009238BF80030554B18791DF0E1FE00224D
:10F5A000F5F754F902F079B903234246314652483F
:10F5B0000BF050F9002802F070814A4B18221A70A3
:10F5C00009238BF80030494B58791DF0C9FE2246BB
:10F5D000F5F73CF902F061B9122C40F041810021AD
:10F5E000464814F090FAB7F81C803F481FFA8AF694
:10F5F0000123424631460BF02DF9054668B1404BD8
:10F6000000221A80364B022201201A70F4F702FF02
:10F6100013238BF8003002F040B9012342463146F3
:10F6200028480BF017F9044660B1354B1D802C4B70
:10F63000042201201A70F4F7EDFE13238BF800303A
:10F6400002F02BB901234246314629480BF002F95A
:10F65000054660B12A4B1C80214B062201201A70FE
:10F66000F4F7D8FE13238BF8003002F016B901230B
:10F670004246314615480BF0EDF8044660B1204B88
:10F680001D80174B082201201A70F4F7C3FE1323C4
:10F690008BF8003002F001B901234246314615488B
:10F6A0000BF0D8F8054668B3154B1C800C4B0A22AA
:10F6B00001201A70F4F7AEFE13238BF8003002F02D
:10F6C000ECB800BF30B9FF1FFD28030058B9FF1F79
:10F6D0009D2403000629030087240300A0C5FF1F03
:10F6E000E88EFF1FEAC6FF1F1CB9FF1F2CD5FF1FA6
:10F6F00044B9FF1F6CB9FF1F80B9FF1F5CC6FF1F15
:10F70000ACC7FF1F012342463146C5480BF0A2F8A3
:10F71000044660B1C34B1D80C34B0C2201201A70FC
:10F72000F4F778FE13238BF8003002F0B6B801230B
:10F7300042463146BD480BF08DF8054660B1B94BE5
:10F740001C80B94B0E2201201A70F4F763FE1323BC
:10F750008BF8003002F0A1B8012342463146B4488C
:10F760000BF078F8044660B1AE4B1D80AE4B102212
:10F7700001201A70F4F74EFE13238BF8003002F0CC
:10F780008CB8012342463146AA480BF063F858B1C1
:10F79000A44B1C80A44B01201C70F4F73BFE1323E8
:10F7A0008BF8003002F079B8012342463146A24876
:10F7B0000BF050F850B100214FF4D870F0F7E6FF8D
:10F7C00000211220F6F76CFD02F067B801234246D3
:10F7D00031469A480BF03EF8044678B14FF4D8749D
:10F7E000204600210134F0F7C3FFB4F5E17FF7D1E3
:10F7F00000211220F6F754FD02F04FB801234246D3
:10F8000031468F480BF026F8002803F047814FF46B
:10F81000E270F1F71AF8012843F04081894907F1B5
:10F8200060001AF060FD884907F170001AF05BFD76
:10F8300007F1600146F22C3307F1700280480BF0AB
:10F84000CDF807F170001AF00EFD07F160001AF014
:10F850000AFD21464FF4E270F0F788FF02F01DB870
:10F86000132C5AD1794C267896B907F1700578494E
:10F8700028461AF038FD0F2300937648029601952A
:10F88000DC2323222D210BF04DF928461AF0EBFC46
:10F89000002171486D4D14F036F901216E4814F0C5
:10F8A0002CF921786C4801EB410149000023272203
:10F8B000323115F0FBFBB7F81C8060481FFA8AF65E
:10F8C0000123424631460AF0C5FF002803F0948127
:10F8D0002B78032B03F2908160495F48F1F706F81B
:10F8E000504A2978138801311B010133C9B21380B2
:10F8F00029700A22C1F1040107F170001AF026FDF7
:10F900004FF6E07207F1700148480BF031F807F14B
:10F9100070001AF0A8FC01F0C0BF082C4FD1504B6A
:10F92000504C1B88313B534519DCFB69132B16DC0B
:10F930004D4BFF221A704D4B01251D704C4B022080
:10F940001D70F5F789FB03238BF80030F2F706F9F9
:10F95000002108462570F6F7A3FC01F09EBFBAF11E
:10F96000330F10DCFB69132B0DDC3F4B0022012110
:10F970000A201A70F6F794FC012364202370F5F72F
:10F9800095FA01F08ABFAAF13606B6B2322E4FF0D0
:10F9900001050ED8FB69132B0BDC334B00210A2029
:10F9A0001D70F6F77DFC64202570F5F77FFA01F0F5
:10F9B00074BF64202570F5F779FA01F06EBF072C4B
:10F9C00040F0C181BA69BD8B2A4800231FFA8AF42E
:10F9D0001370214601232A460AF03CFF064660B117
:10F9E000254A1378591EC9B2FF29117001D10C2183
:10F9F00049E0082948D1072145E001232A4621464C
:10FA00001E480AF027FF8046002844D01A4A13787F
:10FA1000591CC9B20C29117032D9167034E000BFDC
:10FA200080B9FF1FACC7FF1FE88EFF1F94B9FF1FEF
:10FA3000A8B9FF1FBCB9FF1FD0B9FF1FE4B9FF1F52
:10FA4000F8B9FF1FBB290300252603000088FF1F0C
:10FA50002721030058B9FF1F5CC6FF1F7026030053
:10FA60000888FF1F4288FF1F0188FF1FD4C5FF1FA2
:10FA7000E9C6FF1F1CB9FF1FA0C5FF1F30B9FF1F3C
:10FA8000082901D10921117012782D210220F2F7E5
:10FA90009DF903F072BC01232A462146BE480AF0B4
:10FAA000D9FE002857D0BD4DBD482988DFF81093F6
:10FAB0005F393722434609B215F0F8FAF5F752F8E4
:10FAC000B849B748F0F712FFB74B4FF4B370197845
:10FAD000F0F74EFEB54B40F265101978F0F748FE8E
:10FAE00040F2671440F26F1663006FF4337B5B449F
:10FAF000204619F80310DFF8C8820134F0F738FE09
:10FB0000B442F1D140F277166300A3F2DE2320461F
:10FB100018F803100134F0F72BFEB442F4D1322070
:10FB200018F0CCFC29889E480A234FF0000A5F3960
:10FB30008DE8080437225E2309B216F067F99C4B62
:10FB400020461978F0F714FE9A4B40F2A910197864
:10FB5000F0F70EFE81E001232A46214696480AF07E
:10FB600079FE48B1954B1A78082A05D8944911F8BE
:10FB70001230002B43F0848301232A46214691480A
:10FB80000AF068FE20B18D4B1A78082A43F2708380
:10FB9000BAF1190F08DDDFF80482B8F80030A3F1DC
:10FBA0007D029245C3F2708301232A462146824892
:10FBB0000AF050FE002843F0878301232A4621469D
:10FBC00080480AF047FE002843F08F83BAF1190FEE
:10FBD00008DDDFF8C881B8F80030A3F17D02924556
:10FBE000C3F2958301232A46214673480AF032FE68
:10FBF000002843F0AD8301232A46214671480AF0CC
:10FC000029FE002843F0B083BAF1190F06DD634ED8
:10FC10003388A3F17D029245C3F2B58301232A46BE
:10FC2000214665480AF016FE002803F0CA83634B9C
:10FC30001B780B2B43F0C583634A1378002B03F02A
:10FC4000C083012B43F2CA83023B137001210920B8
:10FC5000F6F726FBBA6901231370BB691B78002BEA
:10FC600001F01B86584B504A1978127891429846F9
:10FC700010D9564C207838B1514BD87BF3F7F2FDB0
:10FC80000023237001F009BEF3F7ECFD012323707C
:10FC900001F003BE4FF4D470F0F7D7FD484C0128B3
:10FCA00094F80F902AD14FF0000A0546A27B98F8ED
:10FCB00000309A421FFA8AF60CD80DB194F80F90D2
:10FCC0004846F3F783FD31460246414817F04BFCA6
:10FCD000002507E00020F3F779FD314602463C4855
:10FCE00017F041FC0AF1010ABAF1080FA4F102046D
:10FCF000DCD1374817F06AFB01F0CFBD072501269C
:10FD00004FF6FF7AA27B98F800309A420CD80EB1D9
:10FD100094F80F904846F3F759FD294602462C48BF
:10FD200017F021FC002607E00020F3F74FFD2946DD
:10FD30000246274817F017FC013DADB25545A4F126
:10FD40000204DFD1D5E7052C40F0C780B7F81C903E
:10FD5000204D1FFA8AF801234A46414628460AF0F8
:10FD600079FD2C460646002854D0144E1A4D33789F
:10FD70002A78C2EB0308013BDBB2FF2B5FFA88F85D
:10FD800033702DD1154B1B785A1ED2B20C2A32700B
:10FD90002ED90D3B2B7027E044B9FF1F0888FF1FA9
:10FDA0005CC6FF1F662D03004188FF1FFC87FF1FF5
:10FDB000F08EFF1F2BC4FF1F58B9FF1FA0C5FF1FE8
:10FDC0002F88FF1F6CB9FF1F3E8EFF1FC4C5FF1F8A
:10FDD00014C5FF1F1CB9FF1FE88EFF1F2AC4FF1F99
:10FDE0009A4205D9013A2A7000210420F6F758FA00
:10FDF00033782A78618920899A1AE3891944D2B222
:10FE0000434689B2F1F7E2FF00210520F6F748FAF0
:10FE100001F043BD414601234A4605F114000AF0B2
:10FE200019FD8046002838D0BE4ABF48137890F8A4
:10FE300000E0CEEB03050133DBB2CEEB03010C296E
:10FE4000EDB21370B9499046814607DD0A789A42AF
:10FE500004D90EF101030370314607E00A789A4293
:10FE600007D8002188F8001089F800100420F6F760
:10FE700017FA98F8003099F80020618920899A1AB9
:10FE8000E3891944D2B22B4689B2F1F79FFF0021D2
:10FE90000520F6F705FA01F000BDA54B1B88643B71
:10FEA0009A4581F2FA84FB69142B41F3F6849D4B49
:10FEB0009D4A1B781278698928899B1AEA8911441E
:10FEC000DBB2FF2289B2F1F781FF062041468BF8B1
:10FED0000000F6F7E5F901F0E0BC062C40F0A9823D
:10FEE000B7F81C80934D1FFA8AF60123424631462B
:10FEF00028460AF0AFFC814658B18F4C002120788B
:10FF0000F1F78EFF002120700720F6F7C9F901F004
:10FF1000C4BC01234246314605F114000AF09AFCA4
:10FF2000824658B1844C01212078F1F779FF494687
:10FF300020700720F6F7B4F901F0AFBC0123424668
:10FF4000314605F128000AF085FC814668B37A4CF9
:10FF500005238BF80030794B2078FF2202211A709C
:10FF6000F1F75EFF724B2070198875485F39534670
:10FF7000372209B215F09AF8F4F7F4FD714B2178A5
:10FF8000012203201A70F6F78BF9664B664A1B783C
:10FF90001278698928899B1AEA89DBB2114489B2EF
:10FFA0001A46F1F713FF01F078BC012342463146AF
:10FFB00005F1B4000AF04EFC8246002800F02882C9
:10FFC0005D4D2B78082B2E464CD1DFF858A15E4EA4
:10FFD0009AF8003029784FF0A80808FB0363FF2245
:10FFE00083F891202046F6F75BF901210720F6F708
:10FFF00057F94FF6FF71524813F085FD2B785048A2
:020000021000EC
:10000000CDF8049003EB430203EB82022D32092367
:10001000009312B25A23642115F0F8FE2B78484859
:1000200003EB430203EB82022D324B4612B26721EF
:1000300015F03CF89AF8003008FB03663B4B96F845
:1000400091101B784A4607F170000AF01BFF07F178
:1000500070013B4819F0C2FF07F170001AF003F974
:1000600001F01BBC2B780B2B0FD12E4B1A78364B83
:10007000A82101FB0233D3E920010122F4F7E6FBBA
:1000800009238BF8003001F008BC2B780C2B0FD122
:10009000244B1A782C4BA82101FB0233D3E922010F
:1000A0000122F4F7D3FB09238BF8003001F0F5BBF4
:1000B0002C78E4B2092C0ED11A4B1A78224BA821C5
:1000C00001FB0233D3E926010122F4F7BFFB8BF8D1
:1000D000004001F0E2BB2B78012B0FD1114B1A78B5
:1000E000194BA82101FB0233D3E912010122F4F7D5
:1000F000ADFB09238BF8003001F0CFBB2B780E4C01
:10010000032B23D1074B1A780F4BA82101FB023395
:10011000D3E916010122F4F799FB09238BF800308B
:1001200001F0BBBBA0C5FF1FE88EFF1F2AC4FF1F45
:100130000888FF1F1CB9FF1FEAC6FF1F0188FF1FA9
:100140005CC6FF1FBCC7FF1FF88EFF1F2378052B5F
:1001500035D1BF4D2C78002021460AF06BFE80F08F
:100160000101C9B220460AF03DFE00210720F6F742
:1001700097F84FF6FF71B74813F0C5FC0024092328
:100180008DE818006E223C236421B24815F03EFE33
:1001900023466E226721AF4814F088FF2978204655
:1001A0000AF048FEF2F7CEFE297820460AF042FE19
:1001B0006D2102465120F2F789FD01F06EBB2378D4
:1001C000062B51D1A24DA44E2C78012021460AF0D5
:1001D00031FE80F00101C9B220460AF00DFE3378ED
:1001E00008B1013300E0013B0021072000243370F7
:1001F0004FF00908F6F754F84FF6FF71954813F0E1
:1002000082FC0194CDF800803C237B22642191483C
:1002100015F0FCFD23467B2267218E4814F046FF33
:10022000297801200AF006FEF2F78CFE0194CDF841
:10023000008008237B223D21864815F0E7FD2346F8
:100240007B223D21834814F031FF31788148F0F75B
:1002500051FB297801200AF0EDFD7A210246512058
:10026000F2F76EFD01F019BB237803F0FF057BBBAD
:10027000774B1A78794BA82101FB0233002000212B
:10028000C3E910014CF21861724813F03CFC23786A
:100290007048019503EB430203EB82022D320923E0
:1002A000009312B23C23642115F0B0FD2378694815
:1002B00003EB430203EB82022D322B4612B267217D
:1002C00014F0F4FE66496348F0F710FB01F0E5BA5C
:1002D0002378022B30D15E4B1A78604BA82101FBAA
:1002E000023300200021C3E914014CF2186159487F
:1002F00013F009FC2378574803EB430203EB820217
:10030000002509232D328DE8280012B23C236421F8
:1003100015F07CFD23784F4803EB430203EB820288
:100320002D322B4612B2672114F0C0FE4C494948C9
:10033000F0F7DCFA01F0B1BA2578EDB2072D35D12E
:10034000434C2678032031460AF074FD80F0010109
:10035000C9B230460AF064FD28460021F5F7A0FF37
:100360004FF6FF713B4813F0CEFB002509238DE8C3
:100370002800882246236421364815F047FD2B4685
:1003800089226721334814F091FE217803200AF076
:1003900051FDF2F7D7FD217803200AF04BFD8921AA
:1003A00002465120F2F7B8FD01F077BA23780A2B04
:1003B00041F073822B4B294801221A70244B197883
:1003C000A82202FB010292F868300133DBB2022B53
:1003D00082F8683006D8546840F6FF72944207D01D
:1003E000022B05D1A82303FB0101002381F868300B
:1003F00000210520F5F754FF307801300021C0B20C
:10040000F1F70EFD00210720F5F74AFF01F045BA8C
:1004100001234246314605F150000AF01BFA00283C
:1004200003F03381104B1B78082B43F03F8103F01E
:100430002CB9092C1AD1BB8B7B84A7F820A007F11B
:10044000200393E80300FBF721FC01F026BA00BF6C
:10045000A0C5FF1F5CC6FF1FBFC7FF1FF88EFF1F91
:10046000712D0300CEC5FF1FEAC6FF1F042C01F04B
:100470001482022C40F03D81112300257B61BD6177
:10048000B64B1B78AB4202D0FF2B40F01781BB6903
:10049000B34EB44AB7F81C900133DBB27024BB6191
:1004A00004FB056400231FFA8AF8137041460123F8
:1004B0004A4620460AF03AFD40B1AB4B1B78032B6D
:1004C00004D1AA4B1B78012B26D12EE03B69C3F146
:1004D000F0014246012389B220460AF027FD48B1C7
:1004E000A14B1B78032B05D04FF4E170F0F7ADF969
:1004F0000028E6D001234246396920460AF016FD5D
:1005000098B1994B1B78032B0FD04FF4E170F0F7A3
:100510009CF90028D5D108E094F858302BB194F814
:1005200025B0BBF1000F03F00882904B1A78012A26
:1005300010D1BAF1310F43F3BA818D4B198831399B
:10054000514543F3C481BAF1310F43F3D081514592
:1005500043F3E08194F82530BB60002B00F0AE80BF
:10056000022AFB6903F00F82162B03F3F883A8F12C
:100570009F0189B2312994F8273043F2FA81A8F11A
:10058000D10080B2332808D803F1FF3EBEF1010F3D
:1005900043F222840D2B03F01F84A8F1D20E1FFA20
:1005A0008EFEBEF1180F07D894F82730062B03F003
:1005B0006884032B03F06584A8F1ED03182B07D89A
:1005C00094F82730062B03F06D84032B03F06A8424
:1005D000BEF12E0F04D894F827300C2B03F07C8446
:1005E000A8F1A0032F2B43F27284BEF12E0F07D87F
:1005F00094F82730082B03F06F840E2B03F06C84E3
:10060000312907D894F82730052B05F011870E2BD8
:1006100005F00E8794F82730112B05F06C87092B15
:1006200046F00B80BEF12F0F46F21D80312943F2B8
:100630008A84312802D80A2B06F0A280BEF1300F3E
:1006400045F23387312902D80B2B06F0C280BAF16C
:100650002F0F05F32D87072B05F02A87112B05F0A7
:100660002787444BDFF804914FF0000823F81580EA
:100670000320022389F80030F4F7EEFC3A4B187897
:10068000F0F7CEFF012299F8001020460AF0A2FFF1
:10069000702303FB0566384B327E1A70374B414698
:1006A000284683F80080F1F743F994F8271011B930
:1006B00020460AF057FC0320F0F7B2FF7B69013BAC
:1006C000013513F0FF03EDB27B617FF4D9AEBB6956
:1006D00053B9264C2378FF2B06D00120F4F7BCFC3D
:1006E000F5F7DEFBFF2323700320F0F799FF01F0FD
:1006F000D4B80B2C1E4E49D1B7F81C8020481FFAE5
:100700008AF50123424629460AF0A4F8002803F09E
:100710004F84DFF8749099F80040EF2C03F248847E
:100720000A34E4B240F2951089F80040F0F78DF8F1
:10073000214617F0CFFD348899F800003E3C009424
:1007400032231422FA21F0F734F8A3B281B2322214
:100750000C480AF0DDFA01F0A0B800BF4A88FF1F7C
:10076000B8BCFF1FCEC5FF1F2A88FF1F0188FF1FCF
:100770000888FF1F2EC4FF1FA0C5FF1FE88EFF1FA4
:1007800058B9FF1F80B9FF1F70C5FF1F0C2C40F028
:10079000A1810021BF48C04CC04D13F0B4F9B7F897
:1007A0001C802378BB611FFA8AF60123424631463A
:1007B000BA480AF04FF8814658B32378013BDBB2C0
:1007C000FF2B23701AD1B6490A788AB9B54B1B782A
:1007D0000B2B02D8013B237010E00C2020700C2B57
:1007E000A3F10D00087007D8013B23700A7003E0E5
:1007F000013A00230A702370F4F764FDEB896989DC
:1008000022782889194489B2BB69F1F7DFFA01F02F
:1008100044B801234246314605F114000AF01AF8A3
:10082000824620B323789F4A9D4910780A78013385
:10083000DBB29E18B042237006DC0B2881F80090D2
:1008400084F8009008D905E00C2B05D901320C235F
:100850000A702370F4F736FDEB89698922782889BC
:10086000194489B2BB69F1F7B1FA01F016B8012356
:100870004246314605F1280009F0ECFF8146002888
:100880003CD040F29F10EFF7E0FF022896BF411CDA
:100890005146C9B240F29F10EFF76AFF824907F153
:1008A000600019F020FD40F29F10EFF7CEFF1CF022
:1008B00057FD02460B4600204FF080411AF0CEF85B
:1008C0007A4B00221CF0C2FD1DF0B8F8022201464E
:1008D00007F1700019F08DFD002307F1700207F198
:1008E000600173480AF07AF807F1700019F0BBFC58
:1008F00007F1600019F0B7FC00F0CFBF01234246BA
:10090000314605F13C0009F0A5FF002800F08E807B
:10091000684CDFF8B8815F48DFF8B4A14FF6FF718B
:1009200013F0F1F8B8F8003022885A48CDF8049056
:10093000693B0B3A0B261BB212B24946009615F0E2
:1009400065FA22885348CDF80490213A0A25C82335
:1009500012B20F21009515F059FA22884D480A3A33
:100960004B4612B2052114F0A1FB53494948EFF759
:10097000BDFF49464FF48C70EFF7FAFE07F17000A7
:10098000F4F7BAFD07F17000FDF730FA8AF80000BD
:1009900007F1700019F067FC9AF80030002B00F0A6
:1009A0007C87B8F8003022883A48693B0B3A4946C0
:1009B0008DE840021BB212B215F028FA22883548A1
:1009C00000954FF4E3530B3A01934946782312B252
:1009D00015F01CFA22882F480A3A4B4612B205211C
:1009E00014F064FB35492B48EFF780FF2A460823B3
:1009F00007F170003249EFF775FD07F170012548E6
:100A000019F0ECFA07F1700019F02DFC228821484A
:100A100000954FF478430B3A019312B2782349467C
:100A200013F03EFBF4F74EFC00F037BF01234246C3
:100A3000314605F1640009F00DFF002803F06F83D3
:100A40004FF4E570EFF701FF002843F068831D497C
:100A500007F1600019F047FC1B4907F1700019F01D
:100A600042FC07F160014FF4FC6307F1700205F1ED
:100A7000640009F0B3FF07F1700019F0F4FB07F10F
:100A8000600019F0F0FB01214FF4E570EFF770FE04
:100A900000F003BF5CC6FF1FA0C5FF1F1CB9FF1FEE
:100AA000E88EFF1F06B9FF1F0626030000405F40C7
:100AB00044B9FF1F4488FF1F7D2D0300F325030069
:100AC00034C5FF1F152603001D2603000888FF1FDD
:100AD0002AC4FF1F0D2C40F09F84B7F81C80AF483C
:100AE0001FFA8AF601234246314609F0B3FEB8B137
:100AF000AB4C0023237020780130EFF7A6FEA94A03
:100B0000A94B1278187082429CBFFF221A701A7883
:100B1000A64B21781A700D20F5F7C2FB00F0BDBE80
:100B2000012342463146A24809F094FEB8B19C4CDC
:100B30000223237020780130EFF787FE994A9A4B01
:100B40001278187082429CBFFF221A701A78974B55
:100B500021781A700D20F5F7A3FB00F09EBE01234B
:100B600042463146934809F075FEB8B18C4C0323D8
:100B7000237020780130EFF768FE8A4A8A4B12789A
:100B8000187082429CBFFF221A701A78874B217816
:100B90001A700D20F5F784FB00F07FBE012342465A
:100BA0003146854809F056FEB8B17D4C04232370C8
:100BB00020780130EFF749FE7A4A7B4B12781870A3
:100BC00082429CBFFF221A701A78784B21781A70E3
:100BD0000D20F5F765FB00F060BE0123424631466B
:100BE000764809F037FEB8B16D4C052323702078A4
:100BF0000130EFF72AFE6B4A6B4B12781870824275
:100C00009CBFFF221A701A78684B21781A700D2049
:100C1000F5F746FB00F041BE0123424631466848E5
:100C200009F018FEA0B1604B5D4C197820785F4B3D
:100C30000139C9B201301970EFF79AFDFF210D207B
:100C4000F5F72EFB21780D20F5F72AFB00F025BEE5
:100C50000123424631465B4809F0FCFD90B1504CFF
:100C6000514B20781978514B01301970EFF780FD06
:100C7000FF210D20F5F714FB21780D20F5F710FB6F
:100C800000F00BBE0123424631464F4809F0E2FD19
:100C9000A0B1454B424C19782078444B0131C9B280
:100CA00001301970EFF764FDFF210D20F5F7F8FA18
:100CB00021780D20F5F7F4FA00F0EFBD012342464C
:100CC0003146424809F0C6FD80B1374A1378013BEE
:100CD000DBB2FF2B137002BF324B1B781370304B0B
:100CE0000D201978F5F7DCFA00F0D7BD0123424654
:100CF0003146374809F0AEFD88B12B4A29491378AF
:100D000009780133DBB2994213703CBF00231370A2
:100D1000234B0D201978F5F7C3FA00F0BEBD01236F
:100D2000424631462B4809F095FD044628B1FF2183
:100D30000D20F5F7B5FA00F0B0BD0123424631466B
:100D4000254809F087FD002800F08B80234A13789E
:100D50000133DBB21370062B1546214B88BF14708C
:100D60001A782B78934203D113B11C4A01331370C4
:100D70002B781C49012B07F1600003D119F0B3FA5D
:100D8000194948E0022B03D119F0ADFA174942E0A6
:100D9000032B2FD119F0A7FA15493CE01CB9FF1F0E
:100DA000EAC6FF1F2AC4FF1FA0C5FF1FE88EFF1F52
:100DB00044B9FF1F58B9FF1F6CB9FF1F48BAFF1F86
:100DC00080B9FF1F94B9FF1FA8B9FF1FBCB9FF1F4F
:100DD000D0B9FF1FF8B9FF1F30B9FF1F3C8DFF1FAF
:100DE000E8C4FF1F622603006E260300722603007C
:100DF00076260300042B03D119F075FABD490AE0E9
:100E0000052B03D119F06FFABB4904E0062B09D179
:100E100019F069FAB94907F1700019F064FA4FF452
:100E2000FC6308E019F05FFAB54907F1700019F0AA
:100E30005AFA46F22C3307F1600107F17002B1480B
:100E400009F0CCFD07F1700019F00DFA07F1600010
:100E500019F009FA297840F21710EFF789FC00F031
:100E60001CBD012342463146A74809F0F3FC8146E8
:100E7000002800F08A80A549A5480B7800785A1C04
:100E8000D2B290420A700C4602D108B102330B7004
:100E90002378A049062B82BF9C4B00221A7023782E
:100EA000012B07F1500008D119F01DFA9A4907F1FA
:100EB000600019F018FA994935E0022B08D119F0B1
:100EC00012FA954907F1600019F00DFA94492AE0E9
:100ED000032B08D119F007FA8F4907F1600019F0C8
:100EE00002FA90491FE0042B08D119F0FCF98A4955
:100EF00007F1600019F0F7F97E4914E0052B08D1DD
:100F000019F0F1F9844907F1600019F0ECF97A4918
:100F100009E0062B0ED119F0E6F97F4907F16000D0
:100F200019F0E1F9754907F1700019F0DCF94FF497
:100F3000FC630DE019F0D7F9774907F1600019F06B
:100F4000D2F96F4907F1700019F0CDF946F22C3350
:100F500007F1500107F1600200936B4807F170033D
:100F600009F084FD07F1700019F07DF907F16000C8
:100F700019F079F907F1500019F075F9217840F26C
:100F80001510EFF7F5FB00F088BC0123424631460F
:100F9000654809F05FFC002800F0D480634BDFF85F
:100FA000A0811D78624B98F800401A784FF6E073E4
:100FB00095422CBF1D464FF4FC65FF2C4FF4CD70BD
:100FC00046460AD1EFF741FC5A4988F8000007F17C
:100FD000600019F088F9514961E0EFF736FC84426E
:100FE00040F29B100AD1EFF730FC524988F800001C
:100FF00007F1600019F077F9494950E0EFF725FC57
:1010000084424FF4CE700AD1EFF71FFC494988F8AB
:10101000000007F1600019F066F942493FE0EFF780
:1010200014FC844240F29D100AD1EFF70EFC4149B6
:1010300088F8000007F1600019F055F92D492EE0FD
:10104000EFF703FC844208D13A4988F8009007F191
:10105000600019F048F9284921E04CB901233549CD
:1010600088F8003007F1600019F03DF9234916E0D7
:10107000012C09D109232F4988F8003007F16000BD
:1010800019F031F92C490AE0092C0ED10A2329491B
:1010900088F8003007F1600019F025F9274907F1B9
:1010A000700019F020F92B460EE0FF23214988F843
:1010B000003007F1600019F016F9114907F17000CE
:1010C00019F011F946F22C3307F1600107F17002B3
:1010D000154809F083FC07F1700019F0C4F807F116
:1010E000600019F0C0F831784FF49070EFF740FBD2
:1010F000D3E300BF7A260300B7210300B321030026
:101100008A28030030B9FF1FE4B9FF1FE8C4FF1F9E
:101110003C8DFF1F7E260300672603006E2603001A
:1011200072260300762603000CBAFF1F3F88FF1FBC
:101130002AC4FF1F89260300BB210300BF2103002F
:10114000BDC7FF1F012342463146C54809F082FB57
:10115000002800F0A280C34BC34D5E78C34B6C786F
:101160001A784FF6E07396422CBF1E464FF4FC6689
:10117000FF2C4FF4CD70A84609D1EFF766FBBC49B0
:10118000687007F1600019F0AEF8BA495BE0EFF75C
:101190005CFB844240F29B1009D1EFF756FBB44947
:1011A000687007F1600019F09EF8B3494BE0EFF763
:1011B0004CFB84424FF4CE7009D1EFF746FBAC49AB
:1011C000687007F1600019F08EF8AC493BE0EFF76A
:1011D0003CFB844240F29D1009D1EFF736FBA44955
:1011E000687007F1600019F07EF8A5492BE0EFF771
:1011F0002CFB844208D100239D496B7007F16000ED
:1012000019F071F89F491EE044B9012398496B70A9
:1012100007F1600019F067F89B4914E0012C08D130
:10122000092393496B7007F1600019F05CF8974946
:1012300009E0092C0DD10A238D496B7007F160007C
:1012400019F051F8924907F1700019F04CF8334643
:101250000DE0FF2386496B7007F1600019F043F839
:101260008C4907F1700019F03EF846F22C3307F173
:10127000600107F170027A4809F0B0FB07F17000D5
:1012800018F0F1FF07F1600018F0EDFF98F8011079
:1012900040F21F10EFF76CFAFFE20123424631469D
:1012A0007D4809F0D7FA002800F0F7827B4C2378BC
:1012B0006BB901237A49237007F1500019F013F834
:1012C000784907F1600019F00EF86A496EE0012BC9
:1012D0000DD102237249237007F1500019F003F871
:1012E000704907F1600018F0FEFF63495EE0022BD1
:1012F0000DD103236A49237007F1500018F0F3FF62
:10130000684907F1600018F0EEFF5C494EE0032BDE
:101310000DD104236249237007F1500018F0E3FF58
:10132000604907F1600018F0DEFF55493EE0042BEC
:101330000DD105235A49237007F1500018F0D3FF4F
:10134000584907F1600018F0CEFF4E492EE0052BFA
:101350000DD106235249237007F1500018F0C3FF46
:10136000504907F1600018F0BEFF47491EE0062B08
:101370000DD107234A49237007F1500018F0B3FF3D
:10138000484907F1600018F0AEFF40490EE0072B16
:1013900013D108234249237007F1500018F0A3FF2E
:1013A000404907F1600018F09EFF394907F17000CD
:1013B00018F099FF4FF4FC6312E0002338492370C2
:1013C00007F1500018F08FFF364907F1600018F060
:1013D0008AFF304907F1700018F085FF46F22C3380
:1013E00007F1500107F1600200932B4807F17003E9
:1013F00009F03CFB07F1700018F035FF07F16000C1
:1014000018F031FF07F1500018F02DFF217840F25D
:10141000FB10EFF7ADF940E2102C40F0768100238D
:101420002B703388313B534546DCFB69132B43DC7F
:101430001D4BFF221A701D4B01241C701C4B0220F7
:101440001C70F3F709FE03238BF80030F0F786FBDE
:10145000184B002108461C70F4F722FF1DE200BF64
:1014600020BAFF1F3F88FF1FBDC7FF1F2AC4FF1FF1
:10147000912603006E2603007226030076260300E1
:101480007A260300B7210300B3210300BB21030028
:10149000BF2103008A28030034BAFF1FE8C6FF1FDC
:1014A00099260300F52103000188FF1FD4C5FF1F03
:1014B000E9C6FF1F4288FF1FB7F81C80B2481FFA19
:1014C0008AF601234246314609F0C4F9054698B12F
:1014D00040F21B10EFF7B9F920B1012814BF002129
:1014E000032100E0012140F21B10EFF741F9FE213A
:1014F0001020F4F7D5FED0E1012342463146A3483F
:1015000009F0A8F9044688B1A14B33221A70A14B07
:1015100020225A726420F3F7C9FC7B691B683B6583
:101520009D4B3A6D1A609D4B1D70B6E101234246FA
:1015300031469B4809F08EF9054660B3944B9949B2
:1015400034221A70934B18225A7207F1600018F077
:10155000CAFE954907F1700018F0C5FE4FF6E0731A
:1015600007F1700207F160018D4809F037FA07F1C1
:10157000700018F078FE07F1600018F074FE642027
:10158000F3F794FC7B691B683B66834B3A6E1A60E9
:10159000824B1C7081E1012342463146834809F0A9
:1015A00059F9044660B37A4B814935221A70794B58
:1015B00014225A7207F1600018F095FE7A4907F17B
:1015C000700018F090FE4FF6E07307F1700207F11B
:1015D0006001764809F002FA07F1700018F043FE46
:1015E00007F1600018F03FFE6420F3F75FFC7B69B1
:1015F0001B683B67684B3A6F1A60684B1D704CE183
:101600000123424631466B4809F024F9054600287B
:1016100047D04FF4D770EFF718F9012820D12146B1
:101620004FF4D770EFF7A4F8634907F1600018F0A2
:101630005AFE624907F1700018F055FE46F22C334D
:1016400007F1700207F160015A4809F0C7F907F184
:10165000700018F008FE07F1600018F004FE1CE1AD
:1016600001214FF4D770EFF783F8534907F1600079
:1016700018F039FE514907F1700018F034FE4FF4AC
:10168000FC6307F1700207F160014A4809F0A6F90E
:1016900007F1700018F0E7FD07F1600018F0E3FDB6
:1016A000FBE0012342463146454809F0D3F80028C3
:1016B00000F0F3804FF48A70EFF7C7F8414C4249CD
:1016C0000230C0B21E28207007F1600088BF25706C
:1016D00018F009FE217807F1700018F024FE07F1D8
:1016E0006001002307F17002354809F077F907F12E
:1016F000700018F0B8FD07F1600018F0B4FD217813
:101700004FF48A70EFF732F8C7E00E2CDFF8D49070
:101710006AD13288313A002352452B701BDCFA69BA
:10172000132A18DC294A1370294BFF221A70294A00
:1017300001231370284A2B7013702B70022003238F
:101740008BF80030F3F788FCF0F708FA0021084620
:10175000F4F7A6FDA1E0B7F81C8016481FFA8AF638
:1017600001234246314609F075F8002802F07C86D4
:101770001A4C2378FF2B02F07786194B1A78012A2E
:1017800042F0728602F063BD1CB9FF1F30B9FF1F23
:10179000EAC6FF1F54C4FF1FCC8EFF1FBFC7FF1F29
:1017A00044B9FF1FA0280300A528030058B9FF1F54
:1017B000A92803006CB9FF1FE2240300AF2803002F
:1017C00080B9FF1FAAC6FF1FB5280300BCC4FF1FB6
:1017D0000188FF1FD4C5FF1FE9C6FF1FF18EFF1F41
:1017E000AFC7FF1FFD87FF1F0F2C56D1B74C2678C0
:1017F00096B907F17005B649284618F074FD0F2315
:101800000093B44802960195DC2323222D2109F090
:1018100089F9284618F027FD0021AF48AB4D12F09A
:1018200072F90121AC4812F068F92178AA4801EB5D
:101830004101490000232722323113F037FCB7F869
:101840001C80A6481FFA8AF601234246314609F059
:1018500001F8002803F0A2812B781F2B03F29E8150
:101860009F499D48EFF742F829789E4B31225A5400
:101870000131C9B229700A22C1F1200107F17000BB
:1018800018F064FD98484FF6E07207F1700109F016
:101890006FF807F1700018F0E6FC944B4FF4A0725B
:1018A0001A80934BF0221A80924B1B78012B06D1A1
:1018B000914A92499248EFF741F805F0F4BAC820EE
:1018C000F2F714F84FF4CC70EEF7BFFF03228D4906
:1018D000212888BFFF2016F0ADFC05F0E4BA0A2BE2
:1018E0001ED194F85830002B3DF4E3AA002D7DF46E
:1018F000E0AA854B1878A38B83427DF4DAAA0125F0
:10190000F3F742F9E58381498148EEF7EFFFE18B78
:101910007F48EEF7FEFFFDF7CCBA0A2B3DF4C9AACB
:101920000B2B7DF4C6AA94F85830002B3DF4C1AAC5
:10193000A38B092B05D1774A337812789A4233D199
:101940003BE00A2B04D1744932780978914234D0B3
:101950000A2B29D00B2B02D13278FF2A2DD00B2B4A
:1019600022D00C2B02D13278FE2A26D00C2B1BD091
:101970000D2B03D199F80020022A19D00D2B13D07A
:101980000E2B3DF496AA0F2B3DF493AA98F8002055
:1019900042FA03F3DB077DF58CAA40F21910EEF74B
:1019A00054FF50B9FDF785BA0023E383FDF781BAF0
:1019B0000123E3832384FDF77CBA0123F5E7122B8F
:1019C0000CD100238BF80030BB8B7B84A7F820A0C0
:1019D000524B386ABA8C18609A8090E10A2B1BD15E
:1019E000EB8B00228BF800208BB919464C4A1A4425
:1019F000703392F827000A2808BFD183B3F5EE6F41
:101A0000F4D1414B287F18700124EC8314E03E4B45
:101A1000EA83FF20187073E10B2B7DF4BAAAB5F8A6
:101A20001C80A8F10903032B0AD83E4B1B7803F056
:101A3000FD03012B7CD0FF20F3F738FAFDF7A9BA9C
:101A4000B8F10D0F00F00481B8F10E0F00F02681FF
:101A5000B8F10F0F00F0388140F21910EEF7F5FEE3
:101A6000002840F05281FDF794BA2F4CAA8B2178C0
:101A7000914201D1237001E0D2B22270217840F26C
:101A8000AB10EEF775FE0022254B2848114693F85F
:101A900027E0BEF1090F0BD193F858E0BEF1000F1B
:101AA00006D000EB020E9EF810E0BEF1000F0BD145
:101AB0001432B2F5AA7F03F17003E8D12378EB83E7
:101AC00000238BF800301AE1D983F1E70088FF1F6B
:101AD0002721030058B9FF1F5CC6FF1FE4B9FF1F91
:101AE00070260300C8C4FF1F94B9FF1F0888FF1F9A
:101AF0004488FF1FFD87FF1FA086010051080000DA
:101B0000408EFF1FF16E01004788FF1F882D0300E4
:101B10008C8AFF1FF8B8FF1FEEC9FF1FD4C7FF1F35
:101B2000B8BCFF1F6CC5FF1FF18EFF1F1CB9FF1F44
:101B30000023AF498BF80030184691F827200B2A74
:101B400007D1DAB2914504D08A8B093A92B2032ABE
:101B50007CD90133112B01F17001EED1A54BA98B7A
:101B60001B78A54CB5F81EE0002B14BF4FF4807015
:101B700000200B291AD1BEF1000F03D10123EB8302
:101B8000FF211DE09D4B00212170E98318809C4BB3
:101B90001A789C4BA82000FB02334FF000084FF04E
:101BA0000009C3E90E894FF4F170A6E00C294FF04B
:101BB000010C0FD1BEF1000F04D1A5F81EC0FE210B
:101BC0002170F0E78D4B18808F4B0021E98319803D
:101BD0002170DCE7894A8A4BBEF1000F26D1092922
:101BE0000CBF8A498A49A5F81EC091F8009093F865
:101BF00000801FFA89F1B8F1FF0F118008D0484624
:101C00001BF0AEFB7F4BA82202FB0838C8E90E018F
